:10AEAE00414952434F54454300404556332E3531A8
:10AEBE00404E4C20004143435500532F4E214641F6
:10AECE00494C555245005245454E54455221532F3B
:10AEDE004E00434F4E5441435420414952434F5428
:10AEEE0045430047505300403244400040334440F5
:10AEFE0000554954214E4557404D454E55000A16B2
:10AF0E00000180000300007E0000FE00001E000015
:10AF1E00360003E60001C4000000000FFFE0205AD7
:10AF2E004F454B40534154532000204750534056F9
:10AF3E00414C49442000504943545552450052411A
:10AF4E004E4B494E47004D415020202020200043BB
:10AF5E00454E544552202000564152494F20202044
:10AF6E00004241524F4752414D00524F55544553A6
:10AF7E0020200044494348545354450057415950EA
:10AF8E0054532020004D41524B5320202000444565
:10AF9E004641554C54002020202147454D2120206C
:10AFAE0020204146530020545241434B214F4E2006
:10AFBE00200020545241434B214F464620004D4124
:10AFCE00524B0020545241434B2D5550212000200E
:10AFDE004E4F5254482D5550212000215445525564
:10AFEE00470153454C40524F55544501534554204B
:10AFFE00484F4F47544501564C55434854454E68AB
:10B00E0069015741595054532020686901524F55D8
:10B01E0054455320206869014149525350414345DC
:10B02E00686901494E5354454C20206869014143DB
:10B03E0043454C45522E6869005A455420484F4F9F
:10B04E00475445004241524F40484F4F47544500E8
:10B05E0047505320484F4F47544500514E482020EB
:10B06E002020402148504100464C004C4F47424F53
:10B07E00454B204C45454720003E215445525547EF
:10B08E0000215445525547015350454C454E015AE7
:10B09E00454E440157495353454E00215445525590
:10B0AE004701434F4D3A20202020202001544E438B
:10B0BE002031232035374B01544E43203123203984
:10B0CE002E360101505743403130234035374B0166
:10B0DE00505743403130234031394B01014D5850C8
:10B0EE00403130234035374B014D5850203423200A
:10B0FE0035374B014D58502031232035374B014DFC
:10B10E005850403130234031394B014D5850203189
:10B11E00232031394B00215445525547014E4945A4
:10B12E0055572057505420014544495420574159F2
:10B13E00505401574953202057415950540101434F
:10B14E004F4D3A014F4E5456414E47205750015ADB
:10B15E00454E44205741595054015A454E444041A2
:10B16E004C405750200101414653542057502D5703
:10B17E00500157495340414C4057505420005045C0
:10B18E004920214146535400534156452000414326
:10B19E005455454C4540504F532E004F50534C4143
:10B1AE00414E202020002053544F524521575054D9
:10B1BE0020002046554C4C20002140574953534502
:10B1CE004E005345522000495244410055534220EF
:10B1DE000055534220004C495354005A454E4400EA
:10B1EE00205452414E534D4954204552524F5220F5
:10B1FE00002154455255470153454C40524F55542A
:10B20E0045014E4945555720525450200145444959
:0DB21E005420524F555445014F4D4B4552A1
:10B22B00454E205254015749532020525450202050
:10B23B00015749532020524F5554450143594C2037
:10B24B0052414449555301434F4D3A014F4E5456C9
:10B25B00414E47205254015A454E4420524F5554AB
:10B26B004501434845434B2052540053454C215212
:10B27B004F555445004E4945555700204E574540B4
:10B28B00504F5340210021404F4D4B4552454E40AE
:10B29B00004F4D4B454552002140574953405750A5
:10B2AB00545300214057495320525445004E4945B1
:10B2BB0054204C454547200021405A454E444052AE
:10B2CB0054450020205241444955530021544552C6
:10B2DB005547014C4F414440435452215043015672
:10B2EB00494557404354520144454C40414C4C2135
:10B2FB004354520101434F4D3A01524543562020CE
:10B30B004354520153454E44202043545200564956
:10B31B004557204354520020204D4F5645002020C6
:10B32B004D4F564520544F005343414C4520205818
:10B33B002F5920204558495400434C52204449531F
:10B34B0054004155544F43454E54004155544F20E2
:10B35B004F4646002020205343414C45004449535F
:10B36B0054204B4D0044495354204E4D002154451D
:10B37B0052554701564152494F20202068690158C8
:10B38B00432D53455420206869015254452D534594
:10B39B00542068690147454E4552414C206869016C
:10B3AB005049435455524553686901010145415376
:10B3BB00592D53455401464143544F52595345540B
:10B3CB00210144454D4F464C4947485400215445B3
:10B3DB005255470153494E4B544F4E450153494E1D
:10B3EB004B212D0153494E4B404D4F440153494E78
:10B3FB004B40494E56015641522054434020204069
:10B40B002301564F4C554D4501564152494F204E45
:10B41B00554C4C01504954434801504552494F44F7
:10B42B00015641522041564020304023014E455495
:10B43B00544F2D01534F554E44434845434B0053F6
:10B44B00494E4B21544F4E450053494E4B54214FBF
:10B45B004646004745454E204455414C2000564139
:10B46B0052494F204E554C4C0020574143485440B5
:10B47B003130404D494E2020202000564F4F522056
:10B48B004E554C4C494E47202000215445525547B0
:10B49B000153504F4F52202020014155544F4345EB
:10B4AB004E54010147454D2F4146535401474C49DA
:10B4BB004A50414420014C2F44010157494E44212D
:10B4CB00542D55500143454E5421542D5550015781
:10B4DB00415950542142524700215445525547017E
:10B4EB0053544152544054494D45014649525354CB
:10B4FB000144454C544120203A014D554C54495080
:10B50B004C45014C4153540143594C53494740203E
:10B51B002040230153454C40524F555445010101E6
:10B52B000143594C520143594C20542D5550002185
:10B53B005445525547010145454E4801434C49433B
:10B54B004B40302C40202301434F4E545241535417
:10B55B00014E4D45412131383301494D50454C4C3D
:10B56B00455201494D502D43414C01432D564152FB
:10B57B00494F0154454320202040303040250141A4
:10B58B00004E4F20414750532F464C00414C5449DD
:0DB59B002D475053202000464C47542D4CA6
:10B5A8004556454C0041475053203C3E20464C00F0
:10B5B8002057414954004E4F20464C4947485400B3
:10B5C8004045584954204C4F47403F40004D4D2E70
:10B5D80059590020606869003C2D20202020202D2A
:10B5E8003E2020202053454C003C2D2020202020A8
:10B5F8002D3E20202045584954003C5245432020E8
:10B608005245433E20202053454C00522D4F46467C
:10B6180000202052454300414343454C4552415484
:10B628002E00472D554E4954530021544552554735
:10B63800015245434D4F4445202058015245432E61
:10B648002031352F23015245432E2036302F230138
:10B658005350454C452F5A454E440157495353457D
:10B668004E40414C2001434F4D3A01014E554C4C40
:10B67800494E470058593A204B4545500020484FFD
:10B6880052495A4F4E54414C005A3A20204B454596
:10B6980050004F4E204544474500585920205A2015
:10B6A800404558495400205C2020202053454E44F2
:10B6B8000040575054204245535441415420414C76
:10B6C8004000574159504F494E540020205445528C
:10B6D80055472021004F4E5456414E470056524977
:10B6E8004A40003C2D204C495354202D3E202045F3
:10B6F8005849540053454C004E455854004E45583F
:10B70800542054505400505245562054505400432D
:10B718004C5220404C454700434C52204053554D15
:10B728000055495420202020202020200020554961
:10B73800540047505320464F555420004F50534C07
:10B7480041414E00524F55544500444943485354D3
:10B75800004C495354200045544500414C54403056
:10B76800004C4547452052544520200020544F4F57
:10B77800404D5543482000214053454C404C4953C7
:10B7880054002053454C4057505440210021404F0D
:10B798004E5456414E4740002020404F204B4020F9
:10B7A8002021004F4B00564152004649580047415E
:10B7B800544521580053544152544C4E20202000E7
:10B7C800535443594C2000405549540054502000CC
:10B7D800406A40494E20004067404F5554002020A1
:10B7E800464F5554202021002045584954004544CF
:10B7F800495400404A4041004544495420204E45A0
:10B808005720534C41204F50004E45585420534523
:10B818004C4543542045584954005843542D464CF0
:10B828004947485420005553454400454E54455215
:10B8380020004D4D2E4D4D4D20004D4D2753532E7C
:10B848005300574753213834002040554054404D49
:10B85800402000554054404D002055544320004C92
:10B868004F43414C005357495353474400414C54AC
:10B878000053554940580041564740203040230066
:10B88800353030003136343000205D203130404BC7
:10B89800632F70005D2020203140632F2300205D3E
:10B8A800202035404B5453005D2032303040465004
:10B8B8004D00406340204B63004654204B630040DA
:10B8C8006340204E4D004654204E4D004D2F5300EE
:10B8D8003230305E003530305E00312200322200D6
:10B8E800332200352200382200464C3700464C31BE
:10B8F8003600464C333300464C363500463130303E
:10B9080000463136300046323630005E2526405338
:0DB918004F47005E25264054415300414C2E
:10B92500540056415200225E2F24004B54530053BD
:10B935002F4E002224004B5400225E004E4D003055
:10B945002C3500312C3000322C3000302C360031B3
:10B955002C3200322C3500332C3800372C35004082
:10B9650031350040333000403630005441534B00F0
:10B97500464C2D4441544500545000544F46005305
:10B9850054410046494E004C414E00534554204F0A
:10B995004646534554004953412048454947485474
:10B9A500004155544F2D474F2000535441525400E8
:10B9B50020434845434B40414C4C005241442044B0
:10B9C500495354004053454C404845494748543A2B
:10B9D50000475053404241524F40414C4C0053495F
:0BB9E5004E4B40312D3221632F230018
:1073B900304D2475A7049005C2E0F51CE0F51DE0E9
:1073C900F51EE0F51FE0F56DE0F56EE0F56FE0F50F
:1073D90054127F7B1279B92275C70375C6E475B952
:1073E90001E5BCB48143127F7B1265938E628F6382
:1073F9007568F975690012748F203C2D203B2B129A
:1074090075C4127598856D1C856E1D856F1E855412
:107419001F1274FB203C12203243201D231275C415
:107429001279B9E532242850DC221274FB203CF988
:10743900203DF6203205201DBD80EF301DB880EAC1
:107449001275C41279B9856D1C856E1D856F1E85EF
:10745900541F1275AE1279B9203DCE80991277E783
:10746900201D0D755310740012774A203DBB80868C
:10747900E553540FC553C4540F20350512765F8068
:107489000312774A808BC23CD23B12754BFD1275B1
:107499004BFC12754BC39573F565EC9574F564ED6A
:1074A9009575600504600A800EE56424E05011803A
:1074B90006E5642420400912754B12754B02754B81
:1074C90012754BFD12754BFC12754BC39576F5671A
:1074D900EC9577F566ED9578600904600122E5661B
:1074E900F48002E5668562F0A474E025F04002C2EA
:0D74F9003B22C23C12754BA2E7923DA2E679
:10750600921DA2E592324026A2E492E592E692E727
:10751600FC12754B2565F565EC3564F56412754B03
:10752600FC12754B2567F567EC3566F56622A2E415
:107536009235540F79C6F712754B09F7301D0512AF
:10754600754BF55322E5697023E5686030240440E5
:107556002CE56875F004A485F0C7F5C675B901E594
:10756600BCB4811985BD68756902801E540370100C
:1075760005C675B901E5BC056953690F22D23C22DF
:10758600147004E5BD80F0147004E5BE80E9E5BF23
:1075960080E575A7009006F6E56DF0A3E56EF0A30D
:1075A600E56FF0A3E554F02275A7009006F6E0F526
:1075B6006DA3E0F56EA3E0F56FA3E0F55422E56454
:1075C600B2E7F56D85656EAB67E566FC30E707C328
:1075D600E49BFBE49CFCAA62A96312628DE566301B
:1075E600E707C3E49DFDE49EFEEEB2E7F56F8D541A
:1075F6002275380C12785012789BD55301227538B3
:107606000C127821127891D5530122753800127820
:0E76160039127860D5530122753800127821A0
:10762400127860D55301227538031278501278CC41
:10763400D55301227538031278211278C2D553012B
:107644002275380F1278391278F1D5530122753822
:107654000F1278211278F1D5532622907664237381
:107664008091807780688059804A803B802C801D7F
:10767400800E80DA80CB80BC80AD809E808F80803D
:10768400753815127850127913D5530122753815AF
:10769400127821127908D5530122753809127839E4
:1076A4001278D9D55301227538091278211278D964
:1076B400D5530122753806127850127883D55301B8
:1076C40022753806127821127878D553012275383C
:1076D400121278391278A9D553012275381212780A
:1076E400211278A9D55301220275F775381512783D
:1076F40050127913D553012275380F12782112785C
:10770400F1D553012275380F1278391278F1D55317
:1077140001227538031278211278C2D553012275DB
:1077240038031278501278CCD553012275380012E0
:107734007821127860D553012275380012783912F5
:107744007860D553262290774F2373809E80A9803A
:10775400B480BF80CA80D580E08010801B802680E2
:1077640031803C80478052805D806875380C127887
:1077740021127891D553012275380C127850127861
:0E7784009BD55301227538121278211278A974
:10779200D55301227538121278391278A9D55301BE
:1077A20022753806127821127878D553012275385D
:1077B20006127850127883D553012275380912784F
:1077C200211278D9D55301227538091278391278E5
:1077D200D9D5530122753815127821127908D5535B
:1077E20001220276EF78C686040886037AED1262D9
:1077F2004B78CAA60408A60378C686040886037ACC
:107802006212624B78CCA60408A60378C6860408E6
:1078120086037AB512624B78C8A60408A6032275BD
:107822001A6A751B0A78CA8618088619127A647849
:10783200CC86060886072278C88618088619E4F5D9
:107842001AF51B127A6478C886060886072278C65B
:107852008618088619751A00751B01027A64E51DDF
:107862002519F51DE51C3518F51CC3E51F9FF51FED
:10787200E51E9EF51E22C3E51F9FF51FE51E9EF520
:107882001EC3E51D9519F51DE51C9518F51C22E58D
:107892001D2FF51DE51C3EF51CC3E51F9519F51FAF
:1078A200E51E9518F51E22C3E51D9FF51DE51C9EDC
:0978B200F51CC3E51F9519F51F33
:1078BB00E51E9518F51E22E51F2FF51FE51E3EF55B
:1078CB001EE51D2519F51DE51C3518F51C22C3E514
:1078DB001D9519F51DE51C9518F51CE51F2FF51FBA
:1078EB00E51E3EF51E22E51D2FF51DE51C3EF51C84
:1078FB00E51F2519F51FE51E3518F51E22C3E51DDD
:10790B009FF51DE51C9EF51CE51F2519F51FE51EB2
:10791B003518F51E22E51A7009E51B70058C068DCE
:10792B000722ED851BF0A4A2F792D5ED851AF0A4E2
:10793B00AEF0FFEC851BF0A4A2D53FEE35F0FF9225
:10794B00D5EC851AF0A42FFFE435F030D50104FEF9
:10795B0022E4F51AF51BEF4E7003051B22EF651998
:10796B007006EE65187001227808C3EF33FFEE3313
:10797B00FEEF9519F5F0EE95184003FEAFF0E51A02
:10798B0033F51AD8E5F4F51A751BFF7805C3EF33F9
:10799B00FFEE33FEEF9519F5F0EE95184003FEAFB1
:0379AB00F0E51BE9
:1079AE0033F51BD8E5F4C403F51B22E51D9511E54F
:1079BE001C9510500BE56E9511E56D95105001223A
:1079CE00E51F9511E51E9510500BE5549511E56FC9
:1079DE009510500122E51D9513E51C9512400BE5FF
:1079EE006E9513E56D9512400122E51F9513E51E68
:1079FE009512400BE5549513E56F951240012253F5
:107A0E002CF8C3E51F9554FFE51E956FFE9260504E
:107A1E0007C3E49FFFE49EFEC3E56E951DF519E5D1
:107A2E006D951CF5189261500BC3E49519F519E488
:107A3E009518F518C3E5199FE5189E9262500AE550
:107A4E0018CEF518E519CFF51912795CE52C540707
:107A5E0075F003A4F538E538907A6A73027A8202DB
:107A6E007A96027AA4027ABC027ACF027AE2027A7B
:107A7E00F0027B08851C16851D17C3E4951FF515AE
:107A8E00E4951EF514027B1B851C16851D17851E9D
:107A9E0014851F158077C3E4951DF517E4951CF525
:107AAE0016C3E4951FF515E4951EF514805FC3E427
:057ABE00951DF517E421
:107AC300951CF516851E14851F15804CC3E4951F60
:107AD300F517E4951EF516851C14851D158039854B
:107AE3001E16851F17851C14851D15802BC3E49551
:107AF3001FF517E4951EF516C3E4951DF515E495DA
:107B03001CF5148013851E16851F17C3E4951DF5F8
:107B130015E4951CF5148000C3E5179513E5169538
:107B23001210D70122E5159513E514951210D7010C
:107B330022E519F92517FFE518F83516FED3EF9559
:107B430011EE9510500122E5119517FDE5109516DC
:107B5300FC402A4D6027127920E5152FF515E51411
:107B63003EF514E5159513E514951210D70122E59A
:107B7300199DF9E5189CF8851016851117E5172945
:107B8300FFE51638FEE5139FE5129E500BC3E51380
:107B93009517F9E5129516F8E51A700AE51B7006B4
:107BA300AA00AB018013E9851AF0A4E5F0FBE88590
:107BB3001AF0A42BFBE435F0FAE5152BFBE5143A98
:067BC300FAE5119BE5103C
:107BC9009A10D70122EB9515FDEA9514FCC3E5152A
:107BD9009511E514951010D717E5139BE5129A50E6
:107BE90036E5139515FFE5129514FE127E98802748
:107BF900EB9511FFEA9510FEAA00C001127E98D0FC
:107C090003E5172BFBE5163AFAEB99F517EA98F510
:107C190016851115851014C2D5E5466002D2D5AA7C
:107C290056E98AF0A4ABF0E88AF0A42B30D50475A4
:107C3900F00384F8700122E5172513FDE5163512C6
:107C4900FCED8AF0A4ABF0EC8AF0A42B30D50475D6
:107C5900F00384FEE5152513FDE5143512FCED8AC4
:107C6900F0A4ABF0EC8AF0A42B30D50475F00384B2
:107C7900F9E538907C8073027C98027CA4027CAD83
:107C8900027CB6027CBC027CC8027CCF027CD4C3D5
:107C9900743E9EFFC3743E99FE8032C3743E9EFFBC
:107CA900AE018029AF06C3743E99FE8020AF06AEAF
:0D7CB90001801AC3743E9EFEC3743E99FF05
:107CC600800EC3743E99FF8007C3743E9EFEAF01CB
:107CD60008EF2437FFE51B7007E51A700CE8800EE5
:107CE600A2E7E51A50030460F488F0A4E5F0600109
:107CF60004F923FA98FBC3E998C333F9907D08E5A4
:107D06003873027D20027D4D027D82027DAF027DA9
:107D1600DC027E09027E36027E6305A7800BEB300D
:107D2600E7032A8002291E1FFBEEC45403F583EEE7
:107D36005408C42FF582EE5407243883F5F0E04545
:107D4600F0F0D8DA05A72205A7800BEB30E7032A67
:107D56008002290E1FFBEEC45403F583EE5408C4BB
:107D66002FF582EE5407240B83F5F0E045F0F0D8AA
:107D7600DA05A722804020100804020105A7800B1F
:107D8600EB30E7032A8002291E0FFBEEC45403F5ED
:107D960083EE5408C42FF582EE540724EC83F5F0E5
:107DA600E045F0F0D8DA05A72205A7800BEB30E70F
:057DB600032A800229F0
:107DBB000E0FFBEEC45403F583EE5408C42FF5826B
:107DCB00EE540724BF83F5F0E045F0F0D8DA05A7B1
:107DDB002205A7800BEB30E7032A8002291F1EFB2D
:107DEB00EEC45403F583EE5408C42FF582EE54070A
:107DFB00249283F5F0E045F0F0D8DA05A72205A729
:107E0B00800BEB30E7032A8002291F0EFBEEC454D4
:107E1B0003F583EE5408C42FF582EE5407246583D3
:107E2B00F5F0E045F0F0D8DA05A72205A7800BEBBB
:107E3B0030E7032A8002290F1EFBEEC45403F5839F
:107E4B00EE5408C42FF582EE5407243883F5F0E086
:107E5B0045F0F0D8DA05A72205A7800BEB30E70336
:107E6B002A8002290F0EFBEEC45403F583EE54084F
:107E7B00C42FF582EE5407240B83F5F0E045F0F0A8
:107E8B00D8DA05A7228040201008040201EC701FED
:087E9B00ED20E740D2E023CF07
:107EA30023CF30E7F980357B08801A7B1080167B5F
:107EB3002080127B40800E20E4ED20E3EE20E2EFF1
:107EC30020E1F07B80EE8BF0A4CF8BF0A4E5F02FC4
:107ED300FFEC8BF0A4CD8BF0A4E5F02D2499838FD8
:107EE300F0A433E5F033FBE98BF0A4E5F0C88BF0A5
:107EF300A428F9E435F0F822FFFEFCFAF8F6F4F2D0
:107F0300F0EFEDEBEAE8E6E5E3E1E0DEDDDBDAD92D
:107F1300D7D6D4D3D2D0CFCECCCBCAC9C7C6C5C48B
:107F2300C3C1C0BFBEBDBCBBBAB9B8B7B6B5B4B3A5
:107F3300B2B1B0AFAEADACABAAA9A8A8A7A6A5A491
:107F4300A3A3A2A1A09F9F9E9D9C9C9B9A99999855
:107F53009797969594949392929190908F8F8E8DFC
:107F63008D8C8C8B8A8A8989888787868685858488
:107F7300848383828281818075A700907FA1E546F7
:107F8300FA24FA50027A05EA2323F978107F04933E
:107F9300F60809E9DFF9907FB9EA93F556227FC223
:107FA300803E7F4680BA7E8C81747D1882E87A3069
:107FB30085D074608BA0808040201008127FC5029A
:107FC300821BD215D274D273C219C23A1265938E30
:107FD30047757D0075460575520212AE4B12020CB1
:107FE300E53524EB500E12AE4B7F1990B344128546
:107FF300B512F251E55275F016A4F5701281D175E0
:108003007E1512809C7F237E0990B3221285C712AE
:10801300F25110000810010D10021280E212814487
:1080230075330180DA12818975330180D2757E0040
:1080330012809C7E0090B3331285FA7F237E0590D5
:10804300B3291285C71280ED12F251E55210000FC9
:1080530010010510028780D5045403F55280CE1217
:10806300809C7F237E0B90B3611285C7E546600732
:1080730014600414124E9A12F251E54610000810CF
:10808300010B10021180D860D6154680D2B40502C8
:1080930080CD054680C9027FE075320012F39E7FD2
:1080A300017E1190B3191285FA7E0012EA87E57EEC
:1080B300D26612EADE75170812EF14124ED97571E3
:1080C30000C20612EC2E741BFFF5177E0F90B368E7
:1080D300305D0390B3701285FA12AE8E126BC41228
:1080E300543FC2061273E10229EEE5526014146094
:1080F3001E1460297F647E2D791C1281371E1FD9BF
:10810300F9227F6A7E1F79281281371FD9FA227FCD
:10811300487E2D791C1281370F1ED9F9227F567E96
:108123003379281F12F2E30F0F12F2E31F12F2E367
:108133001ED9F0221E12F2E30E0E12F2E31E02F219
:10814300E3E552605514606814606D800075709E9D
:108153001281BE8003757000E5732540F573E43525
:1081630074F574E43575F5752275701612815B80AC
:108173000375702DE5762542F576E5773541F5777C
:10818300E43578F57822E55260CB1460DC1460E1C5
:108193008000757044128177800375705AE573957A
:0981A30040F573E5749400F574D5
:1081AC00E5759400F575227570711281A0800375C8
:1081BC007088E5769542F576E5779541F577E57823
:1081CC009400F57822E5469081E793F540FEAD47A3
:1081DC00E4FFFC1263208E418F4222020C183060A7
:1081EC00C07F40121A1D122A0412F251128496EB0F
:1081FC00700590B080800B1282A490B7A0500390B1
:10820C00B7E67F3F7E041285C712F25112F20612B6
:10821C00F24775370990B2D71228E590822B73027A
:10822C00026D0283EB027FBF0284C702821B0282B3
:10823C004302825C0281ED7F2E12227080D17F3648
:10824C007E0490B7741285C712F25112F20680BFE9
:10825C007F37121A1D122A0412F25112847A125507
:10826C00CFD2AC1000A9306DFA128354203BCF4012
:10827C00ED7568F97516001283A140FB12853D7FE0
:10828C00367E29E51612E86512F251051612866C37
:10829C0078C6B6F7E20284747C051255CF12F0AAA8
:1082AC00744112F0BB745312F06BEB12F0991286FE
:1082BC007E5003DCE5227515F975160010000EE5ED
:1082CC001560251282F6400512831D5002D3227FC1
:1082DC003F7E29E51612E86512F2517F1412F21D49
:1082EC000516E51664F870D4C322128C3F75B901DB
:1082FC00E5BCB4811AE5BDF51570037516F778C6A3
:0B830C00A616128D88128D80128D8045
:10831700C3028D80D3227F0575F019D5E0FDD5F016
:10832700FA1255CF12F0AA744112F0BB744212F040
:108337006B7E0F78C6E60812F06BDEF912F09C121E
:10834700867E400122DF012275F00080CEC23B12FB
:1083570055CFD2AC12F0E3204C3CB440F712F0E812
:10836700B4400312F0E8B4412DF53812F0E8B453E5
:108377002512F0E8FA12F0E8E538701A12F0E8B4BE
:108387000D1412F0E8B40A0EC3E5169A40030286EC
:1083970063C2ACD23B22C2ACD3221286C21255CFE3
:1083A700D2AC1000F112F0E3204CEBB440F412F021
:1083B700E8B4400312F0E8B441DCF53812F0E8B451
:1083C70042D47E1078C612F0E8F608DEF9E5387078
:1083D700C512F0E8B40DBF12F0E8B40AB9C2ACC3D5
:1083E7002202821B7F0A121A1D122A0412F251124C
:1083F700847A1255EBD2AC1000E712F0E8B440F5DE
:10840700F53812F0E8B46EED12F0E8E538600A12BC
:1084170055EB744F12F07780DC1255EB744012F075
:10842700BBE51612F07712F0877568F9751600121A
:1084370055EBD2AC10003912F0E8B440F7F538121A
:10844700F0E8B44EC07E1078C612F0E8F608DEF900
:108457001255EBE5386007744F12F07780D112851B
:108467003D0516745112F07778C6B6F7C21284DA52
:0C84770002821B751500751603128C366E
:1084830075B901E5BC30E70205160515E51524208D
:1084930050EB227B007515F9128C3F75B901E5BCD1
:1084A300B481010B0515E515240450EC7515011273
:1084B3008C3675B901E5BCB481010B0515E51524AE
:1084C3002050EC227F1C121A1D122A4E40067515ED
:1084D300F91284DA02821BE51560372404401A245A
:1084E3001E5019E515240740028027128C3F128580
:1084F300160515E515240450F2751501128C367511
:10850300B901E5BC30E7031285160515E5152420EE
:1085130050EA2212852B1257AF05C61257AF05C674
:108523001257AF05C60257AF74FF8005740480016C
:10853300E4F5BCF5BDF5BEF5BF22E568606AF51547
:108543000515E5152404501D751501128C3675B9F2
:1085530001E5BC30E70280190515E515242050EB31
:10856300751500800C241C60F750E0E515240650B7
:1085730037E56875F004A485F0C7F5C675BC81E5D9
:1085830015F5BDF56878C6B6F70375BD0008128505
:10859300A012859A12859A86BC0886BD0886BE08F5
:0985A30086BF081257AF05C6227D
:10D4D90012CD9E12D5D812914112D55D12914912E1
:10D4E900D56A02CDA212CD9E12D5D81291417F5A8A
:10D4F900C23C12902312921F783F79437F607EEAE3
:10D5090012D5CC1291497F6512902312921F783D52
:10D5190079417F207E4E12D5CC303C2012D78E1215
:10D52900D5E9783F794312D548783D794112D548F4
:10D5390012D78E78D7E65480F675370002BBA2C39E
:10D54900E796FF1819E796FE0809C3E69FF7181929
:10D55900E69EF7227F5B7E0690B8791285FA1F80D6
:10D569000A7F667E14745912E9801F128EAC7E39C7
:10D57900E402E99F7866E620E73418C3E694720866
:10D58900E694045029C318E6941F08E69404401E43
:10D599007869E620E71818C3E6940E08E694015066
:10D5A9000DC318E6947508E694004002D322C322FD
:10D5B900E67D0030E7011D08E62BFB18E63CFCE49C
:0ED5C9003DFD22C3EB9FF6F71819EC9EF6F716
:10D5D7002212D57D400CE47842F608F67840F6082A
:10D5E700F6227864C3E6946AF55708E6944CF55634
:10D5F7000808C3E69458F55B08E694AEF55A753902
:10D6070000AC56AD57EC12D14B784C12D1D9AC5A6D
:10D61700AD5BEC12D14B785012D1D97F2B7E867D32
:10D62700777C1812D110785012D1CD12D01C12D19C
:10D6370010785012D1CD12D01C12D110785012D1BF
:10D64700CD12D01C12D1107F367E847D257C6412CA
:10D65700D110785012D1CD12D01C12D110784C12A3
:10D66700D1CD12D01C12D1107F3F7EA27D607C8B62
:10D6770012D110785012D1CD12D01C12CE0A12CE70
:10D687000A12D1E57F3F7E807D057CE6053912D001
:10D697001C784812D1D97F2C7E937D477C7F12D18D
:10D6A70010785012D1CD12D01C12D110785012D14F
:10D6B700CD12D01C12D110784C12D1CD12D01C1221
:10D6C700D1107F357EB47DF87CDF12D110785012EF
:10D6D700D1CD12D01C12D110785012D1CD12D01C3E
:10D6E70012D1107F3F7EED7D227CCD12D110784C78
:10D6F70012D1CD12D01C12CE0E12CE0A784412D1FE
:10D70700D97F317E397D9D7CE712D110784C12D1BB
:10D71700CD12D01C12D110784C12D1CD12D01C12C0
:04D72700D110784461
:10D72B0012D1CD12CE0E12D1107F2C7E377D0C7CF8
:10D73B00A312D110784C12D1CD12D01C12D110786B
:10D74B004C12D1CD12D01C12D110784C12D1CD125B
:10D75B00D01C12CE0E12D1E57F3F7E807D027C9FC6
:10D76B00053912D01C784412D1D9784812D1CD1278
:10D77B00D1828E428F43784412D1CD12D1828E400A
:10D78B008F4122753900AC42AD43EC12D14B784836
:10D79B0012D1D9AC40AD41EC12D14B784412D1D956
:10D7AB007F2B7E537D507C0912D110784812D1CD3E
:10D7BB0012D01C12D110784812D1CD12D01C12D11C
:10D7CB0010784412D1CD12D01C12D1107F347EF2BE
:10D7DB007DCD7CA312D110784812D1CD12D01C1262
:10D7EB00D110784812D1CD12D01C12D1107F3F7EB0
:10D7FB000A7D2E7CAE12D110784412D1CD12D01CE2
:10D80B0012CE0A12CE0A784C12D1D97F2B7E4F7DC5
:10D81B00AF7CB212D110784812D1CD12D01C12D1DC
:10D82B0010784812D1CD12D01C12D110784812D1D9
:10D83B00CD12D01C12D1107F357EB17D4B7C951251
:10D84B00D110784812D1CD12D01C12D110784412BD
:10D85B00D1CD12D01C12D1107F3F7E497DCD7C459E
:10D86B0012D110784812D1CD12D01C12CE0E12CE7E
:10D87B000A785012D1D9784C12D1CD12D1828D5554
:10D88B008E568F57785012D1CD12D1828D598E5A18
:04D89B008F5B7864C3
:10D89F00E557246AF608E556344CF608E555340486
:10D8AF00F608E55B2458F608E55A34AEF608E43579
:03D8BF0059F622F5
:10B9F00012CD9E12C08112CDA27F6690B85B1285D7
:10BA0000F812BA5E7F5A78C412BA3A12BA4278C6AD
:10BA100012BA3A12BA257F6578C812BA3A12BA42F7
:10BA200078CA12BA3A7E2DE51B12E99F7E33E51AD9
:10BA300012E99F7E39E51902E99F86040886030210
:10BA400061EA7E15E51C12E99F7E1BE51B12E99F4A
:10BA50007E21E51A12E99F7E27E51902E99F7F5AA8
:10BA60007E01E53A12E8B37E0B90C475E53B930284
:10BA7000E9B2E6FF08E6FE08E6FD339217E450015E
:10BA8000F4FC12D1F675130A75390112D3F478D784
:10BA9000E6C2E775F00A84F9303D02A9F012D1F64A
:10BAA0008913053912D3CD30170A053912D3E005B1
:10BAB0003912D3E0A80302D1D912CD9E12C081C29F
:10BAC0003C7F5A7E031293D012BA5E12F2511000DC
:10BAD0000810011510022080EFE53A146004153AB1
:10BAE0008003753A3CD23C80DFE53AB43C05753AB8
:10BAF0000180F2053A80EE7E031293CB7E0B129307
:10BB0000D012BA5E12F25110000810011510022076
:10BB100080EFE53BB40205753B158002153BD23C36
:10BB200080DFE53BB41505753B0280F2053B80EEF6
:10BB30007E0B1293CB7F5A78C412BA3A12BA4212D1
:07BB4000BBAB12922F78C489
:10BB470012BC0378C612BA3A12BA2512BBDD751CAD
:10BB57000012922F78C612BC037F6578C812BA3AD2
:10BB670012BA4212BBAB12922F78C812BC0378CA22
:10BB770012BA3A12BA2512BBDD751C0012922F7841
:10BB8700CA12BC03303C14E53B24F4500B78C9E6D9
:10BB97002410F618E63427F612BC0912CDA2128D2E
:10BBA700B102F251C2247E15E51C129320F51CD276
:10BBB700247E1BE51B129320F51B1023E77E21E54E
:10BBC7001A129320F51A1023E67E27E519129320FF
:10BBD700F5191023E822C2247E2DE51B129320F5C8
:10BBE7001BD2247E33E51A129320F51A1023E77E21
:10BBF70039E519129320F5191023E622ECF608EB24
:10BC0700F62212C48D78C8E6FE0886073395E0FD54
:10BC1700FC12D1107FE87E037D007C0012D3F41262
:10BC2700D11078CAE6FE0886073395E0FDFC12D3EB
:10BC3700CD12D1107F807E697D677CFF12D3CDEC5A
:10BC470012D14712D1107F3F7E807D0D7C1D12D00F
:10BC57001C12D1107F3D7E407D007C0012D11078F0
:10BC6700BC12D1CD12D01C12D1107F3E7E807D0038
:10BC77007C0012CE0E12D11078BC12D1CD12D01C7E
:09BC870012D1107F3F7E807D0088
:10BC90007C0012CE0A12D11078B412D1CD12D01C71
:10BCA00012D094783C12D1D97F407E807D007C00F8
:10BCB00012D110783C12D1CD12D01C12D27312D1F5
:10BCC000107F3F7EA87D007C0012D11078B812D181
:10BCD000CD12D01C12D01C12D1107F407E007D00EE
:10BCE0007C0012D110783C12D1CD12D01C12D2732C
:10BCF00012D1107F3F7EC07D007C0012D01C12CE7E
:10BD00000E12D11078B812D1CD12D01C12D11078E9
:10BD10003C12D1CD12CE0E785412D1D912D25D7808
:10BD20005812D1D912D11012D01C12D11078C012D1
:10BD3000D1CD12D01C784412D1D9785412D1CD1261
:10BD4000D273783C12D1D912D11012D01C12D1105A
:10BD500078BC12D1CD12D01C783C12D1D97F3E7E56
:10BD6000C07D007C0012D110783C12D1CD12D01CC5
:10BD700012D1107F3F7E007D007C0012CE0E12D1CA
:10BD800010783C12D1CD12D01C12D1107F3F7E8092
:10BD90007D007C0012CE0E12D11078B412D1CD12DB
:10BDA000D01C787012D1D978C4E6FE088607339586
:10BDB000E0FDFC12D1107FE87E037D007C0012D3F1
:10BDC000F412D11078C6E6FE0886073395E0FDFC34
:10BDD00012D3CD12D1107FE07E5E7DF87CFF12D3AE
:10BDE000CDEC12D14712D1107F3F7E7F7DE57CC91B
:05BDF00012D110787073
:10BDF50012D1CD12D01C12D094785012D1D97F3FD8
:10BE05007EF07D007C0012D110783C12D1CD12D08D
:10BE15001C12D1107F3F7EC07D007C0012CE0E1219
:10BE2500D110783C12D1CD12D01C12D1107F3F7E9B
:10BE3500807D007C0012CE0E783C12D1D978BC12E0
:10BE4500D1CD12D1107F3F7E807D007C0012CE0ABD
:10BE550012D110783C12D1CD12D11078B412D1CDB7
:10BE650012D01C12D01C784012D1D9785412D1CDE1
:10BE750012D2AB783C12D1D912D11012D01C7874E1
:10BE850012D1D97F417E107D007C0012D11078C07F
:10BE950012D1CD12D01C12D1107F407E807D007C46
:10BEA5000012D110784412D1CD12D01C12D1107FBE
:10BEB500417E207D007C0012CE0A12D110784412FA
:10BEC500D1CD12D01C12D1107F407E407D007C0068
:10BED50012D110787412D1CD12D01C12D1107F401E
:10BEE5007EA07D007C0012CE0E12CE0E12CE0A125E
:10BEF500D110785012D1CD12D01C12D11078501219
:10BF0500D1CD12D01C12D1107F3D7E2A7DAA7CABEB
:10BF150012D01C12D1107F3F7E007D007C0012CE16
:10BF25000A12D110783C12D1CD12D110787012D1ED
:10BF3500CD12D01C12D110784012D1CD12D094124E
:10BF4500D110785012D1CD12D01C12D110785012C8
:10BF5500D1CD12D01C12D01C12D110785412D1CDD3
:0CBF650012CE0A12D1107F4A7E517DD20C
:10BF71007CCB12D01C12D18278AC12D1D97F407EF9
:10BF8100007D007C0012D110787412D1CD12D01C2A
:10BF910012D1107F3F7E807D007C0012CE0E12D127
:10BFA10010784412D1CD12CE0E12D110785012D188
:10BFB100CD12D01C12D110785012D1CD12D01C123A
:10BFC100D110785012D1CD12D01C12D1107F3E7EEB
:10BFD1002A7DAA7CAB12D01C12D110785012D1CD7F
:10BFE10012CE0A12D110785812D1CD12D09412D19A
:10BFF100107F4A7E517DD27CCB12D01C12D182128D
:10C00100D110AF3AEF3395E0FEFDFC12D1107F4025
:10C011007E7E7D057C0012D3F412D1107F607E7587
:10C021007D587CFF12D3CD12D3CD78B012D1D978FF
:10C03100AC751B6412C0588F1C78B0751B6712C099
:10C0410058E51C75F00AA42FFF249C50027F00784C
:10C05100D7E654802FF62275390012D1CD12D110B6
:10C061007F0A7E007D007C0012D4A0A81BE513F698
:10C0710008E512F608E511F6335004EFF404FF2247
:10C08100C23D78647BAC12BA72D23D78677BB01244
:10C09100BA7212C48D7F007EE47D577C0012D110EC
:10C0A10078AC12D1CD12D3CD12D1107F007E537D49
:0EC0B100077C0012D4A012D12F85133B7F8094
:10C0BF007ECB7DA47C0012D11078B012D1CD12D3DB
:10C0CF00CD12D1107F407E7E7D057C0012D4A01250
:10C0DF00D12FE513F56F04F53A85126E85116D8535
:10C0EF00106C7F407E7E7D057C0012D110786C1223
:10C0FF00D1CD12D3F412D1107F607E0C7DA27C00C3
:10C10F0012D11078B012D1CD12D3CD12D3E0786CFA
:10C11F0012D1D978AC12D1CDEC12D14712D1107FF8
:10C12F00347E9C7D2B7C5F12D01C785412D1D91297
:10C13F00D25D785012D1D9786C12D1CDEC12D14793
:10C14F0012D1107F347E9C7D2B7C5F12D01C12D1BC
:10C15F0010785012D1CD12D01C784012D1D97F4017
:10C16F007E007D007C0012D110785412D1CD12D0F8
:10C17F001C12D27312D1107F3D7EC07D007C001245
:10C18F00D11078BC12D1CD12D01C12D1107F3E7EAF
:10C19F00C07D007C0012CE0E12D11078BC12D1CD12
:10C1AF0012D01C12D01C12D1107F3D7E407D007C1E
:10C1BF000012D11078BC12D1CD12D01C12D1107F29
:10C1CF003E7E807D007C0012CE0E12D11078BC1204
:10C1DF00D1CD12D01C12D1107F3F7E807D007C000C
:10C1EF0012CE0A12D110785412D1CD12D01C12CE09
:10C1FF000A12D1107F407E807D007C0012D1107812
:10C20F005412D1CD12D01C12D27312D1107F3D7E99
:10C21F00707D007C0012D11078BC12D1CD12D01CD1
:10C22F0012D11078BC12D1CD12D01C12D01C12CE4C
:10C23F000E12D11078B412D1CD12D01C785812D161
:10C24F00D9785412D1CD12D273783C12D1D97854F7
:10C25F0012D1CD12D2AB785412D1D9783C12D1CDA4
:10C26F0012D11012D01C12D11078BC12D1CD12D015
:10C27F001C783C12D1D97F3E7EC07D007C0012D14C
:10C28F0010783C12D1CD12D01C12D1107F3F7E00FE
:10C29F007D007C0012CE0E12D110783C12D1CD123F
:10C2AF00D01C12D1107F3F7E807D007C0012CE0EFD
:10C2BF0012D11078B412D1CD12D01C787012D1D9FE
:10C2CF00785012D1CD12D11012D01C12D11078C0CB
:10C2DF0012D1CD12D01C784412D1D9785412D1CDAD
:10C2EF0012D11012D01C787412D1D9784012D1CD3E
:10C2FF0012D11012D01C783C12D1D97F407E807D94
:10C30F00007C0012D110784412D1CD12D01C12D162
:10C31F00107F417E107D007C0012CE0E12D110785E
:10C32F004412D1CD12D01C12D110787412D1CD126B
:10C33F00D1107F407EA07D007C0012CE0A12CE0E5F
:10C34F0012D110783C12D1CD12D01C12D1107F3DDA
:10C35F007E2A7DAA7CAB12D01C12D1107F3F7E00AB
:10C36F007D007C0012CE0E12D110785412D1CD1256
:10C37F00D110787012D1CD12D01C12D110783C127E
:10C38F00D1CD12D01C12D01C12D110785812D1CD91
:10C39F0012CE0E12D1107F3F7E7F7DE57CC912D069
:01C3AF001C71
:10C3B00012D1107F4B7E187D967C8012CE0E12D14A
:10C3C0008212D1107FE87E037D007C0012D4A0127F
:10C3D000D12F78C8A61208A61308A60608A60778C3
:10C3E0007412D1CD12D1107F3F7E807D007C00126F
:10C3F000CE0A12D110784412D1CD12CE0E12D11025
:10C400007F3E7E2A7DAA7CAB12D01C12D1107840D0
:10C4100012D1CD12D01C12D110783C12D1CD12D035
:10C420001C12D110784012D1CD12CE0E12D1107F35
:10C430003F7E7F7DE57CC912D110787012D1CD127C
:10C44000D01C12D01C12D1107F487EF47D247C00B9
:10C4500012CE0E12D18212D1107FE87E037D007CB5
:10C460000012D4A012D12F78C4A61208A61308A6D1
:10C470000608A607223F3F4344454647484A4B4CDF
:10C480004D4E5051525354555657583F3FE4F5398D
:10C49000F5A790C4A1791078B4E493F6A308D9F96C
:10C4A0002232A5C24A4A19DC3A885CDB3BFFD6DC63
:01C4B0003B50
:10CD9E00D2D58002C2D575A70490040078107F0BFF
:10CDAE0012CDCA78267F0512CDCA783C7F2212CDCD
:10CDBE00CA786A7F0F12CDCA75A7002230D506E653
:10CDCE00F008DFFB22E0F608DFFB22D2D58002C29C
:10CDDE00D575A7049006FA78737F0612CDCA75A78B
:10CDEE000022DA0CD902800BD906303701B3500578
:10CDFE0002CF7D923702CF69D9F680F9D236800202
:10CE0E00C23612CFAE303606C86002B237C892367E
:10CE1E00DAD0D9E4B8000A12CFF5A236923702CF93
:10CE2E005260FBB51300400F12CFF5A23692F7A257
:10CE3E00379236A2F79237C398F40424E740DF24E2
:10CE4E0019AD29AC28AB277A00C394084008CDCC85
:10CE5E00CBCAE4CD80F424086010F9C3ED13FDECC9
:10CE6E0013FCEB13FBEA13FAD9F1A236303701B3F8
:10CE7E0040308A17E5102BF518E5113CF519E5122F
:10CE8E003DF51A501A13F51AE51913F519E518138D
:10CE9E00F518E51713F5170513E5137002051402BF
:03CEAE00CF08E4C6
:10CEB100C39AF517E5109BF518E5119CF519E512D4
:10CEC1009DF51A500DB237C378177F04E496F60822
:10CED100DFFA7A047019E513C39408F513500215AB
:10CEE10014E4C517C518C519F51ADAE802CFA92047
:10CEF100E7BAE5137002151415137817C37F04E61A
:10CF010033F608DFFA80E8E51A20E7137817C37FC4
:10CF110004E633F608DFFAE513700215141513E57C
:10CF2100173378187F03E63400F6500E08DFF775E3
:10CF31001A800513E51370020514E51420E75470F7
:10CF410027E513604E046020851A12851911851892
:10CF5100105326F0AC10AD11A237E51313FFE51203
:10CF610092E7FEA81302D12FE4F512F511F510F5A1
:10CF7100147513FF5326F043260580D8E5FFF512FB
:10CF8100F511F510751400F513D2375326F0432629
:10CF91000980C15326F0432603E4F512F511F5107B
:10CFA100F514F513C23780AC5326F080EC79017A81
:10CFB100018512F0E513A2F7339237751400F513CA
:10CFC1006002D2F785F012A813B8FF0809E512C272
:01CFD100E778
:10CFD2006001098C278D288EF0A2F7EF3304700AC6
:10CFE2000AC2F705F00AD5F0011A146002D2F785D9
:10CFF200F02922C88813C512C529C512C511C52832
:10D00200C511C510C527C51022DA03B8000302CF27
:10D012007DD9028002D9F702CF6912CFAE30370133
:10D02200B392377004D9E78005DADEB8000302CF85
:10D03200A9D9E2C3947E500215142513F5135002A8
:10D0420005147815760008B81BFA78277915E608D2
:10D05200FAE8FC78108AF0E608A427F709E5F03729
:10D06200F7500989F00907E760FBA9F0B813E61940
:10D0720019ECF8B82AD802CF0802CF94B8FFFA0206
:10D08200CF7DD9FB02CF69DAF6B800F002CFA91240
:10D09200D1E512CFAE303701B392377007D9E3B87A
:10D0A20000E280DBDAE1B8000280E1D9D5C8C3989A
:10D0B20050021514247F50020514F513781A7600D5
:10D0C2007A1A7B80C3E5109527E5119528E512951C
:10D0D200294016C3E5109527F510E5119528F5119D
:09D0E200E5129529F512E64BF662
:10D0EB00DA0302CF08EB03FB30E703187600C3E546
:10D0FB001033F510E51133F511E51233F51240CA73
:10D10B0030E7DD80B6E53905396010D0F0D0E0C0EE
:10D11B0010C011C012C013C0E0C0F08F138E128D5F
:10D12B00118C1022E539146010D0F0D0E0D013D060
:10D13B0012D011D010C0E0C0F01539227920800C2C
:10D14B007910800479087D007E007F003392D550E2
:10D15B000312D1BFEC33400FEF33FFEE33FEED3351
:10D16B00FDEC33FCD9EE22EECCF5F0747E29A2D582
:10D17B0013FF92F7AEF022EF8EF0A2F7D2F73392B5
:10D18B00D5C3947F5006E4FFFEFDFC22942040049F
:10D19B0074FF80F304CCFEE4FFFAE5F0CC6012C31D
:10D1AB00CC13CCCD13CDCE13CECF13CF0450EEDAA0
:10D1BB00EC30D5D7C3E49FFFE49EFEE49DFDE49CD9
:03D1CB00FC22E65D
:10D1CE00FC08E6FD08E6FE08E6FF22ECF608EDF6A2
:10D1DE0008EEF608EFF622CFC513CFCEC512CECD90
:10D1EE00C511CDCCC510CC22E4F513F512F511F511
:10D1FE001022E493FCA3E493FDA3E493FEA3E49333
:10D20E00FFA322C0E012D11012D01C12D24412D2AF
:10D21E0000D0E0C0E012D11012D23B12D01C12D1BD
:10D22E001012D20012CE0ED0E0D5E0E722AC48ADFF
:10D23E0049AE4AAF4B228C488D498E4A8F4B227491
:10D24E00FF7809FFFEFDFCE52654F048F526221274
:10D25E00D30404A2E1927F1420E01590D3857404C8
:10D26E0012D211802912D30430E102B27F20E0EBFA
:10D27E008C4C8D4D8E4E8F4F90D399740412D211CB
:10D28E0012D110AC4CAD4DAE4EAF4F12D01C307F04
:10D29E0004EF6480FFEE33EF337001FF2212D304EC
:10D2AE00C0E08C4C8D4D8E4E8F4F90D3BD740312BB
:10D2BE00D21112D110AC4CAD4DAE4EAF4F12D01CA0
:01D2CE00EC73
:10D2CF00C54CFCEDC54DFDEEC54EFEEFC54FFF90B5
:10D2DF00D3AD740312D211D08212D110AC4CAD4D1C
:10D2EF00AE4EAF4FE58230E00712D094B27F809DF3
:10D2FF0012D0918098EE33EF3324605007D0E0D0F6
:10D30F00E002D24DEFA2E7547F927FFF12D1107C43
:10D31F00837DF97E227F3E12D01CEE33EF332481C2
:10D32F00501012D11012D18212D147EFB2E7FF1273
:10D33F00CE0EEE33EF33602A2403F8C313FFEE92C1
:10D34F00E7FEE82481E4501A12D11012D182EF04C3
:10D35F00C2E0FCF58212D14FEFB2E7FF12CE0EE51D
:10D36F008203FAEE33EF33600B148FF0A2F713FF43
:10D37F00EE92E7FEEA2283FA703AE4E9AABCF8E0FB
:10D38F00813EE6E99DBF0000803F1A3C283966695F
:10D39F0099BBE335A33DE75D25BFDB0FC93FCCDB71
:10D3AF008D41EE3649C43F91C9453DF8B0C50000E7
:10D3BF00803F34F517C373FA2F45DDFD0AC6EF25FD
:10D3CF0013FFEE3512FEED3511FDEC3510FC02D1D9
:10D3DF002FC3EF9513FFEE9512FEED9511FDEC9512
:10D3EF0010FC02D12FEFF88513F0A4FFE513C5F061
:0AD3FF00CEF9A42EFEE435F0CDFABD
:10D4090088F0E512A42EFEED35F0FDE433CC85134A
:10D41900F0A42CFCE5128AF0A42CFCE51189F0A4F7
:10D429002CFCE51088F0A42CFC89F0E512A42DFD54
:10D43900EC35F0FCE51188F0A42DFDEC35F0FC8A03
:10D44900F0E513A42DFDEC35F0FC02D12FE4CCF866
:10D45900E4CDF9E4CEFAE4CFFB75F020C3E513334C
:10D46900F513E51233F512E51133F511E51033F52E
:10D4790010EF33FFEE33FEED33FDEC33FCEF9BEEA3
:10D489009AED99EC98400CFCEF9BFFEE9AFEED9912
:10D49900FD0513D5F0C622C2D5EC30E705B2D51289
:10D4A900D1BFE51030E70DB2D512D4C312D456124C
:10D4B900D1BF800312D45630D515C3E49513F513A3
:10D4C900E49512F512E49511F511E49510F5102281
:1093E900E57124885002D2191265938E4712E6C39B
:1093F90012AE8E12694F305E0F1268ED12A57A1205
:10940900681E12A1B7124FD41246F012557B1036BE
:109419002C30121F203725201A22E412957212953A
:10942900871296821296A430510302972E1299FF41
:10943900205109C251E4F552F545F5442275A700BA
:10944900758307E559C454F0F582E0F538A3E0F5D2
:1094590018A3A3A3E0F51E74FF1295721265938EEB
:109469001C8F1B7510DF751100E51164B4700612AD
:10947900953D75111012950A4028AE1CAF1B126656
:109489001B20321EAC03AB027A0C126222ED701261
:1094990075A700758304851182ECF00583E510F04A
:1094A9000511D510C412953D75C70375C6E075A79A
:1094B900049005007F041294F8DFFB75A700123AA7
:1094C900111268EDE4F5A7F8F559758307E8C4F5B5
:1094D90082E065387011A3E06518700BA3A3A3E0BF
:1094E900651E700388592208C3E5589850DC22E0AC
:1094F900F5BCE0F5BDE0F5BEE0F5BF1257AF05C616
:1095090022E51075F004A4F5C685F0C775B901E523
:0B951900BC33401F05C605C675B90134
:1095240085BE6485BF6505C675B90185BC6685BD04
:109534006785BE6885BF69C322E51124FE502E7578
:10954400A7007F10AE111E7583048E82E0FD158284
:10955400E0CDB505005012F00582CDF00583E0FDA5
:109564001582E0CDF00582CDF0DEDCDFD7227FB4BA
:1095740075A75490040005A7900500F0F0DFFC7572
:10958400A70022129D8AC2517B077AFFE47F00F56F
:10959400A790040012966EED244C4035EC603075B3
:1095A400A7008D8205A71296347583058D82E02469
:1095B40010401CF005A7E02CF0500505A7E004F0CE
:1095C400BA000CBB0009D251EF24DC50027F23DF28
:1095D400C3EA60051295E78006EB600312961F75D7
:1095E400A7002230E0047553082230E104755318B3
:1095F4002230E2047553282230E3047553382230B4
:10960400E4047553482230E5047553582230E604C7
:109614007553682230E7037553782230E00475539C
:10962400882230E1047553982230E2037553AA224C
:10963400ED54F0C4232390963E735302FE2253024A
:09964400FD225302FB225302F740
:10964D00225302EF225302DF225302BF2253027F25
:10965D00225303FE225303FD225303FB225303FB2C
:10966D0022129C8412CBE8E4F5F7E4ADF7F5F7E4AC
:10967D00ACF7D2B22290050078B4E06015FD54F03D
:10968D00C4CD7C00540FFE1583E0FF126320EFF074
:10969D0005830582D8E42275830478FF088882E06B
:1096AD0060FAF5D38812E512244C50012285D3D2ED
:1096BD0088D4881279FF0512E51260F00908E87563
:1096CD00F0B484A8F08882E060ECF5D3B900028094
:1096DD00D5B9230050D0C395D292D15002F40409CC
:1096ED00FEE4FFFCAD0112632D7401FA25D475F073
:1096FD00B484A8F0AC06AB07126214EB30E7010C92
:10970D00E5D22C30D1029C9C8882F00AEAB501DCAE
:10971D00E512244C50012285D3D28512D4A8128093
:10972D00939004001297ED8C068B051297EDE4FFD4
:10973D00F512F5118C148B13C3ED9BF9EE9CFA40C9
:0B974D0012E51199E5129A500A8C14E5
:109758008B138A1289118F528F82E0F9C3ED99FD1C
:10976800EE9400FEE582245A5002244C75F0B4842D
:1097780085F082E0FA2DFDEE3400FEEB9AFBEC94C6
:1097880000FCE92BFBEC3400FC0FBFB4B0E552241D
:10979800D3400224B4F552C3E51333FBE51433FC7C
:1097A800E511FE2BFBE512FF3CFC126382E9F89001
:1097B80097FF93F511FDEBF513FFECF514FE7C0014
:1097C8001263208F44E89098FF93FAAB13AC1412FD
:1097D800624BAF03AE04AD117C00126320EF700240
:1097E800F552F545227C007B007F5AE02BFBEC34D8
:1097F80000FC0582DFF522B4B4B4B4B4B4B4B4B494
:10980800B4B4B4B4B4B4B4B4B4B3B3B3B3B3B3B317
:10981800B3B3B3B3B3B3B2B2B2B2B2B2B2B2B2B11B
:10982800B1B1B1B1B1B1B0B0B0B0B0B0B0AFAFAF2D
:10983800AFAFAEAEAEAEAEAEADADADADADACACAC49
:10984800ACACABABABABAAAAAAAAA9A9A9A9A9A86F
:10985800A8A8A8A7A7A7A7A6A6A6A5A5A5A5A4A49E
:10986800A4A4A3A3A3A2A2A2A2A1A1A1A0A0A0A0D4
:109878009F9F9F9E9E9E9D9D9D9D9C9C9C9B9B9B10
:109888009A9A9A999999999898989797979696964F
:109898009595959494949393939292929191919192
:1098A8009090908F8F8F8E8E8E8D8D8D8C8C8C8BD3
:1098B8008B8B8A8A8A898989888888878787868618
:1098C800868585858484848383838282828181815D
:1098D8008080807F7F7F7E7E7E7E7D7D7D7C7C7CA0
:1098E8007B7B7B7A7A7A79797978787877777776E3
:1098F80076767575757474000203050608090B0CF5
:109908000E101113141617191A1C1D1F21222425B5
:1099180027282A2B2D2E303133343637393A3C3D1F
:109928003F404243454648494B4C4E4F5052535591
:109938005658595A5C5D5F606163646667686A6B14
:109948006C6E6F707273747677787A7B7C7E7F80AA
:10995800818384858688898A8B8D8E8F9091929455
:1099680095969798999B9C9D9E9FA0A1A2A4A5A619
:10997800A7A8A9AAABACADAEAFB0B1B2B3B4B5B6F7
:10998800B7B8B9BABBBCBDBEBFC0C0C1C2C3C4C5ED
:10999800C6C7C7C8C9CACBCCCCCDCECFD0D0D1D200
:1099A800D3D4D4D5D6D7D7D8D9DADADBDCDCDDDE28
:1099B800DEDFE0E0E1E2E2E3E4E4E5E5E6E7E7E86C
:1099C800E8E9EAEAEBEBECECEDEEEEEFEFF0F0F1C4
:1099D800F1F2F2F3F3F4F4F4F5F5F6F6F7F7F8F834
:1099E800F8F9F9FAFAFAFBFBFBFCFCFDFDFDFEFEBB
:1099F800FEFEFFFFFFFFFFC251E4F544F814FB90A1
:109A08000400A9007C0FC2D1129B1AE82405F8B8FB
:109A1800B4F08B13E5122403FA244C5001FABBFF6F
:109A2800012275112C8A19129B518F16203D12AAFA
:109A380019751123129B518F15751600303DE28060
:109A480011751123129AF9751500303D05E82F1389
:109A5800F515751112129AF9751400303D05E82FA5
:109A680013F514EA2404F552244C5002F552E4F597
:109A78001AF51BF51CE516600AFB7A00AF137EFF8A
:109A8800129ABFE515600AFB7A4FAF137EFF129A50
:109A9800BFE516600DFB7A00E5146006FF7ECF1265
:109AA8009ABFAE1CAF1B7C00AD1A1263208F45EF26
:109AB8002513F544D25122EFF5F0A4FCADF0EBF5F7
:109AC800F0A49CFCE5F09DFDEB8AF0A4FAABF0EF66
:109AD8008EF0A49AF8E5F09BF9E833F8E933F97BBE
:109AE800001263C6051AE51B2BF51BE4351CF51C93
:109AF80022EA2511F9244C5001F9C2D1129B1830E1
:109B08003D428F00C3EA9511F9500324B4F9D2D12C
:109B18007C09E4FDFEFF8982E060062FFFE43EFE3B
:109B28000D09B9B4027900DCEDED20D118F51E2439
:109B3800FE923D500F12632DEFB503005006851EAF
:109B48001FFB881222F51D80E6129AF9203D437406
:019B5800020A
:109B5900129BF0129AF9203D387404129BF8129A5C
:109B6900F9203D2D7406129BF0129AF9203D2274BA
:109B790008129BF8129AF9203D17740A129BF012E9
:109B89009AF9203D0C740C129BF8129AF9203D01A8
:109B990022C3E89F605088148F158A1640081ABAA4
:109BA900FF0A7AB380060ABAB4027A00129AF93027
:109BB9003D34C3E89FF9602EC3E5149515FB693060
:109BC900E7D4E930E703F404F9EB30E702F404C31E
:109BD900995002AA16E5142515C82F28FFE4FC336D
:109BE900FE7D04126320222AFA244C5001FA22C372
:109BF900CA9AFA500324B4FA22121A1385BF6C8543
:109C0900BE6B756A0002CBCB12A13C852E72E55F53
:109C1900030354C0F8E55E543F28F57C305506220D
:109C290012CB44800312CB347410256A54F0F56AC0
:109C3900E4356BF56BE4356CF56C24815003756C78
:109C49000022756A00E4D380E8E54B75F010A4257D
:109C59006A54F0F56AE5F080D8E56A24F054F0F525
:0F9C69006AE56B34FFF56BE56C34FFF56C248115
:109C78005003756C7E22E56A24FF80E4E56D24F0CC
:109C880054F0F56DE56E34FFF56EE56F34FFF56F52
:109C980024815003756F7E22129CFC129D59C22D9F
:109CA800C254C255E57F7002D255147002D254E5F1
:109CB8004A30E00122B4062120540C129C6212A002
:109CC8000E12A0BD02A15312A22B7E0412F213752C
:109CD8004A0112F20D756A202220550C129C31128D
:109CE800A08E12A13C029FE712A22B7E0412F2134F
:109CF800754A052212CBD37870E4F5F7E4A6F70885
:109D0800B880F6D2B222129D8A756D1012CBE8E4A3
:109D1800F5F7E4E5F7D2B264C0702D756D1E12CB6D
:109D2800E8E4F5F7E4E5F7C4F9E4F5F7E4E5F7D294
:109D3800B2C4F8E9540FFD5301F0E8540F49FCE8A8
:109D480054F0FB7F03129F79056EE56E540370B9DA
:109D580022E575F8541F30E40244E0F57585722E4B
:109D6800A2779226E57C543F30E50244C0F55EE5D3
:109D78007C54C02323F55FE57FC2E779BCF709A7C8
:109D88007E22856C6F856B6E856A6D22856F6C850A
:109D98006E6B856D6A22FA7420303B027460851000
:029DA800F0A425
:109DAA00256EF54DE5F0356FF54EEA2323303B0479
:109DBA0075F003A4254DF54DE5F0354EF54E754C7D
:109DCA000022758000C2B212F21BD2B22275800044
:109DDA00C2B2F5F7A4D2B222758000C2B2F5F7A4D6
:109DEA008DF7A48CF7A48BF722EB241054F0FBE434
:109DFA003CFCE43DFD22EB24F054F0FBEC34FFFC88
:109E0A00ED34FFFD22758000C2B2F5F7A4856FF725
:109E1A00A4856EF7A4856DF722E56D241054F0F53C
:109E2A006DE4356EF56EE4356FF56F22756D00E5FC
:109E3A006E240454FC80EDE56D24F054F0F56DE5D4
:109E4A006E34FFF56EE56F34FFF56F22756D00E530
:109E5A006E24FC54FC80EC758000C2B2F5F7A48530
:109E6A004EF7A4854DF7A4854CF722740F254CF5BF
:109E7A004CE4354DF54DE4354EF54E2274F1254C42
:109E8A00F54CE54D34FFF54DE54E34FFF54E2275A0
:109E9A004C00E54D24FC54FC80EC7403129E617561
:109EAA00A70090040075F700A4E5F7F0A3E5832462
:039EBA00F850F26B
:109EBD0075F700A4E5F7D2B2C23C30E602D23C758C
:109ECD004C00E54D240454FC80A77403129E61756B
:109EDD00A7009004007F22129F0C8010E54C2411E6
:109EED00FBAC4D0C0CAD4E7403129DE275A70090AA
:109EFD0004117F00129F0C7FEF129F0CD2B22275BE
:109F0D00F700A4E5F7F0A3DFF622D23CE4F56FF5F8
:109F1D006EF56D7403129E0FE4F5F7A4E5F7D2B25A
:109F2D0004600BC23C129E23E56F24FE50E5923D6A
:109F3D00227F1079B87406129DD77402129E0F8776
:109F4D00F709DFFBD2B280337F1079B87403129E0C
:109F5D000FE4F5F7A4A7F709DFF7D2B278B9793A8C
:109F6D0012DC7602A0DBAD6FAC6EAB6D7406129D8C
:109F7D00D77402129DE28FF7A4D2B2758000C2B2DF
:109F8D0075F705A475F705A4E5F7D2B220E0EC222C
:109F9D007403129DE2E4F5F7A4E5F7D2B222E4FED4
:109FAD00FF740775A704F5838E8274FFF0DFFD75CE
:109FBD00A7002274067E007FB0129FB0E4F55AF51B
:109FCD005B2275A704758306E55A600A75F00A844D
:0A9FDD00E5F07002740AC4F5822258
:109FE700307720E55A24024002055A129FCFE55ADE
:109FF700F0E573F0E574F0E575F0E576F0E577F0F8
:10A00700E578F075A700223077F9129FCF7F10749B
:10A01700FFF0DFFDE55A24F5500312A039155AE584
:10A027005AB4FF02055AC3E55A955B50D6755B00D3
:10A0370080D1129D8A7F0A056D056D12CBE8E4F584
:10A04700F7E4E5F7D2B230E704DF028005129C841B
:10A0570080E5056D12CBE8129FCFE55A24F6F07F15
:10A0670006E4F5F7E4E5F7F0DFF7D2B275A70022CB
:10A077007F4212A07FDFFB22302B0C0542E54224F2
:10A087007C400122754280053FE53FB43C17753F90
:10A0970000053EE53EB43C0D753E00053DE53DB48B
:10A0A7001803753D00802D302B0C1542E5422483A3
:10A0B700500122754280153FE53FB4FF17753F3BBE
:10A0C700153EE53EB4FF0D753E3B153DE53DB4FF3E
:10A0D70003753D1778ABA63A08A63B08A63C1219AC
:10A0E700FAE5BF253D240C75F0188478AEA6F01864
:10A0F7006005640260182216E670121816E67004EE
:0CA10700760C181678ACE690A12F930897
:10A11300F6220618E60890A12F930466700D7601C7
:10A123001806E6640D70047601180622001F1D1F31
:10A133001E1F1E1F1F1E1F1E1F0542E542B43C0F9C
:10A143007542000541E541B43C05754100054022D7
:10A153001542E542B4FF0F75423B1541E541B4FF9B
:10A163000575413B154022AC40AB41A842EC75F06C
:10A173003CA42BFBE435F0FC7A3C126214EB28FB85
:10A18300E43CFC22E53FC313F8AB3E79AEE7800E17
:10A193001219DCE5BE75F005A4FB7800E5BF75F088
:10A1A3003CA42BFBE435F0FC7A1E126214EB28FB73
:10A1B300E43CFC2212A193AE04AD0312A1878C14DC
:10A1C3008B131219E6E5BFFF24F650027F01E5BEAB
:10A1D30075F096A4AAF0F9C3ED9513FBEE9514FC64
:10A1E300924E4B701120110E30480B75364B3003D5
:10A1F300037536FFD22E304E02DF1F7A021262142D
:10A2030075A7009004EEECF0A3EBF0C3E5BF9F0449
:0FA21300BF0102D2E79005CBF022ED29FDEE3A14
:03A22200FE80B506
:10F2000012F20912F20912F2097E0480067E0280CF
:10F21000027E017F0080087F6480027F017E00EF14
:10F220004E6012E4FD0D1D0DEDC394AD40F7EF1FD0
:10F2300070ED1E80EA2212F39E90B7F07F001285D7
:10F24000B512F25112F209753500C200C201C202B4
:01F25000229B
:10F38A00F5D8D2DCE5F520E7FBE5DA540FFEAFD974
:04F39A0075D8002200
:10EFBC007F767E0690AEC31285C7740412F38A7CEA
:10EFCC00007D52126320EFF875F00A84C0F07F7652
:10EFDC007E2312E99F7E29742E12E9B27E2ED0E098
:10EFEC0012E99F7E35745612E9B27F6B7E1190F058
:10EFFC002512E9DEE824E04001220423F824E7503E
:10F00C0002781812F015D8FB227F6CE82411FE79D7
:10F01C000512F2E30E0FD9F922071DFFFFFFE08066
:10F02C00000020C0000038E0000008F0000038F8B4
:07F03C00000020FFFFFFE0D0
:10F0C00012F0E830E6022409540F75F00AA4F51591
:10F0D00012F0E830E6022409540F25152212F0E858
:10F0E000540F2275F000800875F044800375F00716
:10F0F000E4206D09D5E0FAD5F0F7D24C229247C250
:10F10000ACE54F623885504FA26E926D859950C222
:10F110006FD2ACC24CA2472212F122C4FA12F122E1
:10F120002A2212F0E820E603540F22540724092271
:10F04300E612F04A18E608FAC412F050EA540F44E4
:10F0530030F924C6E950112407800D75F00A84C0E5
:10F06300F012F069D0E0443030530975F00085E0C8
:10F07300E0D5F0FA3099FD75F019D5F0FDC299F598
:10F0830099623822E53880EC742A12F0776238E509
:10F093003812F04A800812F06BE53812F06B740DE9
:10F0A30012F06B740A80C1744012F06B744080B824
:0DF0B300742C80B4742E80B075380080ABD2
:10F3B00085A0835383FE438380858384F075840016
:01F3C000222A
:10EE690074A212F3B074A112F3B074A612F3B074C1
:10EE7900A412F3B074C012F3B0742512F3B012EEF9
:10EE8900FA75C70375C6FC75B90112C4B1740812C5
:10EE9900F38AEE75F020A4FEEF54F80303032E2441
:10EEA90092C313FE24EA50027E16EE90EEE39325F8
:10EEB900BCFE24E6502024E8401C748112F3B0EE15
:10EEC90012F3B012EF07744012F3B0742F12F3B0BB
:10EED90074AF12F3B0227E2680E0F7F7F8F8F9FA5A
:10EEE900FBFCFDFEFF00000000010102020203031A
:10EEF90003A8BCA9BDAABEABBFACC7ADC62288BC1E
:0BEF090089BD8ABE8BBF8CC78DC6225D
:10F25100C006C007C5F075A7019000007EB7E58C18
:10F26100240340FA12F2731EBEAFF3C5F0D007D0EB
:10F27100062275A700EE12F3B0741012F3B07404F5
:10F2810012F3B085A08343838185838475A7517F61
:10F2910020E0F0E0F0E0F0E0F0DFF6E4F5A7F5843F
:01F2A100224A
:10F39E0075A711900000E4C583F0C58330E2F8F53F
:02F3AE00A72294
:10F2E300EF20E723EE20E71F20E61C05A7C4540305
:10F2F300F583EE5408C42FF582EE5407240983F5F1
:10F30300F0E045F0F005A722804020100804020138
:10F31300EF20E723EE20E71F20E61C05A7C45403D4
:10F32300F583EE5408C42FF582EE5407240983F5C0
:10F33300F0E055F0F005A7227FBFDFEFF7FBFDFEFE
:10E95D00FDA42582F582E5F03583F583ED227E0059
:10E96D00906F637A0475F00512E95D7D05805E7A1E
:10E97D000580027A04547FC0E0C083C082C3942016
:10E98D005001E4906F1312E972802E9070717A0528
:10E99D00800590712E7A0675F00712E95D7D07806E
:10E9AD002C7A0580027A06C0E0C083C082C3942011
:10E9BD005001E49070BE12E9A4D082D083D0E02241
:10E9CD00906E8775F00A12E95D7D0A7A07C2D180D3
:10E9DD0002D2D1C0A7C082C083C007C006C0E0303C
:10E9ED00D10975A704E493FDE493FAEEFB75A70432
:10E9FD00EBFEEAFC7901D9067908E493F5D4E5D468
:10EA0D0023F5D420E01612F3130EDCEA0FDDE1D06E
:10EA1D00E0D006D007D083D082D0A72212F2E380B7
:10EA2D00E8906DC775F00E12E95D7D0E7A0812E95A
:10EA3D00DA906E6F75F00212E95DE493FDE4A39335
:10EA4D00FACE2408CE7C0812EA5B7C06AD02ED23DB
:10EA5D00FD20E00712F3130FDCF42212F2E380F72E
:10E84800F5D2C2D58036F5D2D2D58030F5D224F6AD
:10E8580050090E0E24A650030E0E0EE5D2F5D27501
:10E86800F0648485F0D3C2D57009D2D5742012E93A
:10E87800B2800312E99FCE2406CEE5D375F00A8450
:10E8880085F0D3700A30D507742012E9B2800312DC
:10E89800E99FCE2406CEE5D312E99FE5D222F5D230
:10E8A80075F0648485F0D3C2D58022F5D2C2D580B4
:10E8B80025F5D2D2D5801FF5D275F0648485F0D3C2
:10E8C800C2D57009D2D5742012E9B2800312E99832
:10E8D800CE2405CEE5D375F00A8485F0D3700A30CE
:10E8E800D507742012E9B2800312E998CE2405CE28
:10E8F800E5D312E998E5D222F5D2C2D58035F5D212
:10E90800D2D5802F30E70DF404C0E0742D12E980D1
:10E918000E0ED0E0F5D275F0648485F0D3C2D570C0
:10E9280009D2D5742012E980800312E96DCE24043F
:10E93800CEE5D375F00A8485F0D3700A30D5077414
:10E948002012E980800312E96DCE2404CEE5D312AB
:05E95800E96DE5D2228B
:1085AC0090B1A91285B502F2517E00800E7405FEC1
:1085BC00F51EE4FFF51DF51F203C3375A700E49371
:1085CC00700122A3B40204051D8003B4010A051F27
:1085DC00EF2409FFAE1E80E612E9B27D06B440021C
:1085EC007D03B421027D02EE2DFE80D27E0075A7A4
:1085FC0000E493700122A3B40204051D8003B401AE
:10860C000F051FEF2407FFAE1E80E612E97C8008E1
:10861C00B45B0050F612E9800EB4210280D30EB484
:10862C00400280CDB42C0280C80E0EB45F0280C113
:10863C00B45B0040BC0E80B9E60812E9B2EE240629
:10864C00FED513F42290AEF130740990AEF5307370
:10865C000390AEFA0285C775F019D5E0FDD5F0FA96
:10866C001255CF12F0AA744F12F0BB744B12F09942
:10867C00C322C2501286C21255CFD2AC12F0E330D4
:10868C004C1212F0E3304C0C12F0E3304C06D2508A
:10869C00C2ACD322B440E512F0E8B4400312F0E8C7
:1086AC00B44FED12F0E8B44BE712F0E812F0E81218
:1086BC00F0E8C2ACC32230530975F008D5E0FDD503
:1086CC00F0FA227F0575F019D5E0FDD5F0FA1255B8
:1086DC00CF12F0AA745712F0BB745012F06B748165
:0A86EC0012F06BE56312F06BE5621B
:1086F60012F06B78D0E612F06B08B8D7F8E6F87986
:108706005F30E702792FE912F06B12F06B12F06B13
:1087160012F06B745812F06B744312F06BE412F0A3
:108726006BE8C2E775F00A84C425F012F06B786432
:10873600E612F06B08B869F8E612F09912867E40E8
:108746000122DF02800A20508B75F0008080D25013
:10875600C2ACD3221286C2C2501255CFD2AC20026E
:10876600EF12F0E3204CE7B440F412F0E8B4400313
:1087760012F0E8B457DAF53812F0E8B450D212F035
:10878600E812F0E8F56312F0E8F56278D012F0E846
:10879600F924A0500353015FE924E04002795FA663
:1087A6000108B8D8E8780612F0E8D8FB12F0E8FC21
:1087B60053040FC4540F75F00AA42CFC249C5002D9
:1087C6007C0078D78601E4B92F02D2E72CF67864CC
:1087D60012F0E8F608B86AF812F0E8E53860030225
:1087E600875612F0E812F0E8C2ACC32290B6B98000
:1087F6000390B1EE7F201285F812F25102F2117544
:108806003400C26B1288C112F211128C7CE516601C
:108816000312881D020241128ECF122A3812F2511B
:1088260010002010010280F8128CE75013122A4320
:108836001287F210000D10010280F81229DE80D78F
:04884600128A6C2204
:10884A00C26BD22775480A123A05753400128DA5F3
:10885A00C26A124155106A0512023280ED120232C2
:10886A00128C0E128D66128DB178D0E664266044A1
:10887A00128ECF122A3812F25110003810010280DB
:10888A00F8128CE7501BE965156018122A43128703
:10889A00F212F20910001D10010280F81229DE807E
:1088AA00BCD26B128D92751607855917123A7E75CE
:1088BA0035008096020241128C7C1288E3128DB137
:1088CA007F191288FD90B6E57E121285FA7E23E59D
:1088DA001602E91C90B82E80EF7862E41288F478C8
:1088EA00D0745F1288F418E4F6227F08F608DFFCD9
:1088FA00227F7B7E007810742012E980CE2404FE49
:10890A00D8F5221222587F197E081285FA7E28305D
:10891A00530590B1D5800990B1D030340390B1DAC3
:10892A000285FAC26B1288E3128938020241C251E7
:10893A00128DB190B6DD12890D122A04128C7C7F39
:10894A00201288CC12F251E516700512F206803612
:10895A0075A6FF30510312866C1255CFD2AC200097
:10896A0025306DFA12875D400C128CE74011128A8D
:10897A006CD25180BB1050031287F7C25180D1D2FA
:10898A00511287F280CAC2AC22D22775480A123A1B
:10899A0005753400C26B128DA5C26A124155106A60
:0F89AA000512023280EB120232128C0E128D6611
:1089B900128DB11289C450DA02024190B1E91289CB
:1089C9000D122A1D12F251C31000131001051002D5
:1089D9000E80F41286CF4001221287F780DDD3C2C0
:1089E900AC22D227C26B75480A123A0575340012B7
:1089F9008DA5C26A124155106A0512023280EDD264
:108A09006B128C0E128D66128C3675B901E5BCB2EB
:108A1900E7F5BC1257AF751607855917123A7E80CC
:108A2900CB128C7CE516601F78D0E53D128A5DE596
:108A39003E128A5DE53F128A5D765A08765F12DC3E
:108A49006C128D92028C4D7F3E7E1190B1C01285C1
:108A5900C702F25175F00A844430F608E5F0443053
:108A6900F60822D26B128D92128C4DE51775F01013
:108A790084240AF54824E8500375480A123A1185F6
:108A8900585922753200129FAB75A70490070075DB
:108A99001500128C3675B901E5BC20E705E515F01E
:108AA900801004600D6482600975BCFF75B9057595
:108AB900B9020515E515242050D8E58224FE4003A6
:108AC900028B65A882187F0075A7007583078882C5
:108AD900E0FE75F004A4128BE1A9BCAABDABBEAC43
:108AE900BF1582E0FD75F004A4128BE1C3E995BCC2
:108AF900404C7052EA95BD4045704BEB95BE403EE7
:108B09007044EC95BF4037703DEE75F004A4041233
:108B19008BE1A9BCAABDABBEACBFED75F004A40442
:108B2900128BE1C3E995BC4015701BEA95BD400E57
:108B39007014EB95BE4007700DEC95BF5008EEF030
:108B49000582EDF01582E5826009C3EF9582500335
:108B5900028AD90FC3E89F4003028AD175A70490FE
:108B6900070075C70375C6A8E0F5BCE0F5BDE0F5DB
:108B7900BEE0F5BF75B90575B90205C6E5822420C1
:108B89004006E5C6242050E00875C70375C6807500
:108B9900B901E5BC128BCBF5BCE5BD128BCBF5BD9C
:108BA900E5BE128BCBF5BEE5BF128BCBF5BF75B910
:108BB9000205C6E5C6245850D6E5320470FB75A7F0
:108BC9000022B4FF0122F975A704900700E5826825
:108BD9006005E06970F7E922F5C685F0C775B90146
:108BE900E5BC645F700375BC27E5BD645F70037500
:108BF900BD27E5BE645F700375BE27E5BF645F707E
:108C09000375BF272275C703E54875F004A42480BE
:108C1900F5C6E55975F00484A8F00825C6F5C675AA
:068C2900B901A9BCAABDBF
:108C2F00ABBEACBF861522E515242050037515DFAA
:108C3F00E51575F004A454FCF5C685F0C722E517B9
:108C4F0024204028E51775F00484A8F00824A8F51F
:108C5F00C675C70375B901A9BCAABDABBEACBFA68B
:108C6F001589BC8ABD8BBE8CBF1257AF22E4F51697
:108C7F00F51579FF128C3675B901E5BCB4FF040503
:108C8F0016A9150515E515242050E9891579FF75E5
:108C9F00C70375C6A875B90109E5BC04601B09E5D2
:108CAF00BD04601509E5BE04600F09E5BF04600946
:108CBF0005C6E5C6242050DD0989172275160075F3
:108CCF001501128C3675B901E5BC20E702051605B2
:108CDF0015E515242050EB227900E975F004A45412
:108CEF00FCF5C685F0C775B901E5BC20E73078D033
:108CFF0066702B08E5BD66702508E5BE66701F0817
:108D0F00E5BF66701905C675B90108E5BC66700E3A
:108D1F0008E5BD66700808E5BE667002D32209E952
:108D2F00242050B6C322128D55128D3DA8017F0805
:0C8D3F00E0F608DFFB22128D55128D4D6E
:108D4B00A8017F08E6F008DFFB2278D0796275A7CF
:108D5B0004758307EBC454F0F58222128C3678D05D
:108D6B00128D80E5BCF9C23C20E702D23C128D800B
:108D7B007862128D8075B901A6BC08A6BD08A6BE87
:108D8B0008A6BF0805C622128C3678D012859A1217
:108D9B00859A786212859A02859A1268ED12F39E73
:108DAB0012A36D02F25112F39E7F007E0990B6CA98
:108DBB001285C77F0A7E12E5150412E8547F141240
:108DCB00DE5D1229DE7F277E0875130778D01286A9
:108DDB0044E6793E30E702792F7E34E912E9B27F1F
:108DEB003D7E0190B84A1285FA20311B30300312B8
:108DFB00B9F0C23B129061128E17D23B12906112E6
:108E0B008E291290A8807C12D4D980E6C23B7F4475
:108E1B007453201702744E7E0012E9B28017D23BB6
:108E2B007F4F745720170274457E0012E9B27E06FD
:108E3B00E51E12E99F7E0CE51D12E99F7E12E51CD3
:108E4B0012E99F7E17748112E9B27E1CE51B12E9B1
:108E5B009F7E22E51A12E99F7E28742E302602741B
:108E6B002712E9B27E2DE51912E99F7E33E5181220
:108E7B00E99F7E39302607742C12E9AE7E3BE5372D
:108E8B0002E99F742D201702742B7F707E1512E957
:068E9B00B2128EAC7E3A1B
:108EA10012E7FD7E0190B8750285C77E1BE51C1295
:108EB100E99F7E21E51B12E99F7E27E51A12E99FB2
:108EC1007E2DE51912E99F7E33E51802E99F128F85
:108ED1004D128F7812924F128DB11292A720171E48
:108EE10010021B125F3512DC6C128F351229E97FDB
:108EF100347E2F128651128DEA12F25180E212292C
:108F0100DE203026203128C23B129061128F8D78ED
:108F110066129161D23B129061128FA2786912910F
:108F2100611290A812901C02920412BAB980F21236
:108F3100D4EE80EDE57D75F01084AAF075F00AA4F9
:108F41002A547FFA78D7E654802AF6227F277E08B2
:108F510079D08700C001D224B9D002C22412932E45
:108F6100D001A70010230909EE2406FEB9D7E32298
:108F710019EE24FAFE80DB7E3479D7E7A2E7921757
:108F81001292DB79D7E7A21792E7F722C224C23BFC
:108F9100751E007F447E001292EB801E1023ED802F
:108FA1002AD23BC2247F4F7E001292F3D2247E0646
:108FB100E51E129320F51E1023E7D2247E0CE51D39
:108FC100129320F51D303BD41023E1D2247E12E50B
:108FD1001C129320F51C1023E17E1CE51B1293202B
:108FE100F51B1023E67E22E51A129320F51A1023B1
:038FF100E87E2DEA
:108FF400E519129320F5191023E87E33E51812932E
:1090040020F5181023E87E393026027E3BE537121E
:109014009320F5371023E3227F707E151292E3C26A
:10902400247E1BE51C129320F51CD2247E21E51B13
:10903400129320F51B1023E77E27E51A129320F5DF
:109044001A1023E67E2DE519129320F5191023E852
:109054007E33E518129320F5181023E82278D7E61A
:10906400C2E775F00A847866F537303B0578698580
:10907400F0371290D130262BE53775F003A40404A1
:1090840075F00584FBE51975F00AA4251875F0063A
:10909400A42BFBE435F0FC12643CF53712643CF578
:1090A400188B1922E563FC339217AB6250031264E8
:1090B400AD305C0A7AD212622278401263C4AE04E4
:1090C400AF037C277D1012632D8F1C8037E6FD33A0
:1090D400921718860418860350031264B57A097926
:1090E4002778C01263C18B1EADD3ACD2AB0679EA2C
:1090F40078601263BF8B1DAF06AED27C177D7012F1
:10910400632D8F1CAF05AE047C037DE812632D8FA5
:109114001BAF05AE047C007D6412632D8F1AED75C0
:0A912400F00A84F51985F01822EC1A
:10912E0033921750031264AD751D30301786751DBE
:10913E002D808178427B607CEA800678407B207CA3
:10914E004E12D5B9792778101263BF8B1CAF06AEBD
:10915E00D280AB30262AE51975F00AA4251875F0D1
:10916E000AA42537FBE435F0FC7A051262148C064E
:10917E008B077C007D031263208E048F0312909B5D
:10918E00E51E75F00AA4251D75F00AA4251C75F0C0
:10919E0006A4251BFBE435F0FC7A0A126214EB25BB
:1091AE001AFBE43CFC7A0A126222EB2519FBE43C22
:1091BE00FCE43DFD7A0A126234EB2518FBE43CFC1C
:1091CE00E43DFD3017031264B5A60518A60418A6D3
:1091DE000378D7E6A2E7923DC2E775F00A84FCABAE
:1091EE00F0303B0EAB37EC75F00AA42BA23D92E7A4
:1091FE00F622AC3780F012921F305C0A7A4012626F
:10920E002278D21263C43017031264AD8C638B6262
:10921E002212922F7A0A126214EB2518FBE43CFC00
:10922E0022E51C75F00AA4251B75F00AA4251AFB6D
:06923E00E435F0FC7A0AA1
:10924400126214EB2519FBE43CFC2212928112F207
:109254000DC202C2231292811000081001051002EF
:109264001B80F51031ED10300D102604D22680E35A
:10927400D230C23180DDD231C23080D7227F3590E6
:10928400B8331285F890B85120300F90B86D203162
:109294000990B84220260390B83A1F7E171285C75A
:1092A40002F2517F357E0190B19C1285FA7F347EA3
:1092B4003A1293D0744E12E9B212F25112F20DC264
:1092C400027F347E3AD21775115975124E80267575
:1092D400112E751227801E75113E75122F8016757A
:1092E400112B75122D800E75114E75125380067553
:1092F40011457512571293D0E511301702E5121279
:10930400E9B212F25110000810010510020B80F5A9
:10931400D23C1017E3D21780DF0293CB4430F8120B
:10932400932AE8540F22C2218002D221A22492223D
:1093340092231293D0E830E709D23C7430302102F2
:10934400745FF812E9B212F25110003410010510E2
:10935400025D80F5D23C102266102367B43909748B
:109364005F2021DF743080DBB45F04742D80D4B4BB
:109374002D04744180CDB45A04743080C60480C373
:10938400D23C302406102237102338B44104742D03
:1093940080B1B42D04745F80AAB45F04743980A3CF
:0593A400B43009745A09
:1093A90020219B74398097148094B48908D223E8CA
:1093B90012E9B2800DF8C223800874898001E8029D
:1093C90093479093E580039093E1C007EF2408FF4A
:1093D90012E9DED00702F2510205F8F80205000091
:10F1A00075A70090F1D275F02D84C2D5C2D1601739
:10F1B000D2D1146007D2D514600DC2D1E5F093FC12
:10F1C000742D95F093FB22E5F093FB742D95F0934D
:10F1D000FC220009121B242C353E474F58606870F2
:10F1E0007880888F969DA4ABB2B8BEC4CACFD4D95C
:10F1F000DEE2E6EAEDF0F3F6F8FAFCFDFEFFFFFFD3
:10F2A200D23D8002C23DED8BF0A430E70205F0C3EF
:10F2B200E895F020D50425F025F0FEED8CF0A43081
:10F2C200E70205F0C3E995F030D10425F025F0FFFF
:10F2D200203D0B2487500122EF24CC40012202F270
:01F2E200E348
:10EC2E00203A7A7E1C7F5312F2E37F5912F2E31ED2
:10EC3E007F5712F2E37F5512F2E37E2312F2E37F47
:10EC4E005712F2E31E7F5912F2E37F5312F2E31FC3
:10EC5E007E2012F2E37F5A12F2E37E1E12F2E37F5F
:10EC6E005212F2E31219E6E5BD20E0143006117FD0
:10EC7E00357E1C90ECECE571700390ECF602E9DE4B
:10EC8E00E5716018E57012F1A0781F79567D0912B2
:10EC9E00F2A6303A0312ECBF0DBD16F3227E1C7F96
:10ECAE005390ECD512E9DE200CD67E1F12DEC48006
:10ECBE00BEC0060E30D5021E1E12F2E3D0061F3065
:10ECCE00D1020F0F02F2E3070700386C446C3800D4
:10ECDE0005052070D8702005057088A88870080773
:10ECEE0010387CFE383838000807102844C628280B
:02ECFE003800DC
:10DC980090B87F7F717E231285FA1219E6E5BC7E63
:10DCA8003112E96D30121AC23C1219E6E5BCFB7557
:10DCB800F00AA4F904FAC23D129D8A12DF3B303DF6
:10DCC8000122DAF712DE3D7C00EBF4042E4019AD98
:10DCD80003126320EFA2D1203C077E237F6502E573
:10DCE800CAAE16AF1702DDDEAD01126320EF12E6F1
:10DCF800B8203C077E237F6502E5EEAE16AF17021B
:10DD0800DE027F567E0512DE697F3D12DE7C7F6F64
:10DD180012DE7C12DEC47E0A7F4112DEF77E227F8D
:10DD28005912DEF720120122129D8A857A1D855E1E
:10DD38001C857B1B855F1A7AC0C23D12DF37203DE8
:10DD48005212DE3D7C007D1412632074562F20D1C0
:10DD5800029F9FFF24CB40028037EF248850028027
:10DD680030EA1475F00384FE12F2E3C3E51B957BD9
:10DD7800FEE51A955F92D55004EEF404FEEEC31347
:10DD8800FE24E0400C741F2E30D5029E9EFE12F237
:10DD9800E3DAA8227F5212DDAE7F5A12DDAE751784
:10DDA80053751600802B7E0012F3130EBE12F92253
:10DDB8007F157E28742012E9B27F1C7E2812F31387
:04DDC8000EBE40F952
:10DDCC00223012E712DDB875171575162DD23C02EC
:10DDDC00DCB1C23D6002D23D92D175F080305C0462
:10DDEC00F5F08001A4A2E792D5E5F075F03284F845
:10DDFC00E5F075F00584C0E0E5F0A2D533C0E0E8AD
:10DE0C00601E12E99FEE2406FED0E0F8D0E012E985
:10DE1C009FEE2406FE742C12E9B20E0EE802E99F66
:10DE2C007420303D07742B20D102742D12E9B2807E
:10DE3C00D4C3ED957AFFEC955EFE92D1500312643B
:10DE4C009D227F1512DE557F327E3E12F2E3DEFB01
:10DE5C00227E0912F2E30EBE36F9227E0112F2E3A3
:10DE6C000E0EBE3FF8227E3312F2E30EBE40F922B4
:10DE7C007E047D1112F2E30E0E0EDDF81F1F7E35AF
:10DE8C0090B888305C057E3190B88C0285FA7405A8
:10DE9C00305C097E32740112E96D74067E3612E92B
:10DEAC006D7E3A740012E96D7E3D02E96D7F1512AC
:10DEBC00F2E30F0FBF2DF8227F417E1F7D0F12F270
:10DECC00E30F0F0FDDF8227F687D0380047F677DF1
:10DEDC000512F2E30FDDFA227F667D0780F37E1FC9
:07DEEC007F5012F2E31F1F3B
:10DEF300BF3EF8227D0A12F2E30E0E0F0FDDF7226A
:10DF0300203D07124A2C7003D23D22056D12CBE847
:10DF1300E4F5F7E4ABF7F5F7E4E5F7FA30E411EBF2
:10DF2300251DF51DE4351CF51C0519EA30E3010E2A
:10DF3300D2B28015780380027801203D07124A2C63
:10DF43007003D23D22D8F3056DE56D2409F56D12FA
:10DF5300CBE8E4F5F7E4ADF7F5F7E485F71BF5F760
:10DF6300E4E5F7FCD2B2543F30E50244C0CC54C0E0
:0BDF73002323F51AE56D24F6F56D225E
:10EB55007E017F0990EBD312E9DE2051097E037F08
:10EB650000743F02E9B2E4FEFFC3E54512E40FFD80
:10EB7500940AED403D9464ED4002746312E84E7EC4
:10EB8500017F09E552240575F02D84AAF075F0057D
:10EB9500A4CA75F00B842A90EBBE9312F1A0BCB801
:10EBA500027BB87D04EE2DF8EF2DF90D12F2A2DDF2
:10EBB500FB227E0312E99F80C6000C1622222D3906
:10EBC500444F4F5A66707C7C87939EA9A90009091A
:10EBD500080041000000000088800000000041009E
:10EBE50008001219FAE5BCB4F8339004C3E0602CB0
:10EBF500FA24F340277F137E0012F2E30F0F12F27F
:10EC0500E30E12F3131F1F12F3130EDAEC7F147EBB
:10EC15000012F2E30E12F3130EBE12F5229005CC8C
:09EC2500E0C3941240F60480C71C
:10E40F00305D0A75F08AA42480E5F0340022207470
:10E41F00157F017E1190E49712E9DE7F0A7E0AE5EF
:10E42F002E540702E8657F087E1190E4A712E9DEFB
:10E43F0020730C7F0A7E1712F3130E0E12F3137F45
:10E44F00007E0BE57112E40F12E8547F0C7E11E58C
:10E45F0071602F0EE57064B4602864B475F0328477
:10E46F00C0F012E998CE2405CED0E075F00584C037
:10E47F00F012E998CE2405CED0E023302D0104020E
:10E48F00E99890A56C0285C7070FFFFFC473BDAF56
:10E49F00A463B5FBCDE7FFFF030F0100FFFE038071
:10E4AF00306701227F3F7E00748812E9B2E5516028
:10E4BF00F21219FF85BCF01207DB12E40F75F0643E
:10E4CF0084F87E06E5F012E8B3E860D77E0002E933
:10E4DF009F1219FFE5BE70012214600814603BE51E
:10E4EF003F1340367F367E00747712E9B2207301F6
:10E4FF002279BC87040987031261BC7E05781DE66B
:10E50F0060097E0012E998EE2405FE18E6600712F6
:10E51F00E998EE2405FE18E6801990B0767F377ED5
:10E52F00001285FAAB60AC611261BF1F7E09781DC6
:10E53F00E6600712E998EE2405FE18E612E998EE58
:03E54F002405FEA2
:10E5520018E602E998202C012290E56102E9DE0525
:10E562000EFFF0E01CF004F81CFFF0301201227FD5
:10E57200637E0090AF0C12E9DE7F1512DE557F1F1D
:10E5820012DE557F2912DE557F177E06E53F30E009
:10E592000B90B89C305C0390B8B0800990B8913071
:10E5A2005D0390B8A61285C77F217E0190AF382007
:08E5B200740390AF2C0285C731
:10E720001261BC7F207E05751900781DC2D5E630C8
:10E73000D51712E998EE2405FE18B818F17E1F745B
:10E7400063305C02748202E9B27005B8191880E285
:10E75000D2D5CE24FACE7484301702742D12E9B2C9
:10E76000EE2406FE80C8742012E9AE80C8781C80B2
:10E770000D7F007E23AC5EAB7A1261BC781DC2D5E2
:10E78000E630D50C12E99FEE2406FE18B818F122E7
:10E790007005B8191680EDD2D53017E4CE24FACE24
:10E7A000742D12E9B2EE2406FE80D5742012E9B26F
:10E7B00080D51261BC781DC2D5E630D51612E96D40
:10E7C000EE2404FE18B818F10E745E305C02742753
:10E7D00002E97C7005B8191680E3D2D53017DACE7D
:10E7E00024FCCE742D12E980EE2404FE80CB74202C
:10E7F00012E98080CBC23D12E8080F0F0E0E746341
:10E80000305C02748202E9B21261BC781DC2D5E6A6
:10E8100030D50C12E9CDEE2408FE18B818F122709C
:10E8200005B8191680EDD2D5301716740BCE24F822
:10E83000CE12E9CDEE2408FE80D5740C12E9CD800D
:08E84000D5303DCB740A80E5E0
:10ED00007F797E24E55F30E70122AC5F1CAB7B128C
:10ED100061EAE51B700E742012E9B2EE2405FE12C2
:10ED2000ED4E800C12ED4EE51B12E998EE2405FE27
:10ED3000E51A12E998EE2405FE742C12E9B20E0EC3
:10ED4000E51912E998EE2405FE745E02E9B2742D0D
:10ED5000201702742B12E9B2EE2406FE22E55F3082
:10ED6000E70122AC5F1CAB7B1261EAE51B700E74FD
:10ED70002012E980EE2404FE12EDA7800C12EDA70C
:10ED8000E51B12E96DEE2404FEE51A12E96DEE248E
:10ED900004FE742C12E9800E0EE51912E96DEE24C2
:10EDA00004FE742A02E980742D201702742B12E9E4
:06EDB00080EE2404FE22A7
:10E5BA007F097E2530040512E6B48028A275E57924
:10E5CA00C23D6002D23D92D175F080305C04F5F014
:10E5DA008001A4A2E792D5E5F075F03284F8E5F05F
:10E5EA0075F00584C0E0E5F0A2D533C0E0E8602A02
:10E5FA0012E9CDEE2408FED0E0F8D0E012E9CDEE23
:10E60A002408FE0F0FE52B5403701F746012E9B241
:10E61A001F1FEE2404FEE802E9CD740C303D067497
:10E62A000A20D1010412E9CD80C9205904742E8030
:10E63A00DC205804747F80D5748080D130040512A0
:10E64A00E6B48028A275E579C23D6002D23D92D136
:10E65A0075F080305C04F5F08001A4A2E792D5E55C
:10E66A00F075F03284F8E5F075F00584C0E0E5F065
:10E67A00A2D533C0E07F3E7E1CE8602012EA2ED08D
:10E68A00E0F8D0E07F3E7E2812EA2E7F447E327484
:10E69A002E12E9B27F3E7E37E802EA2E303DE07460
:10E6AA000A20D1010412EA2E80D59005CAE075F03D
:10E6BA000A84F8E4C5F0C2D522301105E54AB4024D
:10E6CA0050C39006E9E0957AFB9006E8E0955EFC77
:06E6DA0050031264ADECD8
:10E6E000C31360047B63800FEB13FB249C40F52471
:10E6F0004F4004C20480079005CAEBF0D204900694
:10E70000E6E09006E8F09006E7E09006E9F0E55EC6
:10E710009006E6F0E57A9006E7F02212E6FE80DE4B
:10DF7E00E54424F64001227800E552206607C39559
:10DF8E0070500224B40475F00384F9E928FE24C409
:10DF9E005001FE12DFC012DFCC1E12F2E3C3E9986D
:10DFAE00FE5003243CFE12DFC01E12F2E308B81F1F
:10DFBE00DA22EE2420FE24C250032402FE22E8249C
:10DFCE00F1E8C2D55006D2D5E8F4241F23FF90E025
:10DFDE004E93CF0493FAE545F5F0A4ACF0FB126234
:10DFEE004BE544F5F0A49BFBE5F09CFCEB2420FBF9
:10DFFE00EC3400FC12E02FFAE5458FF0A430E70276
:10E00E0005F0E5F020D502F4042A75F00520190379
:10E01E0075F00384FF24DF50027F20C374329FFF0C
:10E02E0022EC24F0500BEB2460EC340090E09E9335
:10E03E0022EB33FBEC33FCEB33EC3390E06E9322AC
:10E04E00FF00FF03FA0BF318EA2ADE40CF58BE7327
:10E05E00AB8D96A880C068D64FE835F51BFD00FF46
:10E06E0000080B0E101214151718191B1C1D1E1F5D
:10E07E0020212223242526262728292A2A2B2C2D27
:10E08E002D2E2F2F3031313233333434353636375F
:10E09E00373839393A3A3B3B3C3C3D3D3E3E3F3FBB
:10E0AE004042444648494B4D4E505253555658598E
:10E0BE005B5C5D5F60616364656668696A6B6D6E0B
:10E0CE006F7071727374767778797A7B7C7D7E7FD0
:10E0DE00808182838485868788898A8B8B8C8D8EBE
:10E0EE008F9091929394949596979899999A9B9CC8
:10E0FE009D9E9E9FA0A1A2A2A3A4A5A6A6A7A8A9E5
:10E10E00A9AAABACACADAEAFAFB0B1B1B2B3B4B413
:10E11E00B5B6B6B7B8B9B9BABBBBBCBDBDBEBFBF4D
:10E12E00C0C1C1C2C3C3C4C5C5C6C7C7C8C8C9CA92
:10E13E00CACBCCCCCDCECECFCFD0D1D1D2D2D3D4E0
:10E14E00D4D5D5D6D7D7D8D8D9DADADBDBDCDDDD36
:10E15E00DEDEDFDFE0E1E1E2E2E3E3E4E5E5E6E691
:10E16E00E7E7E8E8E9EAEAEBEBECECEDEDEEEEEFF3
:10E17E00EFF0F1F1F2F2F3F3F4F4F5F5F6F6F7F75A
:10E18E00F8F8F9F9FAFAFBFBFCFCFDFDFEFEFFFFC9
:10E19E00E54524FD400122E552206607C3957050E7
:10E1AE000224B40475F00384241FFE24C2500324F9
:01E1BE00025E
:10E1BF00FE12DEB9EEFD241EFE24C250032402FE21
:10E1CF0012DEB9E544240275F00520190375F0033A
:10E1DF0084F4042432FF24EE500F12E1EEAE051E3C
:0AE1EF001E7C0512F2E30EDCFA229A
:10EA6D007E00206615E5700475F0B484E5F075F050
:10EA7D000384FE6004C3743C9EFE745312EA9874C2
:10EA8D005712EA98744E12EA9874457F2F12E98056
:10EA9D00BE00077E3C12E9807E00EE240875F03C36
:10EAAD0084AEF00F0F0F12F2E30E12F2E30F12F21B
:10EABD00E31E12F2E3EE240775F03C84AEF0223033
:10EACD00745C301259E54AB4040122B4060122E502
:10EADD007112E0188F057C037E1E30662AE57004E6
:10EAED0075F00384241EFE24C6501C24FB50042400
:10EAFD00038013C00612EB14D0E024C67C0160061F
:10EB0D000C1460020C14FE12EB200EEE24C1400218
:10EB1D00DCF5228D0712F2E30FEF24CE50F722E53C
:10EB2D0053206607C39570500224B40475F0038416
:10EB3D00241FFE24C250032402FE12EB4B0E7F2332
:08EB4D0012F2E30FBF2DF922C3
:100031007E0E78ADE612E8B3EE2405FE742C12E9CB
:10004100B20E0E0E18E612E8B3EE2405FE742C1261
:0A005100E9B20E0E0E18E602E8B345
:10E1F9007F017E00745212E9B27E06E51512E8B974
:10E209007F0A7E0178B8E67D0130E5027D03ED12D3
:10E21900E99F7E07E67D58A2E4922B50027D46EDE8
:10E2290012E9B27F017E181200337F0A7E1378AE9D
:10E23900E612E848EE2406FE743A12E9B2EE240525
:10E24900FEE53E12E848EE2406FE743A12E9B2EE03
:10E259002405FEE53F02E8487F797E00E54012E8A3
:10E26900B37E0A743B12E9AE7E0CE54102E8B37F46
:10E27900797E16743B12E9AE7E18E53F12E8B37F4A
:10E28900797E0078AEE612E8B37E0A743B12E9AEF5
:10E299007E0CE53E02E8B3305EE52043E27F6D7E09
:10E2A9000078AEE612E8B37E0A743B12E9AE7E0C42
:10E2B900E53E12E8B37F757E00E53E75F00A84E518
:10E2C900F012E9CD0F0F7E08743A12E9AE1F1F7ED6
:10E2D9000DE53F75F00A84C0F012E9CDEE2408FE81
:10E2E900D0E002E9CD851C1E851B1FAB1BAC1C3081
:10E2F9005D0A7A1B12622278321263C4C3EB33FBC4
:10E30900EC33FC923D1261F3303D087409F51DF5BB
:10E319001CF51B7F75E51D60157E2412E9CD7E2C49
:02E32900E51CF1
:10E32B0012E9CD7E34E51B12E9CD803D7E22E51C42
:10E33B00601912E9CD7E2AE51B12E9CD7F787E317B
:10E34B00742E12E9AE7F75E51A8019E51B12E9CD23
:10E35B007F787E29742E12E9AE7F757E2DE51A1219
:10E36B00E9CDE5197E3512E9CD7F777E3C126B83C3
:10E37B00851E1C851F1B227F397E1F12F2E30FBFE8
:10E38B0040F9781F79567A007D1A12F1A012F2A685
:10E39B00EA2406FABAAEF3781BC3E5119570500266
:10E3AB0024B4FA604214603E14603A2450603A146C
:10E3BB006036EA24A540278A1E751D007D1912E3DD
:10E3CB00D40D30740312E3D40D781F7956AA1DEACD
:10E3DB0012F1A012F2A60AD3EA951E40F2228A1D70
:10E3EB00751EB380D7080808087F367E1C90ECECAE
:10E3FB00E571700390ECF612E9DE7F3CAE00909372
:04E40B00E102E9DE63
:10EF1400787512EF647453201702744E207406E55A
:10EF24002E54074430AF1712EF8E7E3BE57DC45458
:10EF34000F12E99F2074077E07742012E9B27878D3
:10EF440012EF64E5172409FF745720170274452053
:10EF54007402742012EF8E7E3BE57D540F02E99F0C
:10EF6400E6FD3392171886041886033017031264DB
:10EF7400B5791778701263BF8B13AF06AED27C00DD
:10EF84007D6412632D8F148D15227E0012E9B27EEA
:10EF940007E51312E8657E19748112E9B27E20E553
:10EFA4001412E8487E2B742E2073030E742C12E97D
:08EFB400B27E2FE51502E848CA
:10F13000E54A602E7A2420E00E7A26141460087ABC
:10F1400028141460027A297F667E01EA12E9B2204F
:10F150005505205406800B745B8002745C7E00129F
:10F16000E9B220110778A9B60007802130261EC217
:10F170002690AFCC7F661285B57F64A85AE54AB465
:10F18000060108E875F06484E5F012E2DC20080F5F
:10F19000E537640260097F367E2E744112E98022D1
:10EDB60020144F740512F38AEF33EE33F9EF030391
:10EDC600541FF5F090EE09E993A4C5F013C5F013AE
:10EDD600C5F013C5F013C5F0135403FCE5F013FB9F
:10EDE600E9242093C9244093C39BC4540FFBE99C98
:10EDF600C4FC540FF9EC54F02B2446F57BE934F6A9
:10EE0600F55F22FFFFFFFFFFE6C5AD9C8F857D778F
:10EE1600726E6C6A696A6A6C6F747A828D9DB4D9F7
:10EE2600FFFFFFFAE9DCD3CEC9C6C3C0BEBBB9B784
:10EE3600B5B4B2B0AFADABAAA8A6A4A2A09E9C9949
:10EE460096918C00381CE735D137246F00C5B3C1C5
:10EE5600E61F66B60E68C21867AADBF4EDB94675FA
:03EE660010A200F7
:10F36A00D2A27408D2A1D2A300C2A3C2A1D2A3007E
:10F37A00C2A3D5E0EF7405D2A300C2A3D5E0F82258
:10F34300C2A3D2A2D2A1D2A300C2A375F008339262
:10F35300A1D2A300C2A3D5F0F5C2A175F003D2A335
:07F3630000C2A3D5F0F8225F
:10D8C20012F343D2A300C2A3C2A175F008E4D2A30B
:10D8D20000C2A3A2A233D5F0F5FE75F008E4D2A3EC
:10D8E20000C2A3A2A233D5F0F5FFD2A300C2A322A5
:10D8F200E478806608B88BFB70012274D512D8C216
:10D902007881C3EE13FEEF13F692D118EE2460F67F
:10D9120074D612D8C27888EF33CE33CE33CE33CE1C
:10D9220033A2D192E25407FCEEFB7A08126214ECA5
:10D93200244FF608EBF674D912D8C2EF543F78821E
:10D94200F67886EF33CE33CE33CE33CE335403F66E
:10D9520008EEF618161608E6C4FF54F0F618E6C4E8
:10D96200CF540F2FF674DA12D8C2EF232354FC7867
:10D9720083F67884EEF608EF54C0F67880E4660801
:10D98200B88AFBF62212D8CA7889C3EF96FF18EE3E
:08D9920096FEA2E79216501068
:10D99A0012649D740FF8F9126261EF2CFFEE3DFEDE
:10D9AA00788BEEF608EFF622E6182016072CF7E633
:10D9BA003D19F722C39CF7E69D80F66A405E8056C1
:10D9CA00E050F04B0044803DC0384031D02BA025B8
:10D9DA00601F2018D014000F000AA001440158014A
:10D9EA00680178018801A001B401D001EC0210029B
:10D9FA0038026802A002DA030C034D78BE80208543
:10DA0A008E8A9D8F4D95BA9A97A0BEA631AC53B215
:10DA1A002AB801BD6AC1EDC4D1C78812D8CA788DA7
:10DA2A00EEF608EFF67887798C126261788379903E
:10DA3A0012D9B27885798C1262617881799212D979
:10DA4A00B2788DE624E4FE08E63392D13392D554B7
:10DA5A00FCFFEEA2D133A2D533FE780F799212627F
:10DA6A006178947990C3EC97F61819ED97F6799442
:10DA7A0090D9C57F1F7D11EF93C3971F19EF939715
:10DA8A001F091DED600240EF0F90D9E5798DEF93E4
:10DA9A00F7090FEF93F7788E799412626190DA059D
:10DAAA00EF93C39BFB1FEF939C2420FC7897E62BF4
:10DABA00F618E63CF618E436F6740612F38AEEFC1B
:07DACA00EFFD740712F38A5F
:10DAD100C3ED9FFFEC9EFE78B7E6FD337C0050015D
:10DAE1001CEF2DFFEE3CFE789CEF26F618EE36F685
:10DAF1002220140F789DE6B4050912DB9212DBC7D0
:10DB010012DC0B222014577897799A12DC3C1264AC
:10DB110025C3EE9420FE9245500312649D7C007D46
:10DB21000512632D30450312649D8E618F60E531CE
:10DB3100B40C2B12EEFAE56120E71124F8500DFA2E
:10DB4100C3E5609AF560E5619400F561121A09E593
:10DB5100BC2560F57AE5BD3561F55E12EF07789772
:10DB6100799AC3E697FB1819E697FC7A02126214B8
:10DB710012DB9212DBC720140312DC0B7895799823
:10DB8100E6F776000809E6F776000809E6F7760079
:10DB910022799CE77700FB19E77700FC789DE6B4D2
:10DBA1000506EB33FBEC33FCECA2E792D5500312F4
:10DBB10064AD7A32126222ECFBEDFC30D5031264C3
:0ADBC100ADECFEEBFF22EE2408FE9F
:10DBCB007406307511789DE6B40504740C8007F467
:10DBDB002406C323540FFD7C00126200789FE6FCE1
:10DBEB0008E6FBC374109DFA126222EFF8EEF912ED
:10DBFB006425E878A02FF6FF18EE39F62480FE2274
:10DC0B009275400312649D78BBE6F5F0243840030F
:10DC1B0075F0E1EF33EE3378A8F6A485F07930E7B1
:10DC2B00020579C276307508E57924F15002D27677
:10DC3B0022E627FB1819E637FC1819E637FD227583
:10DC4B006A0079C6876C09876B22756A2080F3128C
:10DC5B00DC4A129CFC7F087871793A12DC7802A0BE
:10DC6B00DB855E63857A62787379647F06E6F708F5
:10DC7B0009DFFA227864797380F1787379AF80EBDE
:0DDC8B0078AF797380E5E6F008A3DFFA2298
:10619A00E4FEFFFC7D0A791DE7540F2FFFE43EFE63
:1061AA00B9190280061912620080ED3017031264D1
:1061BA009D22305C2BEC33921750031264ADEC2411
:1061CA00D950047C277B007AD2126222EB33CC337B
:1061DA00CD33CC33ED33FBEC33FC3017031264AD13
:1061EA00EC33921750031264AD791912643CF70923
:1061FA00B91DF8A70322EFF88DF0A4FFEDC5F0CE84
:10620A00A42EFEEC88F0A42EFE22EB8AF0A4FBE575
:10621A00F0CC8AF0A42CFC22EB8AF0A4FBE5F0CCAB
:10622A008AF0A42CFCE435F0FD22EB8AF0A4FBE50D
:10623A00F0CC8AF0A42CFCE435F0CD8AF0A42DFD34
:10624A0022EB8AF0A430E70205F0E5F0CC8AF0A44C
:10625A002CFBE435F0FC2286F0E7FDA4FAABF0193A
:06626A00E786F0A42BFB07
:10627000E435F0FC18E68DF0A42BFBEC35F0FCE4E3
:1062800033FDE687F0A42CFCED35F0FD22EB89F020
:10629000A4CBAEF08AF0A42EFEE5F03400FDEC892C
:1062A000F0A42EFEE5F03DFDE433CC8AF0A42DFDF4
:1062B000E5F03CCEFC22EB89F0A4CBAFF08AF0A451
:1062C0002FFFE5F03400FEEC89F0A42FFFE5F03E4F
:1062D000FEE433CC8AF0A42EFEE5F03CFCED89F020
:1062E000A42EFEE5F03CFCE433CD8AF0A42CFCE5C2
:1062F000F03D8E058C068F04FF22C2D5EC30E705F9
:10630000B2D51264A5EE30E70DB2D512649D1263CA
:106310002D1264A5800312632D30D50312649D22D3
:10632000C3EC13C0E0ED132FFFD0E03EFEBC000B2A
:10633000BE0029EF8DF084FFADF022E4CCF975F0BA
:0463400008EF2FFF34
:10634400EE33FEEC33FCEE9DEC994005FCEE9DFE35
:106354000FD5F0E9E4CEFD22EDF9F5F0EE8420D27C
:106364001CFEADF075F008EF2FFFED33FD400799EB
:106374005006D5F0F222C399FD0FD5F0EA22EC3392
:10638400EE3400FEEF3400FF7D007A0079007809D6
:10639400C3ED9AFDEE9BFEEF9CFFB392D54009ED51
:1063A4002AFDEE3BFEEF3CFFA2D5E933F9ED33FDC8
:1063B400EE33FEEF33FFD8D92279007A00C380157B
:1063C40079007A00C3EA13FFE913FEE8132BFBEE0E
:1063D4003CFCEF3DFDE4F5D2F5D333FE7F19C3EE6B
:1063E40098FEE5D299F5D2E5D39AF5D3B392D54088
:1063F4000DEE28FEE5D239F5D2E5D33AF5D3A2D590
:02640400EB3378
:10640600FBEC33FCED33FDDF0122EE33FEE5D23348
:10641600F5D2E5D333F5D380C3AD6FAC6EAB6DED7E
:10642600C454F0FEECC4FF540F2EFEEF54F0FFEB05
:10643600C4540F2FFF22EC75F00A84FCEB54F025B0
:10644600F0C475F00A84C4CBC454F025F0C475F0CA
:106456000A842BFBE5F022AC10AB1112643CA904B4
:10646600AD03FA7C197B99126214AE04AF03EA7588
:10647600F006A4F8AC12AB1312643C2875F00A843B
:1064860085F014F8EF2BFFEE3CFEEF28FFE43EFE0E
:10649600E43DFDE439FC22C3E49FFFE49EFE22E4D2
:1064A600C39DFDE49CFC22C3E49BFBE49CFC22C34D
:1064B600E49BFBE49CFCE49DFD2275D4107B807A72
:0C64C6000079807800EAF5F0A4FCADF04D
:1064D200EBF5F0A4FEAFF0EB8AF0A4C333C5F033C2
:1064E200C5F092D52DFDC5F03EFEE430D501043F46
:1064F200FFB5150DEEB51409EDB51305ECB5120196
:10650200224006EA98FAEB99FBD5D40ABB00012295
:106512000ABA00010B22C3E913F9E813F8EA28FAD0
:10652200EB39FB80A478087B807D807C00EDF5F060
:10653200A4FAE5F08EF0B5F007EA8FF0B5F001228B
:106542004003ED9BFDD827BDFF0122EDF5F0A4F934
:10655200A8F0ED04F5F0A4C399FAE5F09813CA1374
:1065620029F9E83AF8C3E99FE89E50010D22C3EBEE
:1065720013FBED2BFD80B6C374689511FB74019576
:1065820010FC8004AC10AB117A0B79B812628D80CA
:10659200177473F8F9E627FB0809E637FC0809E6E1
:0265A20037FDC3
:1065A40030E7031264B5EB33FBEC33FCED3323FD2E
:1065B400242083F8ED241C83FFED241883FAED24B2
:1065C4001483F9EF99F9E89AFA12628DEF9DFFE8C6
:1065D4009EFE22FFFFFFB6FED7FD63FB5DF8C4F508
:1065E4009BF1E3ED9EE8CFE379DD9ED743D06BC901
:1065F40019C153B91CB079A7709E06943F8A237FB2
:10660400B674FF6A045ECB535B47BB3BF130042393
:10661400FB17DE0BB2FF80C21DC232532CF8C3E558
:10662400679576FBE5689577FCE5699578FD30E735
:1066340005D2611264B524F050031266EFAA06A9CC
:10664400071262B6EC2480E43DFBF9F51AE43EFC43
:10665400FAF519E43F6002D23212628D8B128C1368
:106664008D148E15C3E5649573FBE5659574FCE59F
:10667400669575FD30E705D2621264B5EBF9F51F36
:10668400ECFAF51DED6002D2323032012212628D35
:10669400EB2512F512EC3513F513ED3514F514EE64
:1066A4003515F51540E10264C012661B20323BEB40
:1066B400242E40D3EA2401CB3400FC7A07793D121E
:1066C400628DC010C0118E108D118C128B13E4FCDE
:0E66D400FD7E077FD012D45685120385130277
:1066E200D011D010BB0005BA0002D21D22B261C384
:1066F20074809BFB74F59CFC74209DFD22204D69E7
:10670200204866303F637F697E0112DE697E1F1278
:10671200DEE475A7009004EDE0A2E792171392E77A
:10672200FC1582E013FB3017031264ADBC003AEB98
:10673200603720E73420E63110E513201707C374D1
:106742001F9BFE80027E1F12DED90EDBFA22FB2087
:1067520017097E00C374209BFB8008EB241FFE7484
:10676200209BFB12DED30EDBFA2275A7007583078E
:10677200E559C4440FF582E0A2E792522212DC8569
:1067820012676CC2E775F00A84FEAFF075A7045376
:1067920082F178641267F5AE0778671267F575A71C
:1067A20000E57DC4540FFEE57D540FFF7873126738
:1067B200E9AE0778761267E974AF1265951266AD95
:1067C2008B148A13120808ACCCAB017A0A12621439
:1067D200E5139B9004ECF0FBA3E5149CF0FCA2E70C
:1067E200923DD23F02DC8B86030886040886051898
:0967F200188006E0FBE0FCE0FD6C
:1067FB007A0A12623420E70CEB2EF608E43CF6081A
:10680B00E43DF622C3EB9EF608EC9400F608ED94FB
:10681B0000F622204D09204806C23F302A0522C22D
:10682B003380F6E54824F640F5E5580460F075A78B
:10683B0000758307E559C42408F582E0FEA3E0FF49
:10684B0012080874371268E1500B30381BC23878C5
:10685B00C58646801374321268E1400C203809D289
:10686B003878C5A646754600740D1268E1404A1289
:10687B00677F303D38201122204D1F20481C2040BF
:10688B0019BCFF16EB24325011D2401219E1E5BFAF
:10689B0075F019A4F536D22ED22F205238E5596552
:1068AB00586032204D2F20482CD2338028201109DC
:1068BB00204D06204803753600303319204D122029
:1068CB00480F12AE4B0559C3E558955950038558DF
:1068DB0059C233C2402229FBE435CCFCC3EB9FECFD
:1068EB009E22E558B4FF012285581175A7047583C4
:1068FB0007E54824F65002805C2012592029052018
:10690B002A02805112DC85E4F516F517751000127A
:0C691B006979E510700312DC7F126992AC
:10692700302910E51B2517F517F51BE51C3516F55E
:1069370016F51C12699F12DC7F0510C3E51195102F
:1069470050D175A70002DC8BE55AF51124F65003E8
:1069570075110A75A70475830675100012697912F7
:10696700699212699F0510C3E511951050EE75A73E
:106977000022E510C4F582E0E0F564E0F565E0F596
:1069870066E0F567E0F568E0F5692275A701126D25
:106997008B124C5F75A70422E9F0E51CF0E51BF0AC
:1069A70022E510C454F0F582E0F512E5822406F5DD
:1069B70082E0F511E0F51CE0F51B22E512B426157F
:1069C7007F757E34740D12E9CD20442575110012B0
:1069D700E382026AF07F6D7E3BE012E9B2E5137E47
:1069E7003512E9B2E5127E2F12E9B220440312E311
:1069F7008212E2EE026AF0202852E558B4FF012223
:106A070075A704758307E559F51030330965586094
:106A17000520480205101269A8E0F513305E07202B
:106A27004304E5376095E07F797E3D12E980E51301
:106A37007E3912E980E5127E3512E98030480B7FF6
:106A47007F7E3512F2E30EBE40F980392012012213
:106A570075A704758306855B101269A8305E0A2046
:026A67004307E3
:106A6900E5377003026C12E512700B7E3A7F797478
:106A79005D12E9B2800D75F06484E5F07E397F7AA4
:106A890012E900E537B4020512ACE38045B403020C
:106A99008040E51C7006E51B24FB5036E511F964BE
:106AA900B4602F20062CE537600D200C0AC3E99548
:106AB90070F9500324B4F9E912F1A0781D79547DD5
:106AC9001D90ECDEE53F20E00390ECE512F2A61202
:106AD900E9DE75177975161930280375161DE51243
:106AE90064266003126B3375A7009006E3E511F085
:106AF900A31219FAE5BC75F01970040475F014A411
:106B0900951BFBE5F0951CFC922450031264ADEC37
:106B1900F0A3EBF0C24FC263EC700EEB24E6400227
:106B2900D24FEB24C84002D26322E51C24ED402B4E
:106B3900AE1CAF1B126D557C007D3212632DC00552
:106B4900EFAF17AE1612E8B9CE2405CE742C12E9B0
:106B5900B20E0ED0E02312E8B3801B126D4C126BFB
:106B69008DCE2405CE742C12E9B2CE2402CEE8755E
:106B7900F0058412E998CE2404CE7422305D0274A3
:0D6B89008302E9AEEE243D50047EC37F4B35
:106B96007C017DF412632DC004C005EF6007AF17BA
:106BA600AE1612E8B9D007D0067C007D3212632DEE
:106BB600A805EFAF17AE16CE240ACE02E998126DDD
:106BC6004CEE2450305D03EE24A150047EC37F4B6F
:106BD6007C017DF412632DC004C005EF6007AF177A
:106BE6007E2F12E906D007D0067C007D3212632D77
:106BF600C005EFAF177E3712E96D7E3B742C12E9A4
:106C0600807E3DD0E075F0058402E96D7F6D7E2FB4
:106C1600746312E9B2E51275F06484E5F07E35120C
:106C2600E84812E38202E2EE30480320740122E4CF
:106C3600FCF5A79006E3E0F9A3E0FE24FE40EFA3EF
:106C4600E0FF7D78E5376008304FE3200C2A800BA3
:106C56001219E6E5BD20E010304F0DD206E571248D
:106C6600FE5015126D4280107D3CE546600A7D148B
:106C76001460057D0A1470B689111262007D6F12C8
:106C86006320BE00A9EF24E240A4AD07E51112F18E
:106C9600A0202404B2D5B2D1781F795612F2A6A844
:106CA60006A907E511242D75F0B484E5F012F1A0CC
:106CB6007407304F02740EFDFA12F2A6B2D5B2D1A5
:076CC60012F2A6B2D5B2D113
:106CCD00DDF0AD0212F2A6850616850717B2D5B214
:106CDD00D112F2A685061E85071F7A03304F027A60
:106CED0006E511241675F0B484E5F012F1A0A8168E
:106CFD00A917AD0212F2A6DDFBE51124EA4002242C
:106D0D00B412F1A0A81EA91FAD0212F2A6DDFBE57B
:106D1D00377021304F1E90B954305D0390B9507FBC
:106D2D003C7E331285FA1219E6E5BD20E00612DE2F
:106D3D00EA12EC7D22C3E99570500224B4F922E5E4
:106D4D001B2402FFE4351CFE305D1ABEC305BF4D8A
:106D5D00028012AC06AB077A1B12622278321263E4
:106D6D00C4AE04AF0322787379641265971266ADD1
:106D7D00751CC3751B4B2032048B1C8A1B22126D94
:106D8D007330320122AC19AE1AA91DAF1FB900051F
:106D9D00BC00028010C3E913F9EF13FFC3EC13FC21
:106DAD00EE13FE80E8BF29005006BE2900500122D7
:106DBD00C3EF13FFC3EE13FE80EB3E7FE3E3E3E38C
:106DCD00E3E3E3E3E3E37F3E0C1C3C7C7C1C1C1CF7
:106DDD001C1C1C1C7F7F3E7FE3E3E3070E1C3870F9
:106DED00E0E3FFFF3E7FE3E3030F0E0F03E3E3E377
:106DFD007F3E070F1F3F77E7E7FFFF0707070707EF
:106E0D00FFFFE0E0E0FEFF030303E3E37F3E1E3FF1
:106E1D0073E0E0E0FEFFE3E3E3E37F3EFFFFE3E348
:106E2D000303070E1C38383838383E7FE3E3E37F21
:106E3D003E7FE3E3E3E37F3E3E7FE3E3E3E37F3F38
:106E4D00030303E77E3C000000181818FFFF181815
:106E5D0018000000000000000000FFFF000000000F
:106E6D0000003FF00000381C38F00180C1F020F028
:106E7D00FC0038F03FE0000000007CC6C6C6C6C668
:106E8D00C6C6C67C1838781818181818187E7CC60F
:106E9D00C60C183060C0C6FE7CC6C6061C0606C6EB
:106EAD00C67C0C1C3C6CCCFE0C0C0C0CFEC0C0C08B
:106EBD00FC0606C6C67C3C66C0C0C0FCC6C6C67C09
:106ECD00FEC6C6060C18303030307CC6C6C67CC631
:106EDD00C6C6C67C7CC6C6C67E060606CC78000035
:106EED0018187E7E18180000000000007E7E00003D
:106EFD00000000000000000000000000C6E2E2D229
:106F0D00D2CACAC6C6C200000000000000000000C0
:106F1D008080A0C0A000304020C08080C0A0A00014
:106F2D000060A0600000A040A05098D09088205034
:106F3D00A850888850A8502060806000000040E074
:106F4D00400000000000800000E000000000000094
:106F5D0040002040800040A0A0A04040C04040E044
:106F6D00C02020C0E0E0204020E02060A0E020E034
:106F7D00C02020C06080E0A0E0E020404040E0A0C4
:106F8D00E0A0E0E0A0E020C0004000400000800054
:106F9D0080002060E0602000E000E00080C0E0C0E4
:106FAD0080E0E0E0E0E0000000000040A0E0A0A0F4
:106FBD00C0A0C0A0C040A080A040C0A0A0A0C0E0C4
:106FCD0080C080E0E080C080806080A0A060A0A034
:106FDD00E0A0A0E0404040E0202020A040A0A0C0C4
:106FED00A0A080808080E0A0E0A0A0A0A0E0E0E0D4
:106FFD00A040A0A0A040C0A0C0808040A0A0C060C4
:10700D00C0A0C0A0A060804020C0E040404040A093
:10701D00A0A0A060A0A0A0A040A0A0A0E0A0A0A0C3
:10702D0040A0A0A0A0404040E0204080E02020A84B
:0D703D0070202070A8202008F030D0100036
:10704A0000F0A8A8000000E0000000902048708826
:10705A0098984000E0E0E000A0E0E0E040603010F6
:10706A0030604040E0404060909090909060206096
:10707A002020202070609010204080F06090102026
:10708A0010906010305090F01010F080E0101090C6
:10709A0060609080E0909060F01020204040406056
:1070AA0090906090906060909070109060C0E0F056
:1070BA00F8F0E0C00000000000000000000000003E
:1070CA00000050605000707050000078807008F026
:1070DA0000F8888888F800C0C8102040981800C0B6
:1070EA00B098B0C000602040000000000090D8FCBA
:1070FA00D8900000246CFC6C24000020A870A82002
:10710A0000002020F820200000000000000080007D
:10711A000000F0000000000000000060600008109D
:10712A00204080007088888888887020602020200D
:10713A002070708808102040F8F810201008887015
:10714A0010305090F81010F880F00808887030401D
:10715A0080F0888870F80810204040407088887055
:10716A0088887070888878081060006060006060A5
:10717A000000008000008000002040F8402000004D
:10718A0000F800F80000002010F8102000708808AD
:10719A00102000200000000000000070888888F895
:1071AA008888F08888F08888F07088808080887065
:1071BA00E09088888890E0F88080F08080F8F880F5
:1071CA0080F0808080708880B8888878888888F87D
:1071DA008888887020202020207038101010109085
:1071EA00608890A0C0A09088808080808080F88885
:1071FA00D8A8A88888888888C8A89888887088881D
:10720A0088888870F08888F080808070888888A84C
:10721A009068F08888F0A0908870888070088870DC
:10722A00F8202020202020888888888888708888EC
:10723A008888885020888888A8A8A85088885020DC
:10724A0050888888888850202020F808102040809C
:10725A00F800CCAC9CACCC0000CCD4E4D4CC000478
:10726A00781828C800FC40A0401820201800000008
:10727A00000000F800000000A040A05000788888B4
:10728A009868708840308870200000F0A8A8A8A8E4
:10729A007848484848788870888080887020A8880C
:1072AA0098A8C88888805048FC485080304C5C6058
:1072BA0060603C00E0F0080808F88044485C4844F4
:1072CA0080F880808080808078484848484888B81C
:1072DA00A8A8E8A8A8B88888888888F808500070FC
:1072EA00888888708080F088888888F88888888864
:1072FA008888F09090909090F0A8A8A8A8A8A8F8DC
:10730A00888888F808080850008888888878A8A893
:10731A00A8A8A8F80800000000000000000000006B
:10732A0000000088888888E8A8E8A8A8A870A8A803
:10733A00A80000000000000000000000000000009B
:10734A000000000000000000000000000000000033
:10735A0060006060006000600060602050200000F3
:10736A0000005090B890D0908860505000707050D3
:10737A00008820208870000080C0A090F800304863
:10738A00B4B44830003048B4B44830FC0098D02037
:10739A0058C800F8E8D880D8E8F8404050F850407B
:0F73AA0040A0C0A000203828A0C0A010381018A4
:0B00000002005E000000000000000095
:03000B0002C4BE6E
:0C000E00206E06859950D26E32D26F32FF
:0E00230010990AC298206DE385994FD26D3274
:03005B000239B5B2
:10C4B1008530F0C5F065308530F060F722C0D0C01E
:10C4C100E0C0F0C0A775A700C083C08275D0087511
:10C4D1008A4E758CE9202B0C758A00300503758A0C
:10C4E1007A758CEA0532E532700215320530E53095
:10C4F100640A6026201520E531B40C0BE530B40147
:10C501000612C9C012EDB6E531B4180BE530B40618
:10C511000612C9C012EDB602C6E1C2AFD2C075C0E3
:10C521007AD2AFF5300531E53164197040F531202B
:10C531001529C225C22C7D0A740412F38AEF33EE49
:10C54100339005CCF0EE24F540112402400B240178
:10C551004005DDE40239B5D225D22CE5A6600215ED
:10C56100A678B5E660011678B6E6600116302E0BA6
:10C57100E5367007C22FC22E12C8A5E5367004C277
:10C581004B8002153678A9E660011678D8E660017D
:10C59100160535E53570021535E590307B0B30E039
:10C5A10008D278C27BC200801A307C0B30E108D2FD
:10C5B10079C27CC201800C307D0930E206D27AC298
:10C5C1007DC202E59044F8F47003753500304A09E4
:10C5D100E53324FA5003753305E53360051533025D
:10C5E100C686E590F45407700302C686A2E0920065
:10C5F100A2E19201A2E2920230100320143D7533B0
:10C601000820001B20100C2011098013E59030E157
:10C611000E8006E53724FC40F3E543541FF5332033
:10C62100100375A6FF202E5D301004E536705620EC
:10C63100100C201109E53524F55003753304D21B84
:10C64100D2A5D2A612C8A575B44075B24078D8E675
:10C651007002053420272E20682B202928202A2526
:10C66100A2107211501FE52054076019E5342437D8
:10C671005004C24A800F2401400B200026200119DA
:10C68100D27D7534C8201558E531702412F36A74CF
:10C69100E812F343802A02C7E8E53724FC40E6D2DA
:10C6A1007C80DF3011DFE53724FC40D9D27B80D29A
:10C6B10075F00384E5F070DE12D98774E812F34354
:10C6C100E531B4060512DAF28016B40C0512DB0569
:10C6D100800EB4120512DAF28006B4180312DB05DB
:10C6E100201421203705201A02801990C70FE53246
:10C6F100C4540F93FAE532540F60096A7006121898
:10C701003B1218A1E59030E11530E21280160102CA
:10C711000404040405050607070809090A00201096
:10C721000820110520103C807D2027F82068F52085
:10C7310029F2202AEFE534243040E9240750E5604E
:10C741000B205E088590F020F202740190C75D9382
:10C75100D2A5201002C2A512C890806FC8A082691C
:0AC76100554646202F12E536603CD5
:10C76B0024AA500AE53675F01984E5F06040D2A68C
:10C77B00201002C2A6D2A5202F0C7418304B0274C5
:10C78B006412C890803BE53675F00C30480375F0A9
:10C79B000684A2E0744640E9743780E5E52B540328
:10C7AB00600C20100E301106E54A6402600512C8B9
:10C7BB00AB800312C800101B08A25892A5A2599275
:10C7CB00A675A700D082D083D0A7D0F0D0E0D0D070
:10C7DB00201009C5A670030239B5C5A632C218B41C
:10C7EB000202D21812DA2530180874E412F343024D
:10C7FB00C6C102C6BC78A7E5B4600924E040057643
:10C80B000002C8ABE534702920412220751F300D82
:10C81B001CE57924CE40167AFFE5B110E7010A2317
:10C82B0025B3F5B3EA35B4F5B4C313F5B2E660023C
:10C83B001622C2412075028077C246E579FF605807
:10C84B0020120424FD5051206502C21CD265EF2436
:10C85B00B050027F4FEF90C9709375C70375C6FC3C
:10C86B0075B90185BFF0A4E5F0F624F44002760C0F
:10C87B00301C2DE5BEC39FF5F0A4E5F024E040038A
:10C88B0075F020E5F0C21C79AA770375B300F5B4F7
:0CC89B00C31375B100F5B222C26578A786
:10C8A7007680D24179AA7703D21CE4F5B3F5B4F5C3
:10C8B700B1F5B222C26579A1E57924CE500DE72002
:10C8C700E7E27628301CDD743C80BE7680E720E7FF
:10C8D700D3E57997404DC24679AAE7FAE57923234C
:10C8E700B4C500400274C42437300E31F424373005
:10C8F7000D15F7BA0302FA0AC39AF5B175B300EA40
:10C90700F5B4C313F5B222101C07D21C76C802C8AF
:10C9170092763274FF200E02749B02C892C31324CE
:10C927007E80CC75C70375C6FB75B901E5BD60266A
:10C93700C395795004C246801D78A720461B301C3A
:10C9470011E57975F008A42432F6E5792324AA02C3
:10C95700C8907605D24602C8AB301C0776147478A7
:10C9670002C8907696C24680EDFFF3E8DDD3C9C0D2
:10C97700B8B0A9A29A948F8A85817D7975716E6BFB
:10C987006865625F5C595653504E4C4A484644426C
:10C99700403E3C3A383634333231302F2E2D2C2B53
:10C9A7002A2928272625252424232322222121203A
:10C9B700201F1F1E1E1D1D1C1CD2B5C28EAE8DAAA8
:10C9C7008DAF8BAB8BE4F58DF58BD28E30140122B6
:10C9D70078B6BE0007EF24E24002800806E624ECA2
:10C9E70050027614206705E624F64005E4FEFAFFB8
:10C9F700FB7C007D0A1262007C007D5E1263208F43
:10CA070051EE60037551FFEAFC7A33126214EBF5BD
:01CA1700F02E
:10CA1800A4E5F0CB8CF0A425E0C5F035E0CB92D5A9
:10CA280025F050060BBB0002D2D530E7060BBB0041
:10CA380002D2D5ECF5F0A42BFBE5F03400FC30D5A0
:10CA4800010C78A6E6C39BFF18E608F6EB18F61863
:10CA5800E69CFE18E608F6EC18F6301401227A0077
:10CA680050040A12649D7C007D6E1263208FF0785A
:10CA7800A2E6A4FBACF012643CEBBA0002F404FAA0
:10CA8800E4F8FFEA30E70118E57960062075031F2E
:10CA9800F4042AF579EF38D27520E7086003757930
:10CAA800FF02DC2EC2750470F5E579F40460EFF539
:10CAB8007980EE1219DC78BBA6BC1219FAE5BE78AB
:10CAC800A2F624F65007E4F5BEF61257AF120C2C66
:10CAD800E5BEF54824F65008E4F5BEF5481257AF10
:10CAE800E5BFF54324F3503924F340351219F078A3
:10CAF800A1A6BCE5BF789DF61424FB50087403F684
:10CB0800F5BF1257AF78B7A6BE1219E6E5BDA2E386
:02CB1800926623
:10CB1A00A2E49267035403C253B40102D2532274AB
:10CB2A000DF5BFF5431257AF80C0E56A700CE56B8F
:10CB3A0054037006129D0E12CB9E75F08412CBD64A
:10CB4A00787086F708B880FAD2B275F08812CBC42A
:10CB5A00782575F000758002C2B275F7D7E4F5F74B
:10CB6A000000E5F7D2B220E705D5F0E9D8E722754B
:10CB7A00F08412CBD68DF7A4D2B280CE75F084128F
:10CB8A00CBD675F00075F7FFD5F0FAD2B222756BE5
:10CB9A00EC756A00758002C2B275F78475F7007584
:10CBAA00F70075F700780075F7FF75F7FF75F7FF5F
:10CBBA0075F7FFD8F2D2B275F08112CBD6D2B28015
:10CBCA008F75F05312CBC4808775F003758002C24B
:10CBDA00B285F0F7856CF7856BF7856AF72275F0F1
:10CBEA0003758002C2B285F0F7856FF7856EF78507
:10CBFA006DF7221255EB12CD4A745212F06B744D36
:10CC0A0012F06B744312F06B12CD5912F0B37441E7
:10CC1A00207402745612F06B12CCA612CCF012F0E9
:10CC2A00B3E53C12F05EE53B12F05EE53A12F05EC7
:10CC3A0012CD2612F0B3744512F06B12CD8F12CDBD
:10CC4A004A744712F06B744712F06B744112F06B1E
:10CC5A0012CD5912CCA612F0B3E43074010412F0CA
:10CC6A006912F0B39004C3E012F05E12F0B39004BC
:0FCC7A00E4E075F00A84AFF012F05E12F0B7EF4D
:10CC890012F069AC5EAB7A12CD6BAC5DAB5C12CDC8
:10CC99006B12F0B312F0B312CD8F0255BF7875C283
:10CCA9003D12CCB17878D23D12F0B31290D1303D1B
:10CCB90005E51E12F069E51D12F06912CD33E5187C
:10CCC90012F069E57D203D01C4540F12F06912F09C
:10CCD900B3303D09744530170274578007744E30DC
:10CCE9001702745302F06B20740812CD2612CD2658
:10CCF900802775A7049004BFE0FCE0FB7A1B126251
:10CD09002278321263C41261EA12CD309004C1E074
:10CD1900FCE0FB1261EA12CD3075A7002212F0B3D4
:10CD2900E4F51AF519800D12F0B3E51C12F069E566
:10CD39001B12F069E51A12F06912F0B7E51902F051
:10CD490069742412F06B744712F0BB745002F06BD3
:10CD590012F0B3E53D12F05EE53E12F05EE53F02EA
:10CD6900F05E12912D12F0B3E51D12F06B781CE6FE
:10CD790012F06918B817F812F0B7E412F06912F056
:10CD8900B3744D02F06BC038742A12F06BD03812AC
:05CD9900F09202F21B04
:10005E00D2B47581C075AF017590F878FFE4F6D80B
:10006E00FDF4F5A6D2C075C07A75F83075D7507507
:10007E00AE1375AF017581D87590F875EFBC75FD2F
:10008E00FFC2B7D2A412F20DC2A474501239D075A9
:10009E008951D28C75A882D2BC129DCC12F36A12F1
:1000AE00D8FD12CABB12EE6912387A7F407E0190DB
:1000BE00AEB71285C712561012F20D12EFBC12F225
:1000CE005112F2477C1412F2173000030239A5DCEC
:1000DE00F5125EE4753A00125F32E53A701612F3CD
:1000EE009E7F437E0690B73A1285C712F2513000BA
:1000FE00FD0239A575A6FF125EE412CABB12387A4C
:10010E0012F25112F20912F24778B5761E12EE690A
:10011E0012D8F2C215C21412387A90AEFF7F78123E
:10012E0085B5205E0A7F767E1290AF0C12E9DE7FD7
:10013E00401200317F497E0912E237E53F20E00888
:10014E0005A6E5A6700215A67F5312DE5D7F577ECB
:10015E000B12E77512E7FD7F602073102074097E85
:10016E002BE52E540712E99F7E17800E7E0BAC5D99
:10017E00AB5C12E77912E7FD7E311286517F697E04
:10018E001212ED043025087E1290F02512E9DEE5FC
:10019E00A60303543FFDFE0D7F7312F2E30F12F21E
:1001AE00E31EDDF478B5E57124F64002761E307458
:0A01BE0019E660457F727E1674405A
:1001C80012E9807E17E612E9067E1F745312E98051
:1001D80012F2511000261001261002261255BFD225
:1001E800AC75369612F0E8B4E005125F7A800AE53D
:1001F8003670F1125ED212F20602011B0239A50214
:100208003BF88061E53524C85046E59020E241D0AE
:10021800E0D0E012025902821BE53524D25031E5C4
:100228009020E22CD0E0D0E08038E53524D2502070
:10023800E59020E21BD0E0D0E012F39E306B0B7FFC
:10024800091285AC1257E7128A8C1202590205A6C8
:100258002212F39E90B7F07F001285B512F2510278
:10026800F20612F236C215C214C227C26812F24749
:1002780075370190AFE91228E590028573020105F0
:100288000223B0020A3E022C840205A60205E302FC
:10029800821B0202A002055212F24775370790B37B
:1002A800781228E59002B07302026D020853020822
:1002B8008D0208C10202D10204410202A00202A07A
:1002C8000202EF0202D60258B7125F35802A7F5128
:1002D8007E00747212E9AE122A4E40BC1256FB120E
:1002E800EE6912CABB80B17F49A25E120C17925EFA
:1002F800120C3680A31257AF12F24775370290B529
:100308003A1228E5900310730202A0021A27021A73
:100318008C021AE0021B35021B79021B880203714A
:100328000203A7021F490203317F5B121A1D12192B
:10033800FFA8BE12035512F2511000081001071051
:06034800020780EF181807
:10034E000880EA88BE80A85300037F5A7E0590B5C8
:10035E008CE875F00BA42582F582E5F03583F583E4
:10036E000285C77F40121A1D1219FFE5BCF8E87FFF
:10037E003F7E3212E8BF12F25110000810010D102C
:10038E00021280EA18B84AE6787D80E208B87EDE6E
:10039E00784B80DA88BC0202FD12F39E7F0F90B973
:1003AE00E31285B5122A0412F251C214C21512F2CA
:1003BE00067510651000DFE53170F9E510646570A3
:1003CE000D855E14857A15E4F512F513800C78A868
:1003DE00E51326F513E43512F5127F1E7E19E5108E
:1003EE0012E865C3E57A9515F517E55E9514F516D1
:1003FE007F287E0BAC16AB1712E77912E7FD12F2CF
:10040E005112F217D510ADAB17E516FC30E70312FB
:10041E0064AD7A0A790012628DA912A8131263C60E
:10042E00EBF510243840037510C81219DC8510BC8A
:10043E000202FD12F39E90AF447F017E091285C722
:10044E0090AF4C7F0A7E091285C77F1312DE557559
:10045E0017001219EBE5BC120521E5BD120521E5C9
:10046E00BE120521E5BF12052190AF9C7F5F7E066F
:10047E001285C7122A9012F251751700120501103B
:10048E00000810011510024880F20517E51724F731
:0C049E00500375170075100080E2E51790
:1004AA00640870151219EB75BC0175BD2375BE453C
:1004BA0075BF671257AF020441E51012053312F2F5
:1004CA00511204E10510531007E51724FE400353A7
:1004DA00100380AC0202A0A9BCAABDABBEACBFE5AA
:1004EA00171304F8E640085407C42510C4800454BE
:1004FA00702510F6028C707800E875F009A42417AC
:10050A00FF7E3B7D20E8651770027D89ED12E9B216
:10051A0008B809E502F251F8C4120527E8120533B2
:10052A007E030517E51702E99F540775F009A490A1
:10053A00AF542582F58250020583E51775F009A4A8
:10054A002417FF7E0C0285C712F24775370890B64A
:10055A00321228E59005627302010202058402152F
:10056A0092021318020D4502584502057D020552F2
:10057A000214437F3712227080CE7F0A121A1D128C
:10058A000C2C1221F812F251100008100105100269
:10059A000680EFB25A80EB120C3680ACC26812F2B7
:1005AA004775370590B1241228E59005B873020201
:1005BA006D02880502884A0289EB0205A60205DC5B
:1005CA0002892D0289930223790205A602235F027A
:1005DA000B487F2E12227080C312F247753706909D
:1005EA00B1FF1228E59005F37302026D0223B602E9
:1005FA00241802249102255E02259002260702068B
:07060A003802063102265000
:100611000226F50206177F641219E6E5BDA2E7126C
:100621000C171219E6E5BD92E7F5BD1257AF80B27E
:100631007F4912227080AB1207F41239F712F39E30
:100641001229DEE55804607790B2CE1206E112A4B9
:100651002012F25110000810011310021C80F50540
:1006610059C3E558955950D575590080D01559E5AC
:100671005930E7C985585980C4E559B40F02802F14
:10068100B51F02802A75F007A42408F517751627EF
:1006910074B82559F987001206CF12F251100028BB
:1006A10010012810020280F574B82559F9A700E558
:1006B1003524FA508878C7A6481207EB12F39E1228
:1006C100F25112F2090205E31880CC0880C9E875DD
:1006D100F005A485F01CF51BC000126B33D000227D
:1006E10012A4B1B4FF0122751000751FFF12A4C836
:1006F100E510640F6017120718401274B82510F83E
:10070100E675F005A485F01CF51B126BC40510C33A
:10071100E558951050D722121D2DF8602E64046003
:100721002AE814B51025F51F1219FAE5BC70060464
:1007310075F014800375F019A485F01CF51B126B7C
:10074100C47E2290B9841285FAD322C322E558B41B
:0C075100FF0122751000E510640F602EFF
:10075D00E51075F007A42409FF74B82510F8E6120A
:10076D0007D575F00A84C0F07E2012E9067E287444
:10077D002C12E980D0E07E2A12E96D120795051042
:10078D00C3E558951050C322121D2DF8603964042D
:10079D006035E8146510702F1219FAE5BC1207D5F3
:1007AD00F8C313923D7E1C12E91C7E28742C12E9AD
:1007BD0080E4303D067405B80001147E2A12E96DFF
:1007CD007E18742312E98022305D1275F036A42450
:1007DD0032FBE435F0FC12643C12643CEB22120750
:1007ED00FD12859ADFFB221207FD128D80DFFB22A1
:1007FD0075C70375C6F078B87F042275C70375C633
:10080D00F375B901E5BFB54831E55924F1402BE544
:10081D005975F00484A9F024F0F5C675B901C5F039
:10082D00A9BC600CA9BD146007A9BE146002A9BFC4
:10083D00E975F005A4F985F0CC221219FAA9BD7558
:10084D00CC00221257AF12F24775370390B3D8126E
:10085D0028E5900863730202A0020B61021E9E023E
:10086D000B76020B810222D7021F62020C42021F7D
:10087D0096021FDC022326021F180220211257AFF9
:10088D0012F24775370490B4951228E590089D73C0
:09089D000202A0020B90020B9B69
:1008A60002088D020BB1020BBC021BA202088D02CC
:1008B6000BCB020BA6020BE51257AF12F2477537A8
:1008C6000B90B4E41228E59008D1730202A0021C32
:1008D60050021C500209570209950208F802091B2A
:1008E6000223BC021CF5021DBD021D66021E4E023D
:1008F6000BFF1219E6E5BF1470C17F2E121A1D1FD9
:100906001219E6E5BDA2E6120C171219E6E5BD922C
:10091600E6F5BD80A37F37121A1D1219E1A8BFE8BC
:1009260012094F12F25110000810010D1002128028
:10093600EE18B802EA780A80E608B80BE278038077
:10094600DE1219E188BF0208BE7F367E2CE802E877
:100956004E7F1C121A1D1219E6A8BE12098912F240
:100966005110000810010D10021480EF18B800EBAA
:10097600780B80E708E824F450E1780180DD88BE32
:100986000208BE7F1B7E35E875F005A402E8487FA5
:1009960025121A1D1219E6A8BF1209C712F2511024
:1009A600000810010D10021480EF18B800EB78094A
:1009B60080E708E824F650E1780180DD88BF020868
:1009C600BE7F247E3BE802E99F1219DCE5BF75F085
:1009D6003CA4ACF0FDE5BE75F005A42DFDE5F03CAC
:1009E600FC1219E6E5BF14603675F005A485BEF065
:0609F600A42DFFE5F03C1A
:1009FC00FE7C007D3C12632DC005EF75F01884E57C
:100A0C00F07F2D7E2412E8487E30743A12E9B27ED3
:100A1C0035D0E012E84802F2517F2D7E0590B9A640
:100A2C001285C71219E6E5BDA2E67F2D1221EA0256
:100A3C00F25112F39E1229DE120A4A02026D7F173E
:100A4C007E0290B0471285C77F4C7E0290B05E123A
:100A5C0085C7AC5DAB5C7F577E0412E7F5121A09B3
:100A6C0085BC6285BD63E56124F8404490B0697F24
:100A7C00371285B5AE61AF607C017D5E12632DC30C
:100A8C00741F9FFAAC63AB62EC3392175003126481
:100A9C00AD126214AB047C003017031264AD74F514
:100AAC002BFB74033CFC1261EA7F377E1512E76D59
:100ABC0090B0767F697E0F1285C7E560240FFBE44A
:100ACC003561FCA25C923BD25C7E1E12E779A23BA4
:100ADC00925C7E30742012E9B27E36742012E9B238
:100AEC00E5602562FBE5613563FC7F227E0412E73D
:100AFC00F5E56245637016742E7E3A12E9B212F275
:100B0C005110000D100115100226020A727420807B
:100B1C00E81562E562B4FF0C156380080562E562B6
:100B2C0070020563E53524F55003753301020A7232
:0E0B3C00121A098562BC8563BD0257AF7F6344
:100B4A007E00747212E9AE122A4E40087F63128543
:100B5A00AC1257B60205A61219F0E5BCA2E77F0A45
:100B6A00120C1AE5BC92E7F5BC0208507F1CA20DD4
:100B7A00120C17920D80097F25A20E120C17920EE5
:100B8A00120C360208537F0AA20F120C17920F801A
:100B9A002A7F13A208120C179208801F7F52A20CF8
:100BAA00120C17920C80147F25A20B120C17920BB1
:100BBA0080097F2DA209120C179209120C3602081D
:100BCA008D7F491219E6E5BDA2E3120C171219E648
:100BDA00E5BD92E39266F5BD02088A7F5B1219E6CB
:100BEA00E5BDA2E5120C171219E6E5BD92E592439E
:100BFA00F5BD02088A7F6D1219E6E5BDA2E0120C66
:100C0A00171219E6E5BD92E0F5BD0208BE120C2CDA
:100C1A008F1F9217121A1DAF1F1F7E391292CBA275
:100C2A0017221219F585BC2B85BD21221219F585CB
:100C3A002BBC8521BD0257AF1219F085BE12120CCA
:100C4A00571219F08512BE1257AF02085375A6FF44
:100C5A0012F39E12C4B1740712F38A8FF07406124B
:100C6A00F38AEF2512C395F0A2E7923D4010FD24C6
:100C7A00CD50027D32AC05C3743F9DFD800FF40454
:100C8A00FD24C850027D37AC0574402DFD7F40120B
:040C9A00DE557E1293
:100C9E0012F2E30EBE1EF91F303D020F0FEF6D7004
:100CAE00EDE536700A753606EC2513F5148C131225
:100CBE000CD512F251100007100108300207221550
:100CCE00128002051280827F377E28742E12E9B2BE
:100CDE007F347E21740A303D010412E9CDE514FC07
:100CEE00249C50027C637F347E2DEC12E2DC7F4329
:100CFE007E1E12E7757E00E51212E90C7F057E025C
:100D0E0090B4691285C77F6D7E0190B4741285FA16
:100D1E007F747E0490B4861285FA0229DE90B0802C
:100D2E007F1B7E101285C712F25112F206C214C238
:100D3E001512F236020552D214D215E4F56EF56D87
:100D4E00756F02751501751401754280D233120D3F
:100D5E00C4E5156514600585151480F0C24D12F3B7
:100D6E009E1288FB90B6021285F8129F5578B8E64F
:100D7E000460AA751000D24E12121F304D07C24DDC
:100D8E0012F20DC202C233100008100129100248DF
:100D9E0080F3E5151460C7D2D5129E56E56F24FE7A
:100DAE00400430339222129F5578B8E630E6EA308E
:100DBE00D5221515801E129E36E56F24F2500512AF
:100DCE009E568010129F5578B8E630E6E9C2D504DB
:0F0DDE0060C7051530338722E53514601324BE36
:100DED005003020D3B2419509D122A1212F251800C
:100DFD0095E4F511F5121229DEE511451070087F05
:100E0D007B90B1E91285F812E1F91211F9851112F1
:100E1D0012F251E51110001310013410020280F38B
:100E2D00E53524E65056D24D020D6C600415118047
:100E3D0015E5107003020F13151012F39E12121DFB
:100E4D007407F511F5127F4212A0AEDFFB80A724C7
:100E5D00F940157479951775F00D8414D3951140DB
:100E6D00B2051112A077808E203CA8303DA505104B
:100E7D0012F39E12121D12A077020DFE783A7971AF
:100E8D0012DC76854E63854D62120FF3756C7F759E
:100E9D006BE8756AA512F39E122AA212E1F91211DE
:100EAD006C1217381217D812181812F251100008B8
:100EBD0010011810023780F5120FCFE56B24184082
:100ECD0005120FE2801C12A0AE8017120FE2E56B27
:100EDD002414500BE56A24135005120FCF80031212
:100EED00A07FE53524F550AD75330180A878717973
:100EFD003A12DC7685634E85624D754C0012F39E79
:100F0D0012121D020E03122ABE12F251100005100C
:100F1D00010580F8020E03C2531255EB122A12740A
:100F2D004012F0BB747812F06B746312F06B74673F
:100F3D0012F06B742312F05E12335BE51512F04A5A
:0F0F4D0078B8E6C4540344400412F06B12F092DB
:100F5C00E4F514129D9E129EA4747012F0BBE5145D
:100F6C0012F04A75A700900401E012F05EA3E012A3
:100F7C00F05EA3E012F05EA3E012F05EA3E012F0CC
:100F8C005EA3E012F05E12F0927F7B7E1DE51412E0
:100F9C00E91C12F25110022875A700900422751357
:100FAC004275120F753800E012F04AA3D512F812F0
:100FBC00F092D513EC0514303C9C1231F412F2175C
:100FCC00020E0374F1256AF56AE56B34FFF56BE5E7
:100FDC006C34FFF56C22740F256AF56AE4356BF5F9
:100FEC006BE4356CF56C22756C7F756BE812CB9BE2
:100FFC00E5104511C2306002D230303B02806030C7
:10100C003011E511129D9E129E99129EE990055B7E
:10101C00121159E511129D9E129ED7900411756AFA
:10102C00A5121152056B7FEF12115B129EE9900411
:10103C0011056B756A94121152056B7F6C12115B62
:10104C0012CB987F8312115B129ECC129ED7900408
:10105C0000E020E609900411756A831211592230C0
:10106C003011E511129D9E129E99129EE912110BE0
:10107C00121156E511129D9E129ED712110B756A14
:10108C00A5121156129EE912110B056B756A4A12C4
:10109C001156129ECC129ED7900400E020E65D12F1
:1010AC00110B756AEF121156129EE912110B056B9A
:0F10BC00756A94121156129ECC129ED7900400A2
:1010CB00E020E63912110B056B756A3912115612B5
:1010DB009EE912110B756ADE7F2290061012115BCE
:1010EB0012CB987F8312115B129ECC129ED7900469
:1010FB0000E020E60812110B756A83804E02CB9834
:10110B0075A70190061005A7900411AE838E16AF3C
:10111B00828F17E0F54512130BF54412130BF553A1
:10112B007C007D2D12632DED64146006851683857E
:10113B0017821218F412652705A7EDF0A305A7A3D4
:10114B00E58324FA50C5227F0080059006107FA509
:10115B0075F08412CBD6E0F5F7A3DFFAD2B202CB4F
:10116B0054C06FC06EC06D756F7F756EE8756D0086
:10117B0012CBE87517237E00D2D57B0579FF7A0059
:10118B007C1520D5011CE4F5F7E4ADF71212EC2029
:10119B00320CB501005001F9B502004001FADCE652
:1011AB00C3EA9904FAE904F5F0EA141445F0700364
:1011BB00E4F9FAAF01EA600612F2E30FDAFADB0B9D
:1011CB0010D506D2D57B0580027B030EBE40ADD277
:1011DB00B27E087F2412F2E37F2812F2E37E3712ED
:1011EB00F2E37F2412F2E3D06DD06ED06F22E512C2
:0911FB0075F00DA4FF74739FFF51
:101204007E00742012E980E51175F00DA4FF74735B
:101214009FFF7E00743F02E980C24EE4129D9E123D
:10122400E1F975177912123C203C0C203D09304E2F
:10123400F4E53524FA50EE22751201129EA4C23D43
:1012440075A700900400E0F5F0A2E5923BB4FF031B
:10125400D23C22E5176479600320F6F490042275E9
:10126400160475130FE51654014410F514E0FD300F
:101274003B2AF545C083C08212130BF54412130BAD
:10128400F5531218F4AC06AB0712E02FFDD082D050
:1012940083D5130875130F741E12130DAE16121294
:1012A400EC20320312F2E3A3303B22E58324F8500E
:1012B4001C0512E51224FC401F129EA4900400E0B9
:1012C40030E604D23C801190042275130FD5149D8E
:1012D4000516E51624C0508D12F251E51724F3F5D6
:1012E4001724EE4002D23D22C232ED04601624FCE3
:1012F400501224A350027D5FEDC423541FFFC3E5A5
:10130400179FFF22D23222740F2582F582E435839F
:10131400F583E022D22B121582D21412EE6912F355
:101324009E122AAB12E22C12165F1215587516047F
:10133400751500E530651360FA853013533203E503
:011344003276
:1013450070F012183B1218C10515E51524C4500696
:1013550075150012A08E301A03121922E53960099D
:101365001213C712139912F25175A6FF1000081037
:10137500011810020A80BB301AB8121631800920F4
:101385001AB0125F32121604808E121631C237C29D
:101395002B020552E51570030216857F0A147001AC
:1013A500221470077E24E53E02E8481470097E1376
:1013B50078AEE602E84822146001227E35E53F0258
:1013C500E848ED24E1400574769D801A24E2400E3C
:1013D500ED941E3375F00384FC74589C800804C397
:1013E50013FCC374449CFCAE167F7612F2E3EFB592
:1013F500040B1FEF24ED500812F31380F51F80EB4B
:10140500E516FE20E0147F2612F2E37F3512F2E3A3
:101415007F4412F2E37F5812F2E30516E51624C065
:1014250050037516042275A6FF758AFC758CFFE4BA
:10143500F532F539D205D23712EE6902F39EC22B89
:10144500C21412158212142B7F0090B61F1285B597
:101455007F3290B67C1285B57F3C90B6851285B5F6
:101465007F4890B6911285B57F527E1890B69A1234
:1014750085C77F6D90B6741285B57F7990B6A21237
:0814850085B512151712F25192
:10148D0010000B10013C10020280B2020552121A1C
:10149D0009AABE75BE001257AF12F211C203E55371
:1014AD0012150BE54412150B3003048ABE803CE582
:1014BD0053F404C454F0FAE544F404540F2AF5BE71
:1014CD008024121A09AABF75BF001257AF12F2116C
:1014DD00C203E54512150B3003048ABF800DE545A7
:1014ED00F404540FF5BF90B7A0800390B7E61257E0
:1014FD00AF7F641285B512F25112F206808B30E780
:10150D0002F40424F85002D203227F0D7E14745885
:10151D0012E9B2E55312153E7F177E14745912E984
:10152D00B2E54412153E7F217E14745A12E9B2E5DC
:10153D0045F833742B40107E1C12E9B2E830E702F7
:10154D00F4047E2202E84E742D80EC7F2474081280
:10155D00E96B7F33740612E96B7F42740412E96BF9
:10156D007F56740212E96B7F65740112E96B7F740B
:10157D00740002E96BD215C21AC21F125F32121625
:10158D000BE4029572C22BC21412158212142B1287
:10159D00A08E12E22C12165F1216D2122AAB7919F6
:1015AD007B1E123CFA79557B1E123CFA79917B1EFB
:1015BD00123CFA79CD7B13123CFA10002210012F48
:1015CD00100221301A11E53924F14008E5322403C7
:0215DD004005C7
:1015DF0080EF121922E532240250FA80AD12163133
:1015EF0080DF201ADC125F3212160480D4121631FB
:1015FF00C237020552201A57D21AD21F1219E1858B
:10160F00BC4C85BD4D85BE4EE54C700FE54D54036A
:10161F007009753910E4F5520295727401129E77B4
:10162F0080E6301A2AC21AC21F1219E1854CBC85F6
:10163F004DBD854EBE1257AFE4129572D214E54CD4
:10164F007008E54D540370028003121986C21422EC
:10165F007F0A7E007401205A02740312E9987E05F6
:10166F007458201A02742D12E9B27E0B7446202B87
:10167F0002742012E9B2C3E4954DFB740E954EFC33
:10168F004BF5177A46205A027A171262228C038D75
:10169F0004302B0CC3EC13CB13CBC313FCEB13FB9A
:1016AF0012643CC0E07F017E00EB12E8B97E0AD0E5
:1016BF00E012E998E517700A7F2F7E1090B1C012E3
:1016CF0085C7227F197E0590B61F1285C71217385E
:1016DF0075A7008552827583057E3F7C00E0B504B7
:1016EF00004001FC1582E582B4FF037582B3DEED85
:1016FF00EC230475F0038423FD249C50027D63EDDD
:0D170F0075F00A84C0F07F237E2512E9CD1D
:10171C000F0F7E2D742E12E9B21F1F7E32D0E012F5
:10172C00E9CD7F267E0590B62A0285FA7D057F3AA3
:10173C0012DE67EF240FFFDDF778087F387E01E8B3
:10174C0012E96DEF240FFF1818B8FEF17F3D02DE91
:10175C00C675A700F5827583057E3FE92B203D01F8
:10176C002B95324031E0FAC374769AFF1582E582EC
:10177C00B4FF037582B3E0FAC374769AFD1217A313
:10178C001582E582B4FF037582B3E0FAC374769ACE
:10179C00FD1217A3DEC522BE3F0122203D1712F217
:1017AC00E3C3ED9F70012240060F12F2E380E81FA5
:1017BC0012F2E380E212F313C3ED9F700122400694
:1017CC000F12F31380EF1F12F31380E912CBD31215
:1017DC0017F2FD7E001217F2FFFC1218018C050E99
:1017EC00BE40F2D2B222E4F5F7E4E5F704C313FAF3
:1017FC00C374769A2212F2E3C3ED9F700122400665
:10180C000F12F2E380EF1F12F2E380E9C3E56B9451
:0D181C00E8FCAB6A7A081262147D0078A522
:101829001263BDAE037F2590183602E9DE03052059
:1018390070F830B25A758001C2B275F72475F70095
:10184900E4E5F7F545F5F775F700E4E5F7F544F54F
:10185900F775F700E4E5F7F553D2B212EEFA75C75A
:101869000375C6FE75B901E5BEC4540F30E30244E1
:10187900F02553F553E5BE540F30E30244F02544F7
:10188900F544E5BF540F30E30244F02545F5451210
:10189900EF071218F402652775A7007583058552AD
:1018A90082EDC313F00552E552244C5003755200E2
:1018B900E532B4010375390075A7007583048539CC
:1018C900820539E53924F0500475391022EDF0E527
:1018D900822410F582E545F0E5822410F582E5447D
:1018E900F0E5822410F582E553F022E54530E70260
:1018F900F404F5F0A4AEF0FFE54430E702F404F592
:10190900F0A42FFFEE35F0FEE55330E702F404F5BD
:10191900F0A42FFFEE35F0FE22E53924F0407904DA
:10192900600122E54E24F2406F240C506BE54C70A7
:101939004CE54D54037046740830100104302B02F5
:101949004410205A024420301F04C21F444075A786
:01195900008D
:10195A009005CEF0A3783A7F0612DC917F0730100B
:10196A0010786A7F0312DC9178707F1012DC917F05
:10197A001A9005CE1219C77422129E7775A7009085
:10198A000400205A0F7582101219A57582201219A7
:10199A00A57582301219A575390022E54C240E402E
:1019AA00047D0F800F04FD74109DFCAF041219C74B
:1019BA00EC129E77AF051219C7ED029E77740612D4
:1019CA009DD77402129E61E0F5F7A3DFFAD2B20244
:1019DA009F8875C6F4803575C6F5803075C6F68061
:1019EA002B75C6F7802675C6F8802175C6F9801C46
:1019FA0075C6FA801775C6FB801275C6FC800D7510
:101A0A00C6FE800875C6FF800375C6FD75C70375D7
:101A1A00B9012274721F12E9AE0F02F2517F0A1243
:101A2A001A1D7E2A125F351219FAA8BF121A5B1004
:101A3A00001210010510021580F508E824E750ECA1
:101A4A00781880E818E830E7E3780080DF88BF80FC
:101A5A005F7F097E0590B867B80C0390B86112855C
:101A6A00C77E27E53D28240C75F01884E5F012E8B6
:101A7A00487E33743B12E9B27E35E53E12E84802ED
:101A8A00F2517F13121A1D120C2C121ABD100008E3
:101A9A0010010510021780F2105C07205D0BD25C62
:0B1AAA0080E8105DE5D25D80E1D25CB9
:101AB50080DD852BBC0202FD205C10205D1890B8EE
:101AC500BA7F127E231285C702F25190B8CE205DEF
:101AD500F090B8C180EB90B8C780E67F1C121A1D44
:101AE5001219F5A8BF121B171000081001111002DA
:101AF5001A80F2E824F250031880EA780D80E6E8AF
:101B050024E740030880DE781980DAE8F5BFF5435D
:101B150080A37F1B7E26E412E99FE82323B4640893
:101B25007E26740112E99FE47E2E12E84802F251E6
:101B35007F25121A1D121A04A8BCE8121B7012F296
:101B45005110000810010D10021F80EEE824E0502E
:101B5500E9188006E824CF40E108121A0488BC126F
:101B650057AFD21512EE6980D180157F247E3724B8
:101B7500E202E8B97F2EA20A120C17920A120C365D
:101B85000203007F371219E6E5BDA2E4120C171215
:101B950019E6E5BD92E49267F5BD0202FD7F367E4A
:101BA50000747212E9AE0F7E16743F12E9801219A5
:101BB500F0A8BD121C1B12F25110000810010510EF
:101BC500021080EFE824875004240A800224E8F8F4
:101BD50080E17F377E16742012E9807E2C743F12D7
:101BE500E980121C1B12F25110000810011410029A
:101BF5002080EF18B80904787880E7B878E478E7AA
:021C050080E07D
:101C070008B87904780A80D8B8E8D5787980D18877
:101C1700BD02088AE82487923DE8500224917F3666
:101C27007E30C313923B12E8B97E3CE4303B02742A
:101C37000512E9987E1A90B7AE303D0390B7B212FD
:101C470085C77F3C7E3A02F2E37F127E00747212F0
:101C5700E9AE0F7E20743F12E9801219DC85BE10B1
:101C670085BF11121CD710000810011110021B802C
:101C7700F21511E511B4FFEB75111780E60511E5B3
:101C87001124E850DE75110080D9121CD77F137E0E
:101C970020742012E9807E31743F12E98012F251DC
:101CA70010000810011110021B80DF1510E510B499
:101CB700FFD875100B80D30510E51024F450CB75B1
:101CC700100080C61219DC8511BF8510BE0208BE40
:101CD7007F127E24E51112E8487E30743A12E9B289
:101CE7007E35E51075F005A412E84802F2517F49E8
:101CF700121A1D121D2DF8121D3310000810010DA8
:101D070010021280F218B8FF02780480EA08B805BA
:101D170002780080E21219DC88BD1257AFB80003C1
:101D27000208C1021DBD1219DCE5BD227F487E05F0
:101D370090B7C81285C7E8601CB4040A7E0590B73F
:101D4700BD1285C7800C90B7D41285C77E38E812BC
:101D5700E99F02F25190B7CF7E291285C780F3120F
:021D67001D2D30
:101D6900601D640460197F5B121A1D120C2C121D70
:101D7900981219F510000B10010810020C80EF02DF
:101D890008C1105FE9D25F80E5852BBC0208BE124D
:101D99001D2D601F6404601B7F5A7E0590B7C81211
:101DA90085C77E2390B7D8305F0390B7DF1285C708
:101DB90012F25122121D2D70030208C17F527E11A9
:101DC900121A1D1219FAA8BC121DFD1219FA1000D7
:101DD9000810010810020880EF1880EC0880E91249
:101DE90019FA88BC1257AF121A04E875F005A4F560
:101DF900BD0208BE121D2D604BE875F03270040457
:101E090075F028A4ADF0FC305D11ACF0FB7A8A12B4
:101E19006222EB30E7050CBC00010DAE05AF047C76
:101E2900007D6412632DC005EF7F517E1A12E865AB
:101E39007E2C742C12E9B2D0E07E2F12E848124FA2
:101E49003712F251227F64121A1D1219FAA8BD1213
:101E59001E7F10000810010F10021680F218E824E6
:101E6900CD50EC783280E808E824CD50E278008043
:101E7900DE88BD0208BE7F63E823C2E012E40F7565
:101E8900F06484C0F07E2612E99F7E2C742C12E93E
:101E9900B2D0E080A47F13121A1D1219F0E5BCA27A
:101EA900E7923DC2E7F8E8121EE212F2511000086B
:031EB90010010D08
:101EBC0010021280EE18B800EA783280E608B833C7
:101ECC00E2780180DEE8A23D92E7F5BC79A1F70249
:101EDC001F937F6380027F12547F305C01237E2826
:101EEC0075F06484E5F075F00A84C0F012E9987E10
:101EFC002D742C12E9B2D0E07E2F12E9980F7E35AA
:101F0C0090B8D4305C0390B9300285FA7F64121A11
:101F1C001D1219FFA8BDE8121EDE12F251100008A6
:101F2C0010010D10021280EE18B8FFEA780F80E64F
:101F3C0008B810E2780080DE88BD0208507F52128B
:101F4C001A1D1219FAE5BE7F517E2C129320F5BE94
:101F5C0079A2F70202FD7F37121A1D1219F5A8BCDF
:101F6C005300037F367E32E812E99F12F2511000C3
:101F7C000810010710020780E718180880E2E5BC7A
:101F8C0054FC48F5BCF52B0208507F49121A1D125F
:101F9C001A04A8BE121FCD12F25110000810011124
:101FAC0010021A80EFE8240AF8242450E778DB802A
:101FBC00E3E824F6F8247F40DB788180D788BE8064
:101FCC00C6E8F424DC75F00A847F487E3B02E99F66
:101FDC007F52121A1D121A04A8BF12201412F251A9
:101FEC0010000810011110021A80EFE82408F824E0
:071FFC005750E778A880E3CD
:10200300E824F8F824A040DB786080D788BF021F5B
:1020130093E8F424A923C47F517E3B02E99F123B3A
:1020230002754A00D210C211D214D2757579147593
:10203300340012F39E7F007E0290B43F1285C79056
:102043004F607F087E2612E9DEE52B54030F7E39AD
:1020530012E99F1229F912E64612ABD612F2511079
:10206300000810011A10022480C520750405798028
:10207300BE1579E579B4FF05C27575790180B02085
:1020830075EB1579E57970A7D27580A3C210C214D8
:102093000208531219F5E5BE7F097E3A02E99F1241
:1020A30019FAA8BF121A5B120C2C121ABDA8BF1280
:1020B3001B17121A04E5BC121B707F2DA20A1221F2
:1020C300EA7F36A2671221EA1219FFE5BC7F3F7E41
:1020D3003212E8BFA8BE1203551219DCE5BC7F48D3
:1020E3007E3212E8BF1219FAE5BE7F517E2C02E957
:1020F3009F120C2C7F1BA20D1221EA7F24A20E1229
:1021030021EA1219F0E5BC121EE27F09E5BCA2E741
:102113001221EAA8BF1223121219FFE5BD121EDE17
:10212300E52B54037F367E3212E99F121A04A8BFAF
:10213300122014A8BE121FCD1219E6A8BC02235701
:10214300120C2C7F09A20F1221EA7F12A20812217E
:10215300EA1219E6E5BDA2E37F481221EAE5BDA232
:03216300E57F5ABB
:102166001221EA7F51A20C1221EA7F24A20B12212E
:10217600EA7F2DA2091221EA1219F0A8BD021C1B42
:102186001219DC85BE1085BF11121CD71219E6A8DC
:10219600BE120989A8BF1209C71209CF1219F5E59F
:1021A600BE7F3F7E3A12E99F1219E1A8BF12094F7E
:1021B6001219DCA8BD121D331219FAA8BC121DFD96
:1021C6001219F5121D981219FAA8BD121E7F1219BE
:1021D600E6E5BDA2E07F6C800B7F098055120C2CD2
:1021E6007F48A25E744E400274597E3A02E9B212EA
:1021F6000C2C7F097E347401205A02740312E99F65
:102206007F36802E128C7C7F731288CF128CCB7F08
:102216006C1288DE7F2D801A1219E6E5BDA2E77FD3
:10222600631221EA1219F5E5BE7F097E3A12E99F8B
:102236007F48122258B40104BF0901E4F51075F075
:1022460005A47E1E90B1D02582F582500205830238
:1022560085C71219E6E5BD035403C234C25330E103
:1022660003D2342230E002D25322121A1D1F122248
:102276003812F251E5101000191001061002028002
:10228600ED22045403B40104BF090104B4030AE4B3
:102296008007145403B403011423C5BD54F925BDA6
:1022A600F5BD1257AF80C7128496EBF516F5147F6D
:0D22B6006C1288DE12847A7F647E23E516A8
:1022C30012E91CC3E5169514F5167F731288CF7FA8
:1022D3002D0222387F2E121A1D1219F0A8BFE824EE
:1022E300FA5002780312231212F25110000810015F
:1022F3000D10021280E818B800E4780580E008B8F1
:1023030006DC780180D8799DE8F7F5BF0208507F95
:102313002D7E2C7420B80502742E12E9B27E32E8A9
:1023230002E99F7F5B121A1D1219E6A8BCE812236B
:102333005712F25110000810010D10021280EE180E
:10234300B800EA780380E608B804E2780180DE8802
:10235300BC0208507F5A7E2CE802E99FD268754878
:102363000A125F35D214123A05128DA5124155C2D5
:102373006B12023280F3D214751501128C3675B9C3
:1023830001E5BC20E71C128D6675A6FF128DB11204
:102393002A0412F2511286CF10000F50051287F74C
:1023A30080E70515E515242050D10205A61223C2A6
:1023B30002026D1223C20205E31223C20208C112F4
:1023C30023CE1219F58548BE0257AF1239F7123AD8
:1023D300111268ED12F39E90B276D24912A44D12F7
:1023E300A4061229B412F2511000141001051002B0
:1023F3001B80F50548E548640A7002F54880CF154F
:1024030048E54864FF700375480980C2854849124E
:102413003A11E55822125F351239F7854849C250FF
:0C242300E558B40F02D2501268ED803A68
:10242F00D22775480A123A051268ED12F39E12A3CD
:10243F006D90B77F20290390B78A122A7DC26A1246
:10244F004155106A0280E1C227128C0E854948124D
:10245F002824123A11D2291268ED12F39E90B18CF2
:10246F0012A44B20500E122A6712F25110001010B6
:10247F0001AE80F8122A0412F25110000280FB0202
:10248F0005E31239F7E55830E7137F1B90B7697EE4
:10249F00051285C712F25112F2090205E3123A1121
:1024AF001268ED85594912F39E1229EE90B78A12E0
:1024BF00A44B12A41012F25110000810010A1002BE
:1024CF000C80F512252980DB12253680D612F39E5B
:1024DF001229EE90B28612A44B12A41012A4141259
:1024EF00F25110000810010A10020C80F51225425B
:1024FF0080DB12255080D61227EA123A111268EDAE
:10250F0012F39E90B6D312A44B122A3312F251102B
:10251F00000510028880F80205E30559C3E55895B8
:10252F00595003755900221559E55964FF700385F9
:10253F005859220549D3E549149558400375490068
:10254F00221549E54964FF7005855849054922124E
:10255F0039F7E55830E7057F2402249B123A111210
:10256F0068ED12F39E90B29112A44B122A7212F2DE
:10257F005110000A10010280F812289380DE020524
:10258F00E31239F7E55830E7057F2D02249BC26B24
:10259F007559FF1268ED12F39E1229DEE55930E7E7
:0A25AF00031229F990B2A312A44B05
:1025B90012A42012F251E55820E706100008100174
:1025C9001110021B80F00559C3955950CF7559FF59
:1025D90080CA1559E55964FE70C285585980BDE510
:1025E9005920E711D26B75A700758307C4F582E0FE
:1025F900B2E7F080A7306B031228410205E31239D4
:10260900F7E55830E7057F3602249B123A11126824
:10261900ED12F39E90B2AE12A44B122A4E4009124B
:1026290028881228BD1226340205E31219FAE5BDDD
:1026390075F00584F5BCF5BDF5BEF5BF1207FD12B1
:1026490057AF05C6DFF9221239F7E55820E7087FA9
:102659005190B2B802249E12F39E90B79512A44BE2
:10266900122A0412F2511255CFD2AC10001FE558AC
:1026790030E7F8306DF512278A7E207F00501390DD
:10268900B7E61285FA12F25112F20980CAC2AC02F7
:1026990005E31B8B1390B1A91285FA12F251C26B93
:1026A9007B007514B812287D128D35128CE75025E0
:1026B900A814E824384004A60105140BC3E5139BAC
:1026C90050E678B81228BF306B03128A8C123A117F
:1026D9001268ED8082128C7CE51660E6D26B128D51
:1026E90092C003128C4DD003A91580C41239F7E5A5
:1026F9005830E7057F5A02249B123A111268ED12ED
:10270900F39E90B2C312A44B122A2812F251100060
:102719003510010280F875460512275250157F00C1
:102729007E357407954612E91C12F25112F209D549
:1027390046E7D390B7A0500390B7E612A44B12F224
:102749005112F20980B30205E31255CF12F0AA74AF
:102759005212F0BB745412F06BE55804755900120B
:10276900F09912867E4016128C0E128D661286CF53
:10277900400B0559C3E558955950ECC322C2ACD357
:10278900221255CFD2AC12F0E3204CF1B440F7122B
:10279900F0E8B4400312F0E8B452E2F53812F0E878
:1027A900B454DA12F0E8FA60D424EF40D012F0E819
:1027B900E53870C912F0E812F0E81286637B007EF2
:1027C9000312875A50102050B412F0E8204C03B479
:1027D90040F7DEED80A7128D450B128663DAE0C360
:1027E900221228CAE55924C8F88602E54924C8F9FD
:1027F900986013146010500F18E608F618E869700D
:10280900F7A7021228BD22E559640F60F91908E6F5
:1028190018F608E86970F7A70280E81228CA78C88C
:10282900C250E6B4FF02800708B8D8F6D25022B8E1
:10283900D702D250A615807C78B81228CCE4F9F5D5
:10284900A7758307E9C4F582E030E70AE924B8F8F7
:062859002438400276FF66
:10285F0009C3E5589950E712288878B879C8E6B4C3
:10286F00FF028002F70908E8243850F2804079B857
:10287F0077FF09E9243850F82279C877FF09E9244E
:10288F002850F8221228CAC23D78D7B6FF04A900F3
:10289F00D23D18B8C7F5203D0279D81978C8B6FFD0
:1028AF000122C3E8995007C6C7C6081980F478C833
:1028BF001228D77F0412859ADFFB2278C81228D7F7
:1028CF007F04128D80DFFB2275C703E54875F00486
:1028DF00A42480F5C62212F39EC23C1285B9E537B7
:1028EF00605814605214604A14604214603A1460C5
:1028FF003214602A14600E146010146012146019E0
:10290F0014601180351221E380301221F5802B12D3
:10291F0022AD802612218680211221DF801C1222F7
:10292F001E801712220A8012122143800D1220F4EA
:10293F0080081220A2800312209612F25112F20D7B
:10294F001229DE12C8B1A81F08E814C23BB51D0238
:10295F00D23B75F007203C0375F009A4FF7E0030D1
:10296F003C0C7420303B02743E12E980800A740BD9
:05297F00303B02740A68
:1029840012E998D8CF12F251E51D10000810011079
:1029940010021880B9651F7003751DFF051D80AEF8
:1029A4007005851F1D80A7151D80A375F003A42243
:1029B4007F7B7E0090B6EB1285FAE54824F640084A
:1029C4007E0A90B74C1285FA221288FB7E05745B4E
:1029D40012E97C7E1D745C02E97C1229CD7E349060
:1029E400B6FC0285FA1288FB80031229CD7E319051
:1029F400B7000285FA1229CD7E3190B7F10285FA2B
:102A04001288FB7E00800C1288FB7E1880051288D9
:102A1400FB7E2D90B7F10285FA122A287E3190B1FF
:102A2400E40285FA122A047E1A90B1E90285FA12A8
:102A34002A0480B9122A047E1890B1960285FA12EB
:102A44002A047E1A90B7F60285FA122A047E1A9096
:102A5400B7FB1285FA12F251D3100006C31001021B
:102A640080F622122A047E1A90B2800285FA122A73
:102A7400047E1890B29C0285FA7F007E201285FAAB
:102A840002F2511288FB90B8000285F81288FB907C
:102A9400B8110285F81288FB90B5E00285F8128817
:102AA400FB90B5F10285F8122A0B7E2C90B61930F2
:102AB4001A057E0090B6130285FA1288FB90B6AE12
:102AC4000285F812641F0FBF00010E8E04EF799A7D
:102AD400F7FB7F017E28A25C924EC25C12E7B2A291
:102AE4004E925C78B8E654F070091F7E2890B5DBEE
:102AF4001285C7E4FFFE78ADE612E8B37E0A742CB3
:102B040012E9B27E0C18E612E8B37E16742C12E9B0
:102B1400B27E1818E612E8B3303D0A90B5D57F149A
:102B24007E011285FA227F097E0178AEE612E8481A
:102B34007E0D743A12E9B27E1278BDE612E8487F3F
:102B4400097E2378BEE612E84E7E30743A12E9B26A
:102B54007E3508E612E8480886040886037F127E5C
:102B64000012E77912E7FD78C4E612E40F7E291219
:102B7400E8657E3B748B305D010402E9B2780C7F1A
:102B84001C7E02E812E9007E09742E12E9807E0C94
:102B9400E51012E900EF2405FF7E1E12F2E30EBEDB
:102BA4003FF9EF2403FFD8D922C3740C951375F0B1
:102BB40008A4241CFF7E17742012E980C3740C95AA
:102BC4001175F008A4241CFF7E17743F02E9807578
:102BD4001600AD6FAC6EAB6D7403129DE2E4F5F7B5
:102BE400A4E5F7F9540F6046E4F5F7A4E5F765109A
:102BF400703CE4F5F7A4E5F775F008A47F80CF9F57
:102C0400FFE4F5F7A4E5F7D2B2241DFE12F2E3E9DE
:102C140054F0601A1F12F2E3EE6516700DEF65179B
:102C240070081F12F2E31F12F2E38E168F17D2B24E
:102C3400129E00ED30E7A122AD6FAC6EAB6D740354
:102C4400129DE2E4F5F7A4E5F7540F601DE4F5F7EF
:102C5400A4E5F765107013E4F5F7A4E5F7651170C2
:102C640009D2B28D6F8C6E8B6D22D2B2129E00EDA2
:102C740030E7CBD32278B97998E6F70809E6F7224A
:102C8400D215C210C21112F39E129F17303C13903A
:102C9400B0797F1C7E051285FA12F25112F20602F7
:102CA400026DC221C24D129E41E56F20E7E1129FE1
:102CB4005579B8E7540F60EEE764FF60D279B987BD
:102CC4001009871130210979988710098711800A22
:102CD40012F39E122B2AC23D800512F39ED23D129E
:102CE4002AC71229DE122B8112F251122BD385111D
:102CF40013122BAD85111312F2517998A71009A75D
:102D040011E59030E20FC221304D24C24D12F20D74
:102D140012F247801AE53524AA500302026AE53507
:102D240024C3500B90B5C87F731285B512F251209D
:102D340021C810000810011C10023780BDE51114D1
:0B2D4400F51170AD75110C1510E510B5
:102D4F00B40700508A051080A679B9E765107006A0
:102D5F0009E765116099E51104F511640D70877528
:102D6F0011010510022CDE122C3C501DC3740C9562
:102D7F001175F008A4241BFF7E0290B5BE1285C703
:102D8F0012F25112F20D022CDE129F55122C79E520
:102D9F009020E210E53524DC500AD221D24D129F4B
:102DAF0017022CAA12F39E122A99122AC779B8E792
:102DBF0054036003122B2A12DC4A79B8E764C370FC
:102DCF001712DC4A1233CE12DC5A1234B3756A1062
:102DDF00129CFCD23312367312F2511000171001ED
:102DEF003279B8E764C370A410020280EEE535248F
:102DFF00FA4099807C129E41129F55E56F20E70A99
:102E0F0079B8E7540F60EEB7FF82129E23129F55D9
:102E1F00022D9B129E23129F5579B8E7540F60F332
:102E2F00B7FFED80D0122A4E40517FC0129F731210
:102E3F009DF3129F9D60F8B4FFBB78C6866C088621
:102E4F006B756A0012CBCB129CFC121A13E56C65E2
:102E5F00BD701BE56B65BC7015E57064FC700F7879
:102E6F00BEE66577700808E6657870028049022D26
:102E7F009B7995A76F09A76E09A76D7995876F093C
:0E2E8F00876E09876D129F5512DC4A12DC5ABD
:102E9D001234B3756A10129CFCC23312356A90B0AD
:102EAD008FD23C1285B912294F902EBA73022D9BE9
:102EBD0002409E022F3E022E347F6C1285AC12F220
:102ECD0009129E41E56F30E70F1285331257AF128D
:102EDD00588D12586F022C84129F55129E23121A70
:102EED0013ACBFADBE85BDBF85BCBE78C686BD0863
:102EFD0086BC1257AF12CBCBE56C6C700DE56B6DCC
:102F0D00700812CBC112CB54801F12CB86E56B54C7
:102F1D00036403700612CBC112CB54129C4BE56BAC
:102F2D005403700312CBCB80CF7F00129F73022D01
:102F3D009B12F39E7F6490B9C91285B57F7990B9C4
:102F4D00D61285B512F25175160010000A1001093E
:102F5D0010020280F505160516C25312DC5A75379C
:102F6D000A90B0A91228E5902F7873022E8A022FAD
:102F7D009F023172023177022F3E022FA6022FAB34
:102F8D00022F3E022FE9022FED022FF1022FF80240
:102F9D002FFC7F0A12227080981255EB8003125578
:102FAD00E0780A1230CB740C12F06912311312F062
:102FBD009212314C129CFC129D59129C3112A08E12
:102FCD0012325BD5150C75150A12315C1233801255
:102FDD00F092100204E57F70DB022E8A780A8006DB
:102FED007804800278011255EB8009780A80027806
:102FFD00011255E01230CB740C12F05E123113E554
:10300D004812F04AE5165403443012F06B742A123C
:05301D00F06B12F06BE6
:1030220012F09212314C129CFC129D59129C3112D8
:10303200A08E12325BD5154885481512315CE51C0D
:1030420012F04AE51B12F04AE51B2548F51BE43550
:103052001CF51CE4A27792E7A27492E0A27392E1BB
:1030620012F04AAD75AC74AB73E57DC412308CAD11
:1030720078AC77AB76E57D12308C12339E12F092EB
:10308200100204E57F709F022E8A540F2375F0050B
:1030920084F8C3EB33FBEC33FCED33FDC3EB33FBC2
:1030A200EC33FCED33FD20E713EB28FBE43CFCE4BE
:1030B2003D12F04AEC12F04AEB02F04AC3EB98FBE5
:1030C200EC9400FCED940080E88848122A1290B536
:1030D200B81285F812F251E4F54AF549756A20757D
:1030E2001501129CFC129C31D5150E854815E54937
:1030F2002401F549E4354AF54AE57F70E57440124A
:10310200F0BB747812F06B746312F06B742302F0EC
:103112005E12335B799AE712F04A12DC5AE53A12F0
:10312200F05EE53B12F05EE53C12F05EE53D12F02A
:103132005EE53E12F05EE53F12F05E740112F04A67
:10314200E54A12F04AE54902F04A12DC55E4F51C60
:10315200F51BF514F51375150122753800E51412E7
:10316200F04AE51312F04A0513E513700205142222
:103172001255EB80031255D5122A121232B512F2F1
:1031820011756A2075150175A6FF754A01129CA07A
:10319200129C3112A08E12325BD5150975151E12C2
:1031A200327F12F21B123380E57912F04AE412F0F8
:1031B2004AE57112324012F04AE57012F04AE57B9C
:1031C20024ACFFE55F340912F050EF12F04AE51526
:1031D20020E036857D56E412F04AE52EC412F05006
:1031E20012F0A112F21B10020630559B1231F402AA
:1031F2002E8A744012F06B744512F06B744F12F009
:103202006B744612F06B02F0A1E55612321AC4FA40
:10321200E57D12321A2A80BFFBC41232272323CB48
:103222001232272B22540FFC24F650027C009032DB
:1032320036EC932200000101010202030303FA2487
:1032420040400A24804003EA3322D2E72274FF225C
:1032520020E703C3132224C022E53F701F7F7B7E39
:103262000078AEE612E906EE2404FE743A12E98012
:10327200EE2404FEE53E12E90012F25122C015C00E
:1032820016D21212941AC212D016D01578AEE612C5
:09329200F05EE53E12F05EE53F3E
:10329B0012F05EE54512F04AE55212F04A740A123A
:1032AB00F04A74C012F04A02F0A1744012F06B7431
:1032BB005412F0BB744E12F06B743012F06BE516B7
:1032CB005403443012F06B12335B742312F05EE53F
:1032DB003D12F05E799AE712F04A12DC5A78ABE6AF
:1032EB000812F05EE60812F05EE60812F05EE612D7
:1032FB00F05EE53E12F05E123861E51212F05EE50B
:10330B001112F05E740112F04A90B8221233C0759C
:10331B006A10129CFC740212F04AE412F04A787B99
:10332B0012F043787D12F043787712F043E4FEFFFE
:10333B00780712F04312F043E57412F04AE5751268
:10334B00F04AE412F04AE412F04A12F04302F0A100
:10335B0075C70375C6FF75B901C217751D0085BC0E
:10336B001C85BD1B85BE1A85BF1912619AEE12F022
:10337B004AEF02F04AE57512F04AE57412F04AE59D
:10338B007312F04AE57812F04AE57712F04AE576C7
:10339B0012F04AE51664016011E55E12F04AE57A17
:1033AB0012F04AE516640260012278BCE612F04A7C
:1033BB0008E602F04A75A700E493700122A312F00D
:1033CB006B80F512DC5A857946787A796412DC7653
:1033DB0074641265958E471234B3756A20D23D1210
:1033EB009CFC129D591234EA303D09307406C23DE3
:1033FB008E1E8F1FE57F602BE54C24FFF54CE54DB2
:10340B0034FFF54D454C6005129C5280D2751D3C26
:10341B00129CFC129D59129C311234EAE57F600319
:10342B00D51DED12354B90356312E9DE203D0DAE07
:10343B001EAF1F12354B90355C12E9DEE546FD7071
:10344B000B90B958305D1190B954800C04700E90EC
:10345B00B954305D0390B9507F38024F32E4FFFC12
:10346B007E05305D047E027FB3126320AC06AB0792
:10347B001261EA7F38C23DE51C6007D23D7E2C12FB
:10348B00E96DE51B203D026007D23D7E3012E96DF0
:10349B00E51A203D026007D23D7E3412E96DE51935
:1034AB007E3812E96D024F37E54075F03CA425419B
:1034BB00FFF54CE435F0FEF54D7C007D1012632DCD
:1034CB000F8F4BAF4CAE4D7C007D3C1262007C00ED
:1034DB00AD4B12632DEE4F70010F8F4C8E4D22783A
:1034EB00647973C2D1123501FF78677976D2D11224
:1034FB003501FE02F2E3C3E796FB0809E796FC08E9
:10350B0009E796FDA2E7921750031264B575135A9B
:10351B0030D10E751320B217AA47126234AB04AC2C
:08352B0005E546600B04600B8E
:10353300AA4612624BEB03FBEB03FBEB543FFBE5A9
:10354300132B2017029B9B22EE141430E701E4FE99
:10355300EF141430E701E4FF2205057088A8887092
:1035630005052020F8202012F39E7E1E7F1C12F2F8
:10357300E3DFFB12F2E37E1E7F1C12F2E3DEFB7E2F
:103583001D7F1D12F2E3DEFB7F007E2178ADE61284
:10359300E9007E29742E12E9807E2D18E612E900D7
:1035A3007E35742E12E9807E3918E612E9007F0712
:1035B3007E21745412E9807E25744F12E9807E2D9A
:1035C30078AEE612E9007E35743A12E9807E39E579
:1035D3003E12E90078AE1238617F0E7E21744C12E0
:1035E300E9807E25744112E9807E2DE51212E900FF
:1035F3007E35743A12E9807E39E51112E9007F15B0
:103603007E25744412E9807E2DE54012E9067E355D
:10361300743A12E9807E39E54112E9007F217E0187
:1036230090B9231285FA7E0EAC77AB7612E7B27EA1
:103633002B85795F85787B12ED5D7F287E0190B9BC
:10364300271285FA751D2B751E10E5741238157E29
:1036530025742F12E980751D2D751E2BE575123803
:10366300157F367E0290B9131285FAE5721237FF81
:103673001237432033031237F012DC55AE4DAF4CF3
:103683007C007D4012632DBF00010F0FAC07AD0717
:10369300E4FED23D129CFC129D591236E3E57F6095
:1036A3002CE54C24FFF54CE54D34FFF54D454C60BE
:1036B30005129C5280DE751D3C0E129CFC129D5916
:1036C3001236E8E57F6006129C31D51DED7F783018
:1036D30033027F3612DE671F1F7E00743002E980DB
:1036E300DD03AD040E7F783033027F36E55E20E7DD
:1036F3002EE57A8549F0A4A9F0E57A854AF0A42954
:10370300F9E435F0FAE55E8549F0A429E435F02AB9
:10371300FAE55E854AF0A42A30330113CF9FFF12E6
:10372300F2E3103D18C3EF9B50131BEF6B600E8F3A
:10373300018B0712F2E31FEF6970F8AF01AB0722A9
:1037430090B8D8305C0390B8F1754A40754900AF22
:1037530076E577FE20E76B7005EF24105064EF24C5
:10376300A8EE34FD401190B8DD305C0390B8F575D8
:103773004A1975499A8075EF2450EE34FB40119035
:10378300B8E2305C0390B8FA754A0C7549CD805C99
:10379300EF24A0EE34F6401190B8E5305C0390B806
:0D37A300FF754A067549668043EF24F0EE7D
:1037B00034F1401390B8E8305C0390B904754A04C2
:1037C000754944802A8028EF2490EE34E840119017
:1037D000B8EB305C0390B909754A0275498F800FC8
:1037E00090B8EE305C0390B90E754A0175499A2283
:1037F0007F401285F87F4612DE677F5F02DE677EBC
:103800002112E40F12E91C7E2F90B92B305D03903A
:10381000B9300285FAAE1E75F064305C0375F03283
:1038200084C0F0F87004EE2404FEE51D12E980EE79
:103830002404FEE8600712E96DEE2404FED0E07572
:10384000F00A305C0375F00584A8F012E96DEE24EF
:1038500004FE742C12E9800E0EE8305C012302E9AC
:103860006DE53E2541F51124C45003F511D3E6352D
:1038700040F51224E85002F5122212C8ABC2101211
:10388000F39E7F057E0990AEAE1285C77F137E063C
:103890009038B412E9DE7F2B7E0190391C12E9DEEC
:1038A0007F1C7E3390398E12E9DE7F1B7E3C90397F
:1038B0009F02E9DE113007FE1FE001E101F80F0071
:1038C000061B00F80C00180E007C10007006003C6F
:1038D0002000E006003E4001E004001E8003C0041A
:1038E000001F0003C070000F00078060000F8007FA
:1038F00080500017800F00080027C00F0000004311
:10390000C00F00000083E00F00200301F00700C09B
:103910000F01F80383007F87FE01FC000E3E1800B4
:103920000003000000001800000300000000380041
:103930000000000000003000000000000000FC76E5
:103940001F0E1C6030ECFCBC3F172DF0F97861387D
:1039500066264F619A706070C60E1EE330E06060AC
:10396000C60C1CC360C0E0618C0C18C7C0C0C0E1AD
:103970008C1C39C611C0C4C19C9931963180C8C114
:10398000FF1E31E7E180F0C0EE1C31C381800F08DB
:10399000082653C3A599523C180010105C38100437
:1039A000047030508012F39E7F3E7E1790B736121F
:1039B00085C712F251C2AFD2C075C0107581D874DC
:1039C000FE1239D012F20DE4F5F9F5FBC2B480F71E
:1039D000D2A6C2A512C89012F20D02C8B175C703D3
:1039E000E54875F004A42480F5C6C23C75B901E52C
:0239F000BC0415
:1039F2007002D23C221219F5E5BEF54824F65003B6
:103A0200754800753400753704C228D229D22A7548
:103A1200C703E54824E75003754800E54875F004FC
:103A2200A42480F5C6751607751700C23C123A52D7
:103A3200123A52123A52123A52851758155875597B
:103A420000E548B40A09E5586005F4600205592208
:103A5200203C1D75B90105C6AABCABBDACBEADBF4D
:103A6200EA123A73EB123A73EC123A73ED123A73AA
:103A720022203C07F515B4FF03D23C22C0C7C0C6C2
:103A8200128C3675A704851683E517C4F8F582757E
:103A9200B90105C6E5BCF0C582F82406F92403C5C0
:103AA20082E5BDF0E5BEF0E5BFF075B90105C6E5FA
:103AB200BCF0E5BDF0E5BFF08516838982E4F075C0
:103AC200B90105C685BC1385BD14E4F0F08882E512
:103AD200BEF0E5BFF075B901E5BCF0E5BDF0E5BEAD
:103AE200F0E5BFF0758306E51723541E24B0F58276
:103AF200E513F0E514F075A700D0C6D0C70517226C
:103B020012CABB78BEA64808E4F6F559087618082A
:063B1200F6D23608760A27
:103B180008F6060876BEC237C22BC21AC21FC254A4
:103B2800C255129FC0123A05C229C22AC207C2272B
:103B3800C2681219E6E5BDA2E59243C24AE4F52E31
:103B4800F534F536F52F78B6F678B5F678A9F6781F
:103B58009EF678B8A65E08A67A12E71BC26BC23337
:103B6800C238C240C223C222123B8A75460278C5B7
:103B7800A646C23AD221C219C226E4F542F541F559
:103B88004022E45407205E09B40400400274038014
:103B98001B1219EBC313A9BC600C14A9BD60071450
:103BA800A9BE6002A9BFE94001C45407F537221233
:103BB80039F71268ED1207F412F39E122A33E5580A
:103BC80004700A7F327E0590B7691285C790B9C024
:103BD80012A44D12074E7F7290B9B51285B512F234
:103BE8005110000510020480F8D322C322020105F7
:103BF8001219E6E5BD20E705123BB740F0123B027B
:103C080012A228754403125F3212CDD9D54403029B
:103C180039A5201EF1789F7680754A00129C02D241
:103C280010C211C213C2121255BF75A60C12EE694A
:103C380012D8F2E5A624FA4006125ED275A60C2028
:103C4800250CE59054057009E53524E25003023D42
:013C58005714
:103C5900E5322418400D75F00C84E5F070D412415A
:103C69005880CFD21ED2AC306DC87532F012F0ED4B
:103C7900B4E0BF74E0125F7AE53124F392052012B3
:103C890003124001123D1320371EC01412AB1CD081
:103C990014200A0312CBFD1241581293E91241581C
:103CA90012A22B124158803779247B11123CFA1247
:103CB900F39E12EBE712E41D12E77112E5BA121630
:103CC900D212165F122AAB79607B1D123CFA799BDE
:103CD9007B1D123CFA79D67B0E123CFA1241583000
:103CE900120C301A09E532241650F4121922023C3A
:103CF9002FD3E9953250FAE556D23D12175DE552B8
:103D0900F556C23D12175D02F251301238E54024D2
:103D1900F040267A0AC3E53F954B601D402824E20E
:103D29004017305405C254757F01E54B0475F03CCA
:103D39008485F04B129C11DADC79BCE7D2E7F57F78
:103D490009877EC27722F40424E250ED80D412F36D
:103D59009E7F2A7E0E90B8261285C775A6FFC210CF
:103D69001012137F367E0890B1C71285C712F2511F
:103D790012F206020105D221125F35129C117F1E33
:103D89007E0B90B7441285C712F251123DAA7F3EAD
:103D99007E0790B3561285C712F25112F20002390A
:103DA900B5121631C237D215D214120C2C75B905B9
:083DB90075B902129D8AD25572
:103DC100129C7E7D0012CB79129D94E56A600512EA
:103DD1009C3180F7121A1385BEBC85BFBD856BBEB1
:103DE100856CBF75B90575B90285BD6C85BC6B75F0
:103DF1006A20129D8A123E7B857A62129D94756AB1
:103E010000129CFC7570FC854077854178851F798F
:103E11007818797A12DC7612CBCB129C2912F21B1C
:103E210079B877C309A77109A77209A77309A7749C
:103E310009A77509A77709A778129D94756A1012C9
:103E41009CFC7F087810797212DC7885627C855E33
:103E51007D79C0A71509A71409A77409A77509A732
:103E61007209A77309A76C09A76B129F1712641F28
:103E71008E7E8F7F129F3E029C2978107F0EE4F682
:103E810008DFFCF564F565F567F5687515FC751ACD
:103E9100C0751DC0756640756940754A01129CA0C8
:103EA100305503023F31129C31E571B510004002DB
:103EB100F510E4F511E512207502E513C39579506B
:103EC10006207545857913D3E57A9514E515648047
:103ED100FFE55E64809F400C857A14855E15857BC5
:103EE10016855F173074B3C2D178647973123F0FAE
:103EF10078677976123F0FD2D178187973123F0F14
:103F0100781B7976123F0F809185791280B9D3E7BA
:013F11009619
:103F12000809E7960809E66480FFE764809F20D1DC
:103F220001B3400AE7F61819E7F61819E7F622E591
:103F32001AB4C00E7873791812DC76787379641229
:103F4200DC7678187964C2D1123FA2741812659592
:103F52008E47AE1EAF1F781B7967D2D1123FA2C324
:103F6200E51F9FE51E9E50048E1E8F1F7EFF7FFF62
:103F7200AC1EAD1F12632D7A04EF8AF0A4E5F0CED9
:103F82008AF0A42EFEE435F0BEFF011E6005146027
:103F9200057EFF8E1F22EE7E0020E7F77EFE80F375
:103FA200C3E697FB0809E697FC0809E697FD18188F
:103FB200191930E7031264B5C3EB33FBEC33FCEDA4
:103FC20033FDEB33EC33FBED33FC30D105AA471262
:103FD200624B0BBB00010C751E03751FFFEC24FC2A
:103FE20040048C1E8B1FE627FB0809E637FC0809F4
:053FF200E637A2E71311
:103FF700F618EC13F618EB13F62210131978B5E63A
:1040070024FA401AE57124F64008E57924F64002BF
:1040170080310606802D12F217E59030E2DF753603
:1040270012D22EE4F534F55A129FF212404DC219FE
:10403700123B8A12AE4B12AE78D212853F4B205EEE
:1040470002D228023B82D214124093E6F008DFFB2B
:10405700857A621240897570FE783A797112DC763A
:10406700129C2E12408985627A855E7B7570C0121C
:104077009C2E124093E0F608DFFB75A700D254C2CE
:10408700142274FF7870F608B880FB2275A7049095
:1040970004F078707F102212F39E12F251C258C2B8
:1040A70059123B02753901754A0112DC55129CA061
:1040B7001265938E47C210D211D214D212129FF2F8
:1040C70012AE4B12AE7812EE6975A6FF75360975FA
:1040D7003200E59020E206E5352405400CE59054D2
:1040E700057019E53524E25013C211C21212F39E6E
:1040F70012F25112F20912F247022E8AC221E54A40
:10410700B40202D221129CA01293E930260F126941
:104117004F12A22B753606E53670FCC22612A2286E
:10412700124158E54A20E021B40209753900E53605
:0F41370070F98092E53960FAFD24E24002053903
:10414600129CA02026C9DDF880E975390080E47547
:10415600370410003A100116100216E52F540760B6
:104166000312C8A520784C20790A207A1F22024320
:104176006A0242B1E5376009146009146009024415
:10418600160243890243E7C27902444C0242E42004
:10419600110C303709121631753400C27822E53712
:1041A60024FC500FE537640760030244C2024486CC
:1041B60002427B2011FAE59020E202805675340017
:1041C600201203D2132278A9E67017C226767DE55F
:1041D600377005106B02D26BD277753614D22E0269
:1041E6009FE7E5376043146040B40227200B24E6BE
:1041F600249B401F2414501C12AE4B90B7177F20EF
:104206007E081285C712F251753608D22E78A9E6B5
:1042160024ECF622241940FB241450F712AE4B125C
:10422600AE7890B7207F2980D72028E7E54824F686
:1042360040E1E5580460DC7F5D7E10E6249B40D3B8
:1042460024145015C2330559C3E5589559500585B0
:104256005859D22690B70580A9241940B62414507F
:10426600B2E55960021559102606E559600215593E
:1042760090B70E808D10780122753900E534243808
:104286004007754A0175340022700AE54A30E0F2AB
:10429600754A0280F0146008754A0612AE788006E8
:1042A600754A0412AE4B75390180DA302909C229E4
:1042B600D22A7559008005302A1BD22912A3FC1276
:1042C600A3CAE53524AF400475340022753700C211
:1042D60029C22A80F320684E302703D26A22201191
:1042E6000A303707121604C27A8015D22212465EA9
:1042F60012F251107A0122E53424384007123B8A23
:1043060075340022700FAA37123B8A6A70F2740164
:10431600123B8B80EB04123B8B24FC50E3E537B455
:104326000706D22880DA8036C228E53724FC232403
:10433600BEF879C4E7F9A74809A75979C4E8F7860A
:1043460048088607E537B40505754818D236123A87
:10435600118F59E53764067002D2070243061246EA
:104366003A0245E4E537601B14607614600F14606A
:1043760009E53724F9400902453C02441602447512
:10438600024509D223124E1E10790122E534243843
:1043960040077546017534002278D87020304A0BE4
:1043A600C24AE624F85004B243800AD24A7614E59B
:1043B6004624FE40DDE54660D9154680D8B600D5D0
:1043C600B40500500C04F54624FA50C9754605801C
:0343D600C424F903
:1043D9005005128A2A80BB100FB8D20F80B4D2239D
:1043E900E53464C86003124E1E10790122E53424B5
:1043F9003750097011105B4BD25B8047100802D20D
:1044090008124E1E803D100C3AD20C8036D223126F
:104419004E1E10790122D24BE53424374011301257
:104429002210371FD237201A1AE4129572801424E9
:10443900FC402824047010C258C259201105D22EFC
:1044490075360775340022D258C25914700280F3A8
:10445900C258D2591460ECD25880E81219F0E5BC60
:10446900B2E7F5BC79A1F71257AF80D778B8A65E45
:1044790008A67A2011CD753605D22E80C630122BAA
:1044890012A436055BE55B75F00B84E5F0F55BE599
:104499005A24F64009E55A955B5003755B0012A44E
:1044A9003A12F251E5346003D534D275340022D280
:1044B90029D22A75480A0245AAC2401007F13029B3
:1044C900030245AA12A3F812A40C102A1BC2330531
:1044D90059C3E558955920E7025008755900E54830
:1044E900B41816E558B4FF0375590012A42012F246
:1044F90051E5346003D534C122D22A12A3FC80EEDF
:1045090030122312A436155BE55B30E70C755B0AA4
:10451900E55A24F64003855A5B12A43A12F251E592
:06452900346003D534DA12
:10452F0075340022D229D22A754817804CC2401008
:10453F0007F220294412A3F812A40C102A22C23326
:10454F001559E55930E71C855859E558B4FF0375DF
:10455F005900E548B41802800AD22A12A3FC800E33
:10456F00855859E558B4FF0375590012A42012F26B
:10457F0051E5346003D534B52220106220115F7FDE
:10458F00180548E54864187008F548302703754842
:10459F000A1239DD303C2DDFE8802620105A201119
:1045AF00577F181548E54830E705754817800A64A6
:1045BF000970063027037548171239DD303C05DFC7
:1045CF00E275480A123A111268EDE532244C500593
:1045DF0012A3CA800312A36D75340002F251124662
:1045EF00217F15E5486B70048A488002054812390F
:1045FF00DD303CD0DFED80CC1246217F15E5486AD7
:10460F0070048B48800215481239DD303CB6DFED5F
:10461F0080B27A007B09E537B40401227A0A7B174E
:10462F00B40601227418FAFBF5482275A7047583A6
:10463F0007E559C4F582E0E0F573E0F574E0F57530
:10464F00E0F576E0F577E0F57875A7000268EDE51F
:10465F009020E23EE534243750381246A212467FAE
:10466F00205E4F7F2C90AF661246E990AF6F806A45
:07467F00E534243775F00952
:10468600A42435FF205E0624BE50027F3EEF249B05
:1046960050027F627E32748912E9B22275A70490B5
:1046A60000317E087F3AE4F0DFFDE5822446F5829C
:1046B600E43583F583DEED75A700227F2C1219EB16
:1046C600E5BD1246D2E5BE1246D2E5BFF8C4124693
:1046D600D8E8540775F009A490AF542582F58250A6
:0A46E600020583EF2409FF0285B5E9
:10A2250002A2E212F39EE53724FC40F4B4FE1420AA
:10A23500110EE590F45407600122E532247450EFC5
:10A2450002AB2812F39E12EB5512EBE712E41D1236
:10A25500E77112E5BA7E197F3612E55712F1301211
:10A26500E56DC206E53760051460338053C23A12C6
:10A27500A386124ED912506E1253541273B912732B
:10A28500E1124B8CE54864186009E54824F6500353
:10A2950012543F12AABE12E2A0124F748014D23A91
:10A2A50012A3AC1246F8124F4312DDCD12AABE120C
:10A2B500E261126C2E12EC2E1266FF1269FE8012FC
:10A2C50012A39212DD0A12ED0012DD9C12AABE1233
:10A2D500E27830101412E4E012E4AF800C12F39E21
:10A2E500E53724F9401E12A36F30220912465EE5B8
:10A2F500347002C222302309124E1EE5347002C2A8
:10A305002302F2511229DE75170012EF147F121283
:10A31500DE5530124A75100075A70475830612695B
:10A32500A8E51075F009A42415FFF5177E00E512C0
:10A33500602F75F06484E5F00F12E9001F7E0EE5CD
:10A345001112E465751623126B640510C3E55A9561
:10A35500104006E51024F550BF30120312A43A80D0
:10A3650088745D12E9B280D5C2493029051229B435
:10A3750080031229DE90B18C12A44D202A7902A403
:10A3850020301223305E2030501D02A734301217C2
:03A39500305E0631
:10A39800200B1102AD9512DE4E7F17120031751792
:10A3A8002002EF1412EACC12EA6D201A14301211AE
:10A3B80020510512EB2C800612E19E12DF7E125D01
:10A3C8009422E4FEFFE54824F6400D90B74C128530
:10A3D800FA7E16E54802E96DB40E0690B75202857A
:10A3E800FA90B7591285FA7E12E54824F702E90671
:10A3F8007D20800C7D3F302A077D633029027D3C1B
:10A408007F0080247D2080127D3E800E7D3CE549C2
:10A4180075F007A42406800A7D3FE55975F007A466
:10A428002409FF64027001FF7E1CED02E9807D2093
:10A4380080027D3FE55B75F009A42416FF7E09EDD7
:10A4480002E980C24912A4B1B4FF012275100012BA
:10A45800A4C87920E030E702792F304917121D2D62
:10A46800FAB40408E510700C79658008EA146510E0
:10A4780070027923E97E1812E9807E20E51230E720
:10A488000890B1C71285FA8016E51112A53E126B25
:10A49800C4201005201102800630120312A4F00512
:10A4A80010C3E558951050A7227E207F001285FA28
:10A4B80012A3CA7E007F0690A57012E9DEE5582235
:10A4C80075A7047583071269A8E51075F007A42419
:0EA4D80009FFF5177E00E51212E9807805EE07
:10A4E6002404FEE012E980D8F62212A5FB12A6117A
:10A4F600FD7C00AE1CAF1B126320BE003A8F00C36A
:10A50600E57A9513FFE55E9514FE402B7C007D28C9
:10A5160012632DC3EF98401F75F0058404FB24F9E0
:10A5260050027B067E2CAF170F12F2E30F12F2E3F6
:10A536000F12F2E30EDBEF2264B4602464B475F00C
:10A546003284C0F012E96DCE2404CED0E075F00559
:10A5560084C0F012E96DCE2404CED0E02302E96D6A
:10A5660090A56C0285FA2D2D2D000140FFFFFFE01E
:10A57600FFFFFFFFC25030124220283FE558F4602B
:10A586003A204803200934D250E559F510303309F2
:10A5960065586005204802051012A5C512A621754A
:10A5A600A7049006DCE512F0E511F0E517F0E510DA
:10A5B600F075A7049006E0ECF0EBF075A7002275A5
:10A5C600A7047583071269A87813E0F608B819FA84
:10A5D6009006D07811E6F008B819FAE51CF516F0E1
:10A5E600E51BF515F012A5FB9006DAE514F0E51368
:10A5F600F075A7002275A704758306E51023541E7F
:10A6060024B0F582E0F513E0F514221219F0E5BD49
:02A61600248797
:10A61800E5BD923B500224912212A61175F005A4C3
:10A6280085F012F511E4F519FEF51CF51D129D8A49
:10A63800C23DC2567F3C12DF03303D0575190080CC
:10A648007DDFF3E5596558700A301007EE24D350C2
:10A6580002D2568C1B8D1AE519FD24E250DEAE1C81
:10A66800AF1D7C00126320EFF51924F650CEAC1B09
:10A67800AD1A12DE3D20D1108E048F05E51975F054
:10A68800A7A4AEF0FF126320AC12AB117AA012623D
:10A698004BEB33FBEC33FC20D11AEF9BEE9C5014B0
:10A6A800C3E51213FCE51113FBC3EF9BEE9C4004BA
:10A6B800AC06AB07204807203B048C128B11900690
:10A6C800E2E519F012A709AC16AB157AC812622296
:10A6D800A912A8111263C6ED7005EC249E50057CE2
:10A6E800807B0822C3E57A305602E55C9513FFE5C6
:10A6F8005E305602E55D9514FEC3EF9BFBEE9CFCB5
:10A7080022AE16AF157C00E519FD24F6501A126327
:10A71800207C007D061262007C007D051263208F7C
:08A7280010EEF51724E95003BF
:10A730007517FF2212DE4E12A75112A79412E720BE
:10A7400012A7BA20480912A8A812A8D802A93B80CB
:10A75000747F177E2020480E748A204D1012676C7B
:10A76000500E742F8007746A305F02746712E9B26A
:10A7700075A7049006D07811E0F608B819FA7F178B
:10A780007E007812751905E60812E9B2EE2406FE7D
:10A79000D519F42275A7049006D8E0F516E0F51552
:10A7A000E0F514E0F513E0F512E0F511E0F517E03F
:10A7B000F510E0FCE0FB75A700227F187E26AC14A4
:10A7C000AB1302E7B29006E4E0F51CA3E0F51B7FB3
:10A7D0002A304E131219E6E5BF90B7B6B4010390C4
:10A7E000B9AF1285B580420F7E00745312E9809094
:10A7F00005CBE0F830E705E53F30E0091F7E00E8D3
:10A80000540F12E9989004EEE0FEF51EA3E0FFF568
:10A810001F12A850E51E24E9500C7E06742B12E985
:10A82000B27E0C12E9B212A880C20375172A7516FF
:10A8300027126B33202415205F15D2037F2A7E1E3A
:10A8400090A86E304E0390A87702E9DE205FEB22DD
:10A850007C007D3C12632DA805EF7F2A7E0812E85C
:10A86000B97E12743B12E9AE7E14E802E8B3070722
:10A87000384C9EBAF264380707387CE6C2E67C386A
:10A88000AC1CAB1B7A48305D027A27126222A91EEB
:10A89000A81F1263C6ED4C60027BFF7F207E28EB71
:10A8A00012E8BF7E3902AE287F2B90B75F1285F881
:10A8B000E517F46022AE17AF107C007D3C12632DCB
:10A8C000A805EF7F2A7E0C12E8B97E16743B12E9C8
:10A8D000AE7E18E812E8B322AE12AF117C007D0AFA
:10A8E00012632DA805EF7F207E3012E8B97E3A74FE
:10A8F0002C12E9B27E3CE812E9980F7E29744502D9
:10A90000E98074858007748720560274867E291238
:10A91000E9B2301707742D7E3A12E9B2227C007D2D
:10A920000A12632DA805EF7F2A7E3012E8B97E3A1D
:10A93000742C12E9B27E3CE802E99812AA6CE54850
:10A9400024F6500512A91D80B9E559046558600D1B
:10A9500012A91D12A902E559655860AA22A21792F0
:10A960003D8E1E8F188515179006D0E0F51185587D
:10A97000101510125334C3E51195105002F404F968
:10A9800024A65005C374B399F9E975F00584F92438
:10A99000EE5002791190AAACE993F5F0120808E59F
:10A9A000CC7004E930E702747F23A4A9F0E51B25ED
:01A9B000178F
:10A9B100FDE51C3516FEC3ED99F515EE9400F5166F
:10A9C10075A700758306E55823541E24B0F582E06F
:10A9D100A3F513E0F51412AA6C203D2C20172912BF
:10A9E10019F0E5BD2487E5BD5002249175F007A457
:10A9F100FB9518E5F0951E400FEB9FE5F09E400892
:10AA0100EF9518EE951E500EA23D9217AE1EAF188F
:10AA110012A91D02A902306B1012AA09E53F20E01C
:10AA21000774867E2212E9B22275A7009006E0E53E
:10AA310016F0A3E515F012A91D12A90674857E234F
:10AA410012E9B285581012A5C512A75112A7948C0C
:10AA5100168B1512A7BA12A6CF12A5B712E720902E
:10AA610006E2E0F51912A70902A8A8C3E57A305653
:10AA710002E55C9513FFE55E305602E55D9514FE37
:10AA81009217500312649DAC16AB157AC81262225C
:10AA9100A906A8071263C67E037FE7ED700CEB24BD
:10AAA10018EC34FC4004AE04AF032200172E4357C8
:10AAB1006C8092A4B6C5D3DFE6EDF3F8FD305E4FAE
:10AAC10030504C75A7009006E0E0A3FCE0FBECA23F
:10AAD100E79217402024FE50047F3B8022AE04AF52
:10AAE100037C007D1412632D74542F2017029F9F45
:10AAF100FF7462800C1264ADEC24FE50E07F6D7433
:10AB01003D7E0012E9807E017D197C0312AB11228A
:10AB11007F3D12F2E3EF2DFFDCF822E537B40206A8
:10AB2100E534243750292212F39E12EB5512E41D0D
:10AB310012ACA812DC9812E28812AD001269FE7FF5
:10AB4100207E2B12E55712EBE712F13012465E120E
:10AB5100E64612ABD6125D2E02F25120041EE579B3
:10AB6100FD24A050027D5FED24CD401E744520756B
:10AB71000C2DFFF51212ABAB1FBF44F922C39DFF91
:10AB8100F51212ABAB0FBF46F92220750EED24135F
:10AB9100FFF51212ABAB0FBF78F922C374779DFF9B
:10ABA100F51212ABAB1FBF12F922EF24BA400824F1
:10ABB10033FCC374329C1404FC24D750047C2380DE
:10ABC10009EC2375F005842413FC7E0512F2E30ED3
:10ABD100ECB506F822E59020E206E534243740037F
:10ABE10012AB5C7F457E047D1212F2E30EDDFA7F2B
:10ABF100437E00746412E9807F4F7D1212AC917F15
:10AC01003B7D1212AC917F597D1612AC917F317D43
:0DAC11001612AC917F637D1A12AC917F2763
:10AC1E007D1A12AC917F6D7D1E12AC917F1D7D1E33
:10AC2E0012AC917E057F1912F2E30FBF72F9780410
:10AC3E00E57924CD50027809E8305C0123F87F1BBA
:10AC4E0012AC807F6B12AC8018305C01187F25121D
:10AC5E00AC807F6112AC8018305C01187F2F12AC73
:10AC6E00807F5712AC8018305C01187F3912AC808F
:10AC7E007F4D7E00E875F00A847004E802E96DE805
:10AC8E0002E906EF6512600C7E04EE20E00712F278
:10AC9E00E30EDDF62212F31380F790B8757F287E4F
:10ACAE002C1285FA7E3B12E7C9AC5EAB7A7F307E02
:10ACBE0019C23D12E80890B7637F5D7E2D1285FAAA
:10ACCE0078B9C3E57A9618FBE55E96FC7F507E193F
:10ACDE00D23D02E808E51164B4700122E51112F1CB
:10ACEE00A07831790F7D0B12F2A61F1E90AD900247
:10ACFE00E9DEE5716012E57012F1A07831790F7D11
:10AD0E000412F2A20DBD0AF97F0112AD687F1D1269
:10AD1E00AD687E2312AD727E3F12AD727E247F1718
:10AD2E0012AD7C7E397F0212AD7C7E247F0712AD80
:10AD3E00867E397F1C12AD867E317F0212F2E37F52
:10AD4E001C12F2E37F0F7E2412F2E37E3E12F2E338
:10AD5E007F0C7E2E90ECD502E9DE7E2A12F2E30EF7
:10AD6E00BE39F9227F0812F2E30FBF17F9227D06D2
:10AD7E0012F2E30E0FDDF9227D0612F2E30E1FDD55
:10AD8E00F9220303E0A0E012DE4E7F1890AFA4126A
:10AD9E0085F87F217E01744112E9807F2A7E01743D
:10ADAE005312E9809005BEE0F51AA3E0F519A3E071
:10ADBE00F51EA3E0F51D851A1C85191B75172012AB
:10ADCE00AE45E519251DF51BF51DE51A351EF51CBD
:10ADDE00F51E75172912AE459005BA12AE35AC1A8E
:10ADEE00AB1975172012AE039005BC12AE35AC1E12
:10ADFE00AB1D751729EC7006EB24CD4001227A4865
:10AE0E00305D027A271262221263C6ED4C60012277
:10AE1E00AF177E07EB12E8657E1A0F90B938305DDA
:10AE2E000390B93B0285FAE0FEA3E0FD12A16AC3CE
:10AE3E00EB9DF8EC9EF922751627026B6412A16A3F
:10AE4E0075A7049005B478737F06E6F008DFFBEC77
:10AE5E00F0EBF0E0E0E0FCE0FDE0FEE0FFEF2DFFC8
:0DAE6E00EE3C9005C0F0EFF0801275A704D7
:10AE7B009005BAE0FBE0CBF0EBF0E0E0E4F0F0752E
:10AE8B00A7002275A7049005B478647F06E0F60846
:10AE9B00DFFB75A700126D739005BEE51CF0A3E5F3
:03AEAB001BF02277
:1046F000D23C799E77008002C23C129D8AE4F5107C
:10470000F511F512F513F514F515F516F517C23D6B
:10471000124A3D203D1F124A3D203D19E51F30E55C
:104720001130E40E124767303C08799EE724F550BB
:104730000122D510DBAE14AF157C00AD121262FA67
:104740008F55AE16AF177C00AD131263201265278C
:104750007E00E55530E7011E2DFFE43E30E7027F85
:1047600000740A2FF55622C235E51CAF1DBFFF05A8
:104770000FD235F404FABF003F532CF8E518AF19F7
:10478000BFFF050FD262F404BF002D20E72A205B93
:104790000123FF24AA4021E51AAE1BBEFF050ED25D
:1047A00061F404BE00128547F0A4E5F020E709207B
:1047B0005B0123FE24AA5001227C807B803051665D
:1047C000302163C006C0078AF0E545A4AEF0FFE5DE
:1047D00056205B011375F009A4ACF0FD1263207440
:1047E000FFBE0001EFFA24C050027A3FD007D00686
:1047F000E55212F1A0303504B2D5B2D1EA8CF0A462
:1048000030E70205F0748025F020D10495F095F092
:0A481000FCEA8BF0A430E70205F08B
:10481A00748025F030D50495F095F0FBC3EC2F2079
:10482A006203C39F9FFFEB2E306103C39E9EFE204F
:10483A003C64200C051248D440641248B6405F120A
:10484A00F2E3E51EFD24FB50550E12F2E3ED24F6C9
:10485A00504C1E1F12F2E3ED24F150421E0F12F2C9
:10486A00E3ED24EC50380F12F2E3ED24E7502F1F4A
:10487A001F0E0E12F2E3ED24E250231E0F0F12F266
:10488A00E3ED24DD50180E12F2E3ED24D8500F1E8A
:10489A001E1F1F02F2E31248B64003799E0722E95F
:1048AA00242AFFE82461FE1248D4401DEF24604008
:1048BA0018243F5013EE2460400F243F500AEF247F
:1048CA00D6FFEE249FFEC322D322532CF8432C0496
:1048DA00EE10E706D2E7F404D261FE24D340EAEFF1
:1048EA0010E706D2E7F404C262FF24D340DBEFB537
:1048FA0006005003CED26070057480FE8062FF24E9
:0D490A00FD50609049C0938EF0A4AAF033D8
:10491700CA33CA33CA33CA33CA33FA9049EA938FC0
:10492700F0A433C5F033CA904A0B93FB124988951C
:1049370070500224B412F1A0EA8BF0A430E702050C
:10494700F0C3748095F020D50425F025F0FEEA8C9D
:10495700F0A430E70205F0C3748095F030D1042548
:10496700F025F0FFC3227A01EE6F70097B16BF02B4
:10497700BB7A0380B7BF01047B0080B07B0D0A8040
:10498700ABE52C540723C390499273800E800E80A9
:1049970024801E8010800A80108012EB22742D9BC9
:1049A70022742D2B22745A9B22745A2B2274879BB4
:1049B7002274872B2274B39B22FFFFCCAA928071AB
:1049C700665D554E4944403C383533302E2C2A28F5
:1049D700272524232221201F1E1D1C1B1A1A1918E4
:1049E7001817178181818282838384858687898AC4
:1049F7008B8D8F90929496989B9D9FA2A4A7A9AC0C
:104A0700AFB1B4B400010203040405060708090A9C
:104A17000A0B0C0D0D0E0F0F101111121313141496
:104A27001515161616129C8412CBE8E4F5F7E4E583
:104A3700F7D2B264C022203D07124A2C7003D23D40
:104A470022056D056D12CBE87D008DF7E485F71F14
:104A57008DF7C3E5F79573F5188DF7E4E5F79574CA
:104A6700F5198DF7E4E5F78DF7C3E5F79576F51AB0
:0C4A77008DF7E4E5F79577F51B8DF7E46B
:104A8300E5F78DF7E4E5F7F51E8DF7C3E5F7957ABE
:104A9300F51C8DF7E4E5F78DF7E4E5F7D2B2543F63
:104AA30030E50244C0955EF51D156D156DE51024C6
:104AB300784001227E00AF55EF30E7011E0512E575
:104AC3001FA2E592D5400EE515951EF515E5149444
:104AD30000F514800BE515251EF515E43514F514C2
:104AE3007800E51E600620D50318F404C39FF5F093
:104AF300E89E30E701220513E5F0A42517F517E535
:104B0300F03516F51622303D03D23D22124A2C60B1
:104B1300F8124A2C60F3E546600A124A2C60EA1246
:104B23004A2C60E5056D056D056D12CBE87D008DA2
:104B3300F7C3E5F79573F5188DF7E4E5F79574F585
:104B4300198DF7E4E5F78DF7C3E5F79576F51A8D3B
:104B5300F7E4E5F79577F51BD2B2156D156D156D75
:104B630022307424129D8AC23D75101E124B0920F7
:104B73003D167902124BD0400CA806A9071248A98A
:104B8300400312F2E3D510E422200F4030123D20FF
:104B930006CF304806200C03204FC6E54679026055
:094BA30014790614600F79161450
:104BAC00600A79361460057976147017129D8AC2E2
:104BBC003D7896124B09203D0A124BD0400312F25D
:104BCC00E3D8F022532CF8AB18E519FC339262129F
:104BDC004C22BC002BEB89F053F00784FF24DF4000
:104BEC001FAB1AE51BFC339261124C22AA471262CE
:104BFC004BBC000CEB89F053F00784FE24DF500211
:104C0C00D32274562F2062029F9FFF741F2E306197
:104C1C00029E9EFEC32250031264ADE920E40122E1
:104C2C00C3EC13FCEB13FBE920E50122C3EC13FCF2
:104C3C00EB13FBE920E60122C3EC13FCEB13FB2284
:104C4C0074542F2062029F9FFF741D2E3061029EB0
:104C5C009EFE2279B4203249201D46EFB506009203
:104C6C0060AC06AB074004AC07AB06904CAEEC2333
:104C7C0004938BF0A4A9F0EC23938BF0A429F99066
:104C8C004D0E93C9904E0EE52C54079313E9500129
:074C9C00F4904E16F9E52C1F
:104CA3005407932975F0B484A9F022FFFFFFFF7F17
:104CB300FF55553FFF33332AAA24921FFF1C711956
:104CC300991745155513B1124911110FFF0F0F0E07
:104CD300380D790CCC0C300BA20B210AAA0A3D0922
:104CE300D8097B092408D30888084207FF07C107AE
:104CF300870750071C06EB06BC06900666063E06B1
:104D03001805F405D105B0059005720000000000F8
:104D13000101010101010101010202020202020279
:104D2300020203030303030303030304040404044D
:104D33000404040405050505050505050506060621
:104D430006060606060606070707070707070707F7
:104D530008080808080808080808090909090909CA
:104D6300090909090A0A0A0A0A0A0A0A0A0A0B0BA2
:104D73000B0B0B0B0B0B0B0B0C0C0C0C0C0C0C0C78
:104D83000C0C0C0D0D0D0D0D0D0D0D0D0D0D0E0E51
:104D93000E0E0E0E0E0E0E0E0E0F0F0F0F0F0F0F29
:104DA3000F0F0F0F0F101010101010101010101005
:104DB30010101111111111111111111111111112E1
:104DC30012121212121212121212121213131313BC
:104DD300131313131313131313131314141414149B
:104DE300141414141414141414141515151515157A
:104DF300151515151515151515151616161616165A
:104E0300161616161616161616161600FFFF00FFB0
:104E13000000FF002EB5875B2D5A88E537606C14C0
:104E23006036B402507F347E12E53424375046F89E
:104E3300904F6012E9DEE824FC501179A1E77E056A
:104E430090B44A20E70390B4540F803A24040F7EB1
:104E53002312E99FD26480627F357E02E5342437D2
:104E6300401410641090B34D30081B1285C77E1A8E
:104E730090B735801122700590B35F800990AFD150
:104E8300200C0390AFDD1285C780C97F35E534243C
:104E930033402A2404501B7D0F600C7D1E146007D1
:104EA3007D3C1460027D78ED305D02C3137E2B12CE
:104EB300E8657E0090B3601285C702F2517E052437
:104EC300FE500590B1B4800990AFB4200F0390AFAA
:104ED300C01285C780E4E546604A14603C14602E26
:104EE30014602014601290B96C205D41904F597F7B
:104EF300367E3412E9DE803C90B96C305D0390B9A4
:104F030068802A90B968305D0390B964801F90B9B6
:104F130064305D0390B960801490B960305D039094
:104F2300B95C800990B958305D0390B9547F367EDF
:104F3300331285FA7E3C7422305D02748302E9B237
:104F4300305D0890B944305BE4800690B94C205B37
:104F5300DC90B94880D70508B28D8DB5BA09100623
:104F6300000A10F248922492249224F2480A10066E
:0E4F730000305E5220434F20284CE55864FF6A
:104F81006046E54824F640407F3FE55804F9C23DBC
:104F9100124FCA121D2D601AB404047401D23D755A
:104FA100F003A4243CB5070A7E3A303D027E361256
:104FB1004FCC0F0F0FD9D7E55975F003A4243EFF4D
:104FC100124FCA0F0F124FCA227E3D12F2E30EBEDC
:104FD10040F922C248C249305E56202853E5586440
:104FE100FF604DE54824F64047121D2D6042D2492D
:104FF100B40402803B1465597036D248304E31E515
:10500100596558602B3074281250371219E6E5BFE4
:10501100B4011DE5BD20E618202416205F1290067C
:10502100E4E0700CA3E024CE40062425500205598B
:1050310022305FFC80E820113375A7009006E4E080
:105041007028A3E0302402F404305F02F404240445
:10505100F924F74015E924FC4003D26C22700122A7
:10506100306C097536A7D22ED22FC26C22305E0861
:10507100307405E558B4FF0122C244C24D78007571
:10508100A7047583071253B688188A1E8E168F17C8
:10509100C23EC23BE54824F65003025147D23EE5E9
:1050A1005860F7E8655970F22048EF1251FC30D191
:0750B1003BAE16AF17A81873
:1050B800E5467055120808E5CC49604DD244E5CC68
:1050C8007033E924CD402EE975F038A4ACF0FB121A
:1050D800643C12643CEBFDF51112515D304D2CC25D
:1050E80006C23B8043E546705C120808E5CC7005B3
:1050F800E924CD5050125B6575A704758307A8187D
:105108001253B68A1E8E168F1780371219E6E5BD20
:10511800A2E0B3923B50113074281248A94026A946
:1051280007A806D20612DEEA1251791251701251FE
:10513800B9890788061E1F9053B112E9DE80063030
:10514800D103125191A81808C3E55898400302509A
:105158008075A7002274562F2062029F9FF9741F42
:105168002E3061029E9EF822E51865586001227D66
:10517800057A00EA12F1A012F2A60A0AED24F2401A
:10518800020A0AEA244C50EB22AE16AF17124C4C16
:105198001E303E021E1EE51E12E980EE2404FEE5C6
:1051A8001212E980303E09EE2404FEE51312E9806C
:1051B80022E5186558603CC001C000C012C01385C4
:1051C8001810125334D013D012D000D001E510308B
:0751D8003B07C39570500274
:1051DF0024B412F1A0203B07AE16AF1712515DE5B4
:1051EF00112402FD7A0612F2A61DDAFA22121D2DE3
:1051FF00B40457E87054121A04E5BD604D78C6A682
:10520F001308A61208A62C12DC8575A70475830750
:10521F0075100112697912DC7F1510126979126508
:10522F00938E628F6312661B8B1C8A1B12DC8B2082
:10523F00320E1252E4203B08D24D1275C412525A4C
:10524F0078C6861308861208862C22121A04AABD65
:10525F007C027BB312624B8C128B13AA1DA91F12F7
:10526F00628DA91CA81B1263C68C1D8B1FAC12ABC1
:10527F0013AA19A91A12628DA91CA81B1263C68C36
:10528F00198B1AE56E251AF9E56D3519F8C3E56E18
:10529F00951AFBE56D9519FAC3E554951FFDE56F5A
:1052AF00951DFCE554251FFFE56F351DFEE52C23ED
:1052BF00652C30E206ECCEFCEDCFFD75A704900512
:1052CF00C2E8F0E9F0ECF0EDF0EAF0EBF0EEF0EF21
:1052DF00F075A70022D23BC3E5649573C56595743D
:0E52EF00F564E5669575600404600822E564C8
:1052FD0024E0500822E5642420400122C3E567958F
:10530D0076F567E5689577F566E569957860090442
:10531D00600122E566F48002E5668562F0A474E022
:10532D0025F04002C23B2212DC8575A70475830768
:10533D0012697912DC7F0510126979C02C126992FD
:10534D00D02C891002DC8B30125120064E7800755E
:10535D00A7047583061253B630D139124C4CE5466D
:10536D0024FE500A0E0F9053AC12E9DE8026EA702F
:10537D0007745D12E97C801C75F06484ADF0700FCC
:10538D00ED75F00A847008E5F00E12E96D80051ECA
:10539D00ED12E90008C3E55A9850B475A700220331
:1053AD000340A040030340E040D2D1E8C4F582E0C1
:1053BD00FA797312540F30D146AF06532CF8EDBF66
:1053CD00FF07F40460390FD262BF0033125543401A
:1053DD002E797612540F30D126E5822403F582E022
:1053ED00F512E0F513EEA2E713FEED13BEFF07F481
:1053FD0004600C0ED261BE0006125560400122C23F
:10540D00D122C3E09709FDE09709FEE097600904FA
:03541D00700AEE24
:1054200030E7068007EE30E703C2D122E546600E82
:1054300014600BF9EDCEA2E713CE13D9F8FD227C50
:10544000007B44E54660207C007BCC1460197C0125
:105450007B981460127C037B3014600B7C067B60AD
:105460001460047C0C7BC08C148B157AE9126222C8
:10547000A8471263C48C168B1775C70075C60475D0
:1054800010DF75B901E5BC20E76FF51385BD120586
:10549000C605C675B901532CF8C3E5BE9573FBE587
:1054A000BF9574FC05C675B901E5BC9575FD500541
:1054B000D2621264B5C3E5159BE5149CE49D4033AC
:1054C0008C198B18C3E5BD9576FBE5BE9577FCE599
:1054D000BF9578FD5005D2611264B5C3E5179BE511
:1054E000169CE49D400D8C1B8B1A12550AE5322444
:1054F00028401305C6E5C68006E5C62404F5C67037
:105500000205C7D5100122025482AE19AD181254FB
:105510002CED125543AE1BAD1A12542CEE13ED13A5
:10552000125560124C4CE54624FB50080E0F905368
:0B553000B102E9DE1EE51312E980EE77
:10553B002404FEE51202E98075F0067FFDA946B949
:10554B00000575F0027FFF84C5F02F500205F0C5F2
:10555B00F0FF24DE228547F0A430E70205F0E5F0EA
:10556B00A946B9000280050475F00384FE24E022ED
:10557B00E537B4020122E5377002D23964027002BA
:10558B00C239E53724FC799EE76005640B600C2279
:10559B00D27E20081E401C107F1022D27F200813C1
:1055AB004011107E01227537012275370020390317
:1055BB007537022275F9FF75FB00801175FBFF75BE
:1055CB00F9FF801F1222582053F2125600759E8548
:1055DB00759D2D8014125600759E84759D2D800926
:1055EB00125600759E83759D09C2AC759852C26D9B
:1055FB00C26EC26F22122258C253E4F5F9F5FB308A
:10560B00340215FB221256A5851617203D01227F69
:10561B005A90AEC81285B57F64E5166404700C9081
:10562B00AEE01285F812F25102F20090AED4128560
:10563B00B57F6E7E0890B9341285C71229EE12F22F
:10564B00517515B87514047F6E7E20C224A815E819
:10565B002404F9C23DE71256ED203D06E612E9B2ED
:10566B008008E6129320E8A815F60515EE2406FE31
:09567B00D514DA851716122A4332
:1056840012F25110000510018D80F878B8121A0E2C
:1056940086BC0886BD0886BE0886BF1257AF12F3C3
:1056A4009E121A0EC23D75160078B87F4B7E089084
:1056B400B9341285C77E20E5BC12E9B21256E47EE5
:1056C40026E5BD12E9B21256E47E2CE5BE12E9B21B
:1056D4001256E47E32E5BF12E9B21256E402F251E8
:1056E400F608080808F618181824D0500524F640BF
:1056F4000122D23D05162275C70375C6FE128533F5
:105704001257AF75C6FC75BC2675BD6475BEA97508
:10571400BF701257AF75C6FB12853375BC64125740
:10572400AF75C6FA75BC1475BD1475BE0075BF0C93
:105734001257AF75C6F975BC4E75BDBF75BE007501
:10574400BF191257AF75C6F875BC0A75BD7E75BE14
:105754000075BF011257AF75C6F775BC0175BD233F
:1057640075BE4575BF671257AF75C6F675BC027531
:10577400BDAB75BE0175BF011257AF75C6F5128575
:105784003375BE0275BF0A1257AF75C6F41285335E
:1057940075BCE11257AF75C6F312852F1257AF15BA
:1057A400C61257AF15C61257AF15C675B90575B9E8
:1057B4000222751500128C3675B901E5BC6481604E
:1057C400031285160515E515242050E975C70375E0
:1057D400C68075B90505C6E5C6241C50F51257E701
:1057E400028A8CE4F5C7F5C6742612853475BD4E5D
:0757F4001258011257FEE4F8
:1057FB001257FE1285341257AF05C6227F3E7E002C
:10580B00E54B12E91C7E10E54C12E91C7E20E54DA0
:10581B0012E91C7E30E54E12E91C227F467E00E524
:10582B006C12E91C7E10E56B12E91C7E20E56A12F6
:10583B00E91C7E30E57F12E91C227F2E121A1D1205
:10584B002A4E40167F2D1285AC1258681219E1E4CE
:10585B00F5BCF5BD75BE021257AF0205527F0E7532
:10586B006F0280057F02756F00E4F56EF56D7406AF
:10587B00129DD774D8129E0FD2B2129F88056FDF7C
:10588B00ED22E4F56CF56B756A00E56B700C7F79B6
:10589B007E32E56C12E8BF12F25112CBC1E56B24DC
:1058AB0004F56BE4356CF56C30E7DF221258BD0262
:1058BB0002A012F39E7F5A7E0590B7441285C71241
:1058CB00F251125F35C210D214D215C255121A13EF
:1058DB0085BF6C85BE6BE56B54036005129C4B80DA
:1058EB00F5856CBF856BBE75B90575B902129F172F
:1058FB0012641F7B17756F7FE4F56EF56D75800273
:10590B00C2B275F753856FF7856EF7856DF7A4D225
:10591B00B212CB5ABB172B756A007539FC75F08424
:10592B0012CBD67C07783986F708DCFBD2B2756AC6
:10593B001E75F08412CBD68EF7A48FF7A4D2B27556
:0E594B006A0012CBC112CB54E56E2404F56E37
:105959007C04129C4BDCFBDBA6121A1385BEBC85AA
:10596900BFBD856BBE856CBF75B90575B90279B8C0
:1059790077C309A73A09A73B09A73C09A73D09A786
:105989003E0977000977180977050977CE0977273E
:1059990009773B09775B09770009A7BD09A7BC12FD
:1059A9009F17029F3ED214D2151259BCC214C215B8
:1059B90002026D756F00756E00756D007403129E9D
:1059C9000F784075A700900700E4F5F7C2B2C2B29C
:1059D900E5F7F0A3D8F3D2B212F39E85354B856F64
:1059E9004C856E4D856D4E7F0012580975A7009044
:1059F900070078107F09E8540370020F0FE0F54B98
:105A0900A3E0F54CA3E0F54DA3E0F54EA3C083C098
:105A190082125809D082D083EF2407FFD8D812F216
:105A29005110000910012F10020280F522100214F2
:105A3900E53524964002800C756D00536EFCE56EC9
:105A490024FC800AE56D24C0F56DE56E34FFF56E22
:105A5900E56F34FF8026100214E535249640028054
:105A69000C756D00536EFCE56E2404800AE56D2407
:105A790040F56DE56E3400F56EE4356F540FF56F42
:105A89000259C5D214D215125A9AC214C215020269
:105A99006D756F00756E00756D0012CBE8784075F5
:105AA900A700900700E4F5F7E4E5F7F0A3D8F6D2EC
:105AB900B212F39E85354B856F4C856E4D856D4EC3
:105AC9007F0012580975A70090070078107F09E830
:105AD900540370020F0FE0F54BA3E0F54CA3E0F57A
:105AE9004DA3E0F54EA3C083C082125809D082D0DD
:105AF90083EF2407FFD8D812F25110000910012FA3
:105B090010020280F522100214E535249640028025
:105B19000C756D00536EFCE56E24FC800AE56D245E
:105B2900C0F56DE56E34FFF56EE56F34FF80261024
:105B39000214E53524964002800C756D00536EFC05
:105B4900E56E2404800AE56D2440F56DE56E3400A8
:105B5900F56EE4356F547FF56F025AA32074012264
:105B6900D24475A700758307E559C454F02407F595
:105B790082E0F51A244C40E7A3E0F512A3E0F513FF
:105B890012080889381219E6E5BDA2E0923BE51A28
:105B990040069570500224B4F51A203B05D206122E
:105BA900DEEAE51A125CC8E5152437F51DE435145B
:065BB900F51CE51724377E
:105BBF00F51FE43516F51E85CC12853813AC12ABE4
:105BCF00137A0412621475380124FA401A05382426
:105BDF0002401405382401400E05380538240140D1
:105BEF0006053805380538C3E51A945A500224B40F
:105BFF00F51AC23BC23CC23D751B00A23B823C4022
:105C0F006D203B2CE51A75F008A4951BFBE5F030D1
:105C1F003D04940180029400FC5008EB24A0FBEC9F
:105C2F003405FC125CCF125C7E923B4003125CA1E8
:105C3F00203C2CE51A75F008A4251BF9E4303D0132
:105C4F000435F0FAE994A0FBEA9405FC5004AB018B
:105C5F00AC02125CCF125C7E923C4003125CA1E559
:105C6F001B2538F51B5094203D04D23D808D22E535
:105C7F001F2517FEE51E35167016EE24914011E50F
:105C8F001D2515FFE51C35147006EF2491400122E8
:105C9F00D3228E027C8A7B3B126222ED2402FE8F7E
:105CAF00027C8A7B3B126222ED2439FF02F2E3125F
:105CBF0065868031126579804675F008A4ACF0FBDB
:105CCF00751900C3EB9468F9EC9401FA40080519B3
:105CDF00AC02AB0180ED8C108B11531903E5192029
:105CEF00E0CD126579125D23AF05E51924FE50034F
:105CFF0012649D8E168F17E51920E0B81265861273
:105D0F005D23AF05E51914600614600312649D8EC0
:105D1F00148F1522AC06AB07AA12A91302628D12BB
:105D2F005E10203D4974857F227E0812E9B27E08FD
:105D3F0030173CAC1EAB1FEB2418EC34FC402F1279
:105D4F0061F3E51B60077F207E0812E9CD7F207E7F
:105D5F0010E51A12E9CD7F237E17742E12E9AE7F5C
:105D6F00207E1BE51B7011E519C2E012E9CD227FE1
:105D7F00207E0E740A02E9CDE51975F0058475F0E1
:105D8F0005A402E9CD125E10203D5E74857F227E50
:105D9F003A12E9B2301753AC1EAB1FEB2418EC3498
:105DAF00FC4046EC7033EB249C402E7E2D125E029D
:105DBF0012643CC0E07F2A7E2EEB12E9CD7E39D0F3
:105DCF00E0C2E012E9CD7F347E3712F2E31E12F209
:105DDF00E31F12F2E30E02F2E37E30125E02126450
:105DEF003CEB7F2A7E3112E2DC227F2A7E39740A55
:105DFF0002E9CD7F2912F3130FBF34F90EBE40F322
:105E0F0022D23D3012661219F0E5BDF51C75F00A6D
:025E1F00A4F8E5
:105E210024E15002781EE4FCFBFEFFC23D129D8A74
:105E3100125E7C203D44D8F8751DCEE51C14600926
:105E4100751D9C146003751D6AC217EC30E705D2FD
:105E5100171264AD8C018B00E9487003D23D22EE2C
:105E61007008EF251D4003D23D22AC06AB077A1C1A
:105E71001262221263C68C1E8B1F22203D07124A1A
:105E81002C7003D23D22056D12CBE8E4F5F7C2B2C6
:105E9100C2B2ADF7F5F7C2B2C2B2E5F7FAD2B2308B
:105EA100E4E3ED2FFFE43EFEE56D2408F56D12CB32
:105EB100E8E4F5F7C2B2C2B2ADF7D2B2EA30E50812
:105EC100EB2DFBEC3400FC22C3EB9DFBEC9400FCBE
:105ED10022D2A47F3212F21DC2A412EE6912F25133
:105EE10012F206C214C2151255BF74C012F0BB746F
:105EF100A312F06B748F12F06B125F1874C012F062
:105F0100BB75A704905F227F10E49312F06BDFF959
:105F1100125F1875A70022E53812F06B74CA02F0FF
:105F21006BA29494859C8080808080818380819EF7
:105F31008075A60A125EE4D269D2ACE5A624FA50B5
:105F41000C306DF712F0EDB4E0F1125F7AC2ACC221
:095F51006975A6FF22D21EC2747C
:105F5A00C273E4FDF571F570C22D1255BFD2AC12B1
:105F6A00F0EDC5F07005DDF7C2AC22C5F0B4E0EF84
:105F7A00F538E4F53212F0E8A2E19273A2E29274E3
:105F8A0075A7049004B4F012F0E8C2D1126103209C
:105F9A00690330740B8D758E748F73E514C4F57DA7
:105FAA0012618312610320690330740C8D788E7735
:105FBA008F76E514257DF57D126183D2D1126103B6
:105FCA00EEF0F55DEFF0F55C207303E4FEFF79BCBB
:105FDA00A70609A70712F0E87D0A1261708F71EE11
:105FEA0060037571FF7D14126170C22DED24F150AA
:105FFA00010F240A5002D22DBFB4027F008F701203
:10600A00F0E8F05407C52E54F8252EF52EE57170E8
:10601A000EE4F571F570C22D9004BFF0F0F0F012A5
:10602A00F0E8E5386009D21EC27412CDDD8005C2DF
:10603A001E12CDD912F0E8B4E1FA75A7049004C48F
:10604A0012F0E8F012F0E8F0F53A12F0E8F0F53B59
:10605A0012F0E8F0F53C12F0E8F0F53D12F0E8F045
:10606A00F53E12F0E8F0F53F12F0E812F0E8B4E27B
:10607A00FA12F0E8F07E0C12F0E8FF12F0E812F0E3
:0C608A00E812F0E812F0E820E1027F00CC
:10609600EFF012F0E8DEE412F0E8B4E3FA12F0E80A
:1060A600FF12F0E8CF60027F7F9004E4EFF0E4F0A7
:1060B60012F1189004D812617012F0E8B4EAFAC22C
:1060C600AC75A7049004DAE561F0E560F0E55EF0F2
:1060D600E57AF0E579F0E52EF0E55FF0E57BF0E5B1
:1060E60051F0207412E4F571F5709004B4F0900448
:1060F600BDF0F0F0F0F0F075A70002A0DB12F0E8BA
:10610600FC12F0E8FD12F0E8FE12F0E8FFECA2E661
:1061160092E7921713FCED92E713FDEE92E713FE5A
:10612600EF92E7301701F4F513ECA2E713FCED92BA
:10613600E713FDEE92E7301701F4F512ECA2E71330
:10614600301701F4F510ED92E7301701F4F511124E
:10615600645D20D10E8C1C8D1D8E1E8F1F12D1E505
:1061660012645D30170312D1BF2212F0E8C313FE8A
:10617600F012F0E892E7FFF07C0002632DAC1CAD54
:106186001DAE1EAF1F30170312D1BFECF0EDF0EEBF
:04619600F0EFF02214
:00000001FF
